:020000040800F2
:200000000000012069AE050805AF0508F93304085D34040805AF050805AF05080000000083
:2000200000000000000000000000000005AF050805AF05080000000005AF0508E5DB0308B2
:2000400005AF050805AF050805AF050805AF050805AF050805AF0508BD350408B535040826
:20006000AD350408A53504089D350408659E0508559E0508459E0508359E0508219E050822
:200080000D9E0508F99D050805AF050805AF050805AF050805AF050805AF0508953504086A
:2000A000A18005089981050891800508C1810508898105087981050869810508E5A10508D6
:2000C000F1A10508CDA10508D9A1050805AF050805AF05087DDC03086DDC03085DDC030801
:2000E0008D35040805AF050805AF050881800508B180050805AF0508D9800508E59D0508AE
:2001000005AF0508057005085981050805AF05084DDC03083DDC0308E98005081DDC000825
:20012000D19D0508BD9D0508A99D0508959D0508819D050800000000000000000000000020
:20014000000000000000000000000000B5E000086D9D0508599D0508459D05082DDC0308E5
:20016000B5A10508C1A1050805AF050805AF050805AF050805AF05080000000000000000A9
:2001800005AF050805AF050805AF050805AF050805AF050805AF05080000000005AF050818
:2001A00000000000000000000000000005AF050805AF050805AF05080000000000000000FC
:2001C0000000000000000000000000000000000000000000000000000000000005AF05085E
:2001E000C0A90500010000000E02010002000000245301208853012000000000FC300708AE
:200200008453012014020100050000004C2B01209053012000000000FE3007088C530120F1
:20022000031101000A000000D85201209C53012000000000850F0108985301202320010057
:2002400010000000A8520120AC53012000000000DD6D0208A85301200D1001007000000055
:2002600030520120C053012000000000FD570308BC530120FD01010024000000B4510120CF
:200280003454012000000000B3C3030830540120FB01010001000000705101205C540120DE
:2002A0000000000079BF040858540120FC010100090000003C5001206454012000000000A0
:2002C00081BF040860540120F7010100060000001050012074540120000000000431070850
:2002E00070540120F90101000400000000500120805401200000000021C403087C540120D3
:2003000034000100100000002C4F01208854012000000000957502088454012011020100DE
:2003200008000000044F01209C540120000000000A310708985401201212010004000000B0
:20034000FC4E0120A85401200000000012310708A45401201830010038000000C44E0120F6
:20036000B054012000000000E1C70408AC540120000201000B000000484B0120EC54012060
:2003800000000000BDBF0408E8540120FF21010005000000EC4A0120FC540120000000008A
:2003A00059BF0408F85401200812040014000000F84A01200855012000000000E5BF0408E9
:2003C000045501201302010004000000442B01202055012000000000163107081C5501207B
:2003E000FA010100030000004C4A01202855012000000000DDBF0408245501202A0201003A
:2004000008000000404A012030550120000000001A3107082C55012020520100080000000C
:20042000F84901203C55012000000000B9750208385501200610010024000000D449012049
:20044000485501200000000065C00408445501200C02010004000000704801207055012021
:200460000000000069BF04086C550120FE010100140000008C340120785501200000000083
:20048000C5BF0408745501200B3001001A000000BC8F0120C8910120000000002431070842
:2004A000C49101201F50010024000000808F0120E89101200000000040310708E491012052
:2004C0000502010004000000309001201092012000000000643107080C9201201B200100CD
:2004E0000C0000002C950120CC9F012000000000FD740108C89F012021020100F00000006C
:200500005C930120DC9F012000000000A9810108D89F01203710010030000000E89C012047
:20052000D0A001200000000068310708CCA001201610010006000000E896012004A1012063
:20054000000000009831070800A101202F10010022000000A49F012010A101200000000069
:200560009E3107080CA1012023220100100000004C96012038A1012000000000C03107087C
:2005800034A101201E00010009000000349601204CA1012000000000D031070848A101202A
:2005A000052001000C000000BC9601205CA1012000000000DC31070858A1012012300100FF
:2005C000100000001C9601206CA1012000000000E831070868A10120FD0701007C00000037
:2005E0002092012080A10120000000006D6E01087CA10120F59101006C000000E09201203E
:2006000000A2012000000000CD800108FCA10120261001000E00000080A2012070A2012048
:2006200000000000716C01086CA201201400010005000000E4B501200CB6012000000000EE
:20064000F831070808B60120012001000C000000D0AA012018B6012000000000FE3107088D
:2006600014B601200C400600E400000084A9012028B601200000000045FF020824B60120C3
:200680000A9001002400000040A9012010B7012000000000956D02080CB701200E30030078
:2006A000BC0100007CA7012038B7012000000000D575020834B701201310010004000000A1
:2006C00070B30120F8B80120000000000C320708F4B801200101010004000000B4A6012069
:2006E00000B901200000000000000000FCB801200001010004000000ACA6012008B90120F0
:20070000000000001032070804B901200201010003000000A8A6012010B90120000000004A
:2007200089FF02080CB90120220201001C010000BCB0012018B9012000000000B9C80408F3
:2007400014B90120010201000B000000C0A6012038BA012000000000ADBF040834BA01207B
:20076000020201000300000048AB012048BA0120000000000000000044BA01201B020100FD
:200780001000000024AB012050BA01200000000051C004084CBA0120150010007000000055
:2007A00074C7012038C80120000000000000000034C801202A0008006000000084C60120A2
:2007C000ACC80120000000006D750208A8C801202C0004001000000020C9012010C90120C3
:2007E00000000000497402080CC901202920140078000000FCC3012034C901200000000069
:200800000000000030C901201A0001000E00000020C30120B0C901200000000014320708A2
:20082000ACC901202B00120024000000FCC20120C4C90120000000001D740208C0C90120EF
:20084000190201001000000000C20120ECC90120000000009DBF0408E8C901201C02020059
:200860001C00000034C0012000CA012000000000C5C50408FCC90120283001001600000071
:2008800050C0012020CA012000000000CD7602081CCA01200A02010014000000B8D40120FA
:2008A000D4D401200000000011FF0208D0D40120101001000200000040CE0120ECD401205D
:2008C0000000000022320708E8D40120F83101000600000048CF0120F4D401200000000087
:2008E00024320708F0D40120030001000100000058CF012000D5012000000000000000006B
:20090000FCD401201900010005000000F8CD012008D50120000000002A32070804D501207E
:20092000020001000C00000020D6012074D80120000000000000000070D80120F6210100A3
:200940000C000000BCD7012084D80120000000003032070880D8012025201E002C010000E0
:200960002CD6012094D80120000000000000000090D8012029020100400000004CD5012090
:20098000C4D90120000000003C320708C0D901202C020100040000003CD8012008DA0120F7
:2009A000000000007C32070804DA01202802040004000000C8E10120A0E7012000000000D7
:2009C0004DC004089CE701202702040004000000C4E10120A8E701200000000041C00408A6
:2009E000A4E70120160215003F000000B8DA0120B0E701200000000099BF0408ACE701205C
:200A00001A0201003C0000007CDA0120F4E70120000000003DC80408F0E7012003120100EB
:200A20003D000000C8E3012034E80120000000008032070830E8012038200100030000001A
:200A400048DA012078E8012000000000BE32070874E8012004000800800000003CE9012084
:200A6000BCEA012000000000000000003CEB01200B2201003D000000A4EE012098F401209C
:200A800000000000C432070894F401200D1201001400000070F40120DCF4012000000000FE
:200AA00004330708D8F401201E0201000600000004EF0120F4F40120000000001833070865
:200AC000F0F401201D0202000600000010F4012000F501200000000000000000FCF401209E
:200AE000061204001800000018F401200CF501200000000055C6040808F501201F02080005
:200B00001000000038F5012028F501200000000011BF040824F501202700010004000000F7
:200B200020EF01204CF50120000000001E33070848F50120100201000100000048190220CE
:200B400044190220000000002233070840190220FFFFFFFFFFFFFFFFFFFFFFFFFFFFFFFF47
:200B6000FFFFFFFFFFFFFFFFFFFFFFFFFFFFFFFFFFFFFFFFFFFFFFFFFFFFFFFFFFFFFFFF95
:200B8000FFFFFFFFFFFFFFFFFFFFFFFFFFFFFFFFFFFFFFFFFFFFFFFFFFFFFFFFFFFFFFFF75
:200BA000FFFFFFFFFFFFFFFFFFFFFFFFFFFFFFFFFFFFFFFFFFFFFFFFFFFFFFFFFFFFFFFF55
:200BC000FFFFFFFFFFFFFFFFFFFFFFFFFFFFFFFFFFFFFFFFFFFFFFFFFFFFFFFFFFFFFFFF35
:020000040800F2
:202800000828000800400008232042657461666C69676874202F2053544D3332463758322C
:202820002028533758322920342E312E30204F63742031362032303139202F2031313A3509
:20284000383A3435202863333761376339316129204D5350204150493A20312E34320A2343
:2028600020636F6E6669673A206D616E7566616374757265725F69643A20424546482C2074
:20288000626F6172645F6E616D653A2042455441465056463732322C2076657273696F6E9B
:2028A0003A2065646364323434622C20646174653A20323032322D30362D32395430323A0D
:2028C00032343A34365A0A0A626F6172645F6E616D652042455441465056463732320A6DF8
:2028E000616E7566616374757265725F696420424546480A0A23207265736F7572636573A5
:202900000A7265736F75726365204245455045522031204331340A7265736F7572636520C7
:202920004D4F544F522031204230300A7265736F75726365204D4F544F52203220423031BB
:202940000A7265736F75726365204D4F544F522033204130310A7265736F75726365204D60
:202960004F544F522034204130300A7265736F75726365204D4F544F522035204230360AB4
:202980007265736F75726365204D4F544F522036204230370A0A7265736F75726365204C17
:2029A00045445F53545249502031204130380A7265736F757263652053455249414C5F547E
:2029C000582031204130390A7265736F757263652053455249414C5F545820322041303212
:2029E0000A7265736F757263652053455249414C5F54582033204231300A7265736F7572BA
:202A000063652053455249414C5F54582034204331300A7265736F75726365205345524926
:202A2000414C5F54582035204331320A7265736F757263652053455249414C5F5458203630
:202A4000204330360A7265736F757263652053455249414C5F52582031204131300A72655E
:202A6000736F757263652053455249414C5F52582032204130330A7265736F757263652034
:202A800053455249414C5F52582033204231310A7265736F757263652053455249414C5FA5
:202AA00052582034204331310A7265736F757263652053455249414C5F525820352044300F
:202AC000320A7265736F757263652053455249414C5F52582036204330370A7265736F7511
:202AE000726365204932435F53434C2031204230380A7265736F75726365204932435F5360
:202B000044412031204230390A7265736F75726365204C45442031204331350A7265736FD0
:202B200075726365205350495F53434B2031204130350A7265736F75726365205350495FA6
:202B400053434B2032204231330A7265736F75726365205350495F53434B203320423033A6
:202B60000A7265736F75726365205350495F4D49534F2031204130360A7265736F7572631B
:202B800065205350495F4D49534F2032204231340A7265736F75726365205350495F4D49A1
:202BA000534F2033204230340A7265736F75726365205350495F4D4F53492031204130372C
:202BC0000A7265736F75726365205350495F4D4F53492032204231350A7265736F757263B9
:202BE00065205350495F4D4F53492033204230350A7265736F75726365204144435F424177
:202C000054542031204330300A7265736F75726365204144435F52535349203120433032E8
:202C20000A7265736F75726365204144435F435552522031204330310A7265736F7572637D
:202C40006520464C4153485F43532031204231320A7265736F75726365204241524F5F431E
:202C6000532031204331330A7265736F75726365204F53445F43532031204131350A726583
:202C8000736F75726365204759524F5F455854492031204330340A7265736F7572636520FF
:202CA0004759524F5F455854492032204230320A7265736F75726365204759524F5F43535C
:202CC0002031204130340A7265736F75726365204759524F5F43532032204330330A0A23C7
:202CE0002074696D65720A0A74696D657220423030204146320A232070696E204230303A33
:202D00002054494D33204348332028414632290A74696D657220423031204146320A23205A
:202D200070696E204230313A2054494D33204348342028414632290A74696D65722041304D
:202D400030204146310A232070696E204130303A2054494D32204348312028414631290A91
:202D600074696D657220413031204146310A232070696E204130313A2054494D3220434821
:202D8000322028414631290A74696D657220423036204146320A232070696E204230363A76
:202DA0002054494D34204348312028414632290A74696D657220423037204146320A2320B5
:202DC00070696E204230373A2054494D34204348322028414632290A74696D6572204130A8
:202DE00038204146310A232070696E204130383A2054494D31204348312028414631290AE2
:202E00000A2320646D610A646D6120414443203120300A232041444320313A20444D4132AA
:202E20002053747265616D2030204368616E6E656C20300A646D612070696E204230302008
:202E4000300A232070696E204230303A20444D41312053747265616D2037204368616E6EA4
:202E6000656C20350A646D612070696E2042303120300A232070696E204230313A20444D34
:202E800041312053747265616D2032204368616E6E656C20350A646D612070696E20413080
:202EA0003020300A232070696E204130303A20444D41312053747265616D203520436861D3
:202EC0006E6E656C20330A646D612070696E2041303120300A232070696E204130313A208D
:202EE000444D41312053747265616D2036204368616E6E656C20350A646D612070696E20FC
:202F000042303620300A232070696E204230363A20444D41312053747265616D20302043C1
:202F200068616E6E656C20320A646D612070696E2042303720300A232070696E20423037B0
:202F40003A20444D41312053747265616D2033204368616E6E656C20320A646D61207069D5
:202F60006E2041303820300A232070696E204130383A20444D41322053747265616D203330
:202F8000204368616E6E656C20360A0A232073657269616C0A73657269616C2032203634C5
:202FA000203131353230302035373630302030203131353230300A0A23206665617475722F
:202FC000650A666561747572652052585F53455249414C0A66656174757265204F53440AA7
:202FE0000A23206D61737465720A0A736574206261726F5F7370695F646576696365203DFD
:2030000020330A7365742073657269616C72785F70726F7669646572203D20534255530AEF
:2030200073657420626C61636B626F785F646576696365203D20535049464C4153480A73BB
:203040006574206473686F745F69646C655F76616C7565203D203435300A73657420637578
:203060007272656E745F6D65746572203D204144430A73657420626174746572795F6D65C2
:20308000746572203D204144430A7365742069626174615F7363616C65203D203435300AA2
:2030A000736574206265657065725F696E76657273696F6E203D204F4E0A7365742062659E
:2030C000657065725F6F64203D204F46460A736574206D6178373435365F7370695F627547
:2030E00073203D20330A73657420666C6173685F7370695F627573203D20320A73657420B0
:203100006779726F5F315F62757374797065203D205350490A736574206779726F5F315F64
:20312000737069627573203D20310A736574206779726F5F315F73656E736F725F616C69F6
:20314000676E203D2043573138300A736574206779726F5F315F616C69676E5F79617720E9
:203160003D20313830300A736574206779726F5F325F62757374797065203D205350490A83
:20318000736574206779726F5F325F737069627573203D20310A736574206779726F5F3206
:2031A0005F73656E736F725F616C69676E203D204357313830200A736574206779726F5F46
:2031C000325F616C69676E5F796177203D20313830300A0A00414C5FFFFFFFFFFFFFFFFF65
:2031E000FFFFFFFFFFFFFFFFFFFFFFFFFFFFFFFFFFFFFFFFFFFFFFFFFFFFFFFFFFFFFFFFEF
:20320000FFFFFFFFFFFFFFFFFFFFFFFFFFFFFFFFFFFFFFFFFFFFFFFFFFFFFFFFFFFFFFFFCE
:20322000FFFFFFFFFFFFFFFFFFFFFFFFFFFFFFFFFFFFFFFFFFFFFFFFFFFFFFFFFFFFFFFFAE
:20324000FFFFFFFFFFFFFFFFFFFFFFFFFFFFFFFFFFFFFFFFFFFFFFFFFFFFFFFFFFFFFFFF8E
:020000040800F2
:20400000AEBE08000E02000000000B0014020000000000FF001000030101000000000000E7
:2040200000000000001600230002000A00000000000000000000000000000076000D0001B7
:20404000000100000014050405000000000000000000050405000000000000000001050425
:204060000500000000400000000205040500000000000000000305040500000000000000DA
:20408000000405040500000000000000000505040500000000000000001E050405000000CF
:2040A00000000000001F05040500000000640052002A00FD01000019122A3A3C36000000F4
:2040C0000000001A132B3B42370000000000000000000000000000000000000700FB0100D1
:2040E00000000F00FC0100000000000000000000000C00F70100003E01000000000A00F96E
:204100000100003F000000160034000000DC0532000000000000000000000001040E0011DE
:2041200002000000000000010101010A0012020100FFFFFFFF3E00180003000001030204FB
:2041400005060702000000000001006400DC051A046C070019750343080E00000100000089
:20416000001E1E1E0101000000000000000000000000001100000200000000000000FF00D1
:20418000000000000B00FF01020000000000001A0008020100151617FFFF2D2E2FFFFF2302
:2041A0002425FFFF000000FFFF0A0013020000000001000900FA0100002C02000E002A022E
:2041C0000000960058022C0103000E002002050003643200F40196002A0006000100E00154
:2041E000070000000020211110262700000002000001020304050607C2012E04D007E80334
:204200000E000A000C020000011F03001A00FE0100000130003201310000010000000000A6
:20422000000000FFFF0020000B000300AE014A015E012C0164010100000001000A019A01BF
:20424000001E0A0000022A001F0005000000000000010001000500000102030000000000D9
:20426000000000000000000000000000008017000A00050200000000000012001B00020067
:20428000001800020301F40132000164F6002102000000000000000000000000000000005B
:2042A0000000000000000000000000000000000000000000000000000000000000000000FE
:2042C0000000000000000000000000000000000000000000000000000000000000000000DE
:2042E0000000000000000000000000000000000000000000000000000000000000000000BE
:20430000000000000000000000000000000000000000000000000000FFFF000000FF1E0082
:2043200000FF3C0000FF5A0000FF780000FF960000FFB40000FFD20000FFF00000FF0E015C
:2043400000FF2C0100FF4A0100FF0000000000000000010B020D0A03050B030D0A030A0B7E
:20436000040D0A03080B040D0A03070B030D0A03000000000000060A0100000203060000A3
:20438000000336003700010020003200C800D00796001400320028004C04400600055000CC
:2043A00014000F00080064000100010005000A000000F40196000F000C0016000100C409D3
:2043C0000000190028002F000100000000000000000000000000000000000000000000006C
:2043E000000000000000000000000000160023020200000000000000000000000000FF0081
:2044000000000F001E0000000005010000000000001200050002000201000000000000004D
:20442000000000160012000300000000010000055337583200000002008200FD070000EAC5
:2044400000EA00CD004E00CE00EA00EA00EA00EA00EA00EA00EA00EA00EA00EA00EA00EA91
:2044600000EA00EA00EA00EA004939EA00EA00EA00EA00EA00EA00EA00EA00EA00EA00EA04
:2044800000EA00EA00EA00EA00EA00EA00EA00EA00EA00EA00EA00EA00EA00EA00EA00EA7C
:2044A00000EA00EA00EA00EA00EA00EA00EA00EA002300EA00EA00CD00EA007200F501098D
:2044C00000980864001401000A010A0000FF1F0000142800002C3700008000FFFFFFFF462F
:2044E0000001020000000000000000000000000000000000000000000000000000000000B9
:2045000000000000000000000000000000000000000000000000005000C4FF00FFFFFFFF8C
:204520000100000005180B0C000000000014002600010002033D00000015005802D903007E
:20454000000B00140000000300002300120001000200E80364000F0A00010A001E00EA0086
:204560000C000400320003070707000000434343410046050064CE07CE07CE0701000000A8
:2045800000000000000000000000320003070707000000434343410046050064CE07CE076E
:2045A000CE0701000000000000000000000000003200030707070000004343434100460586
:2045C0000064CE07CE07CE070100000000000000000000000000320003070707000000436A
:2045E0004343410046050064CE07CE07CE0701000000000000000000000000003200030789
:204600000707000000434343410046050064CE07CE07CE0701000000000000000000000053
:204620000000320003070707000000434343410046050064CE07CE07CE07010000000000F7
:2046400000000000000000002A000A00090030000000FA00F40100000000000000000000FE
:20466000020000029E077D00FA00F401000105016400C2010E00030064004B000000000037
:204680002D50280078002F542E007D002D500000780032324B0000002800000000000055AE
:2046A000F401900101374B000000FA00AC0D00000000320090015E01F40100000A64C800F1
:2046C0009001960000050F00010F0114004B3200005A140B00004B00960000140028010066
:2046E000C8001E220025146400000000000000000000000032323296000019070F5A05005B
:2047000000026464646464646401646464004B00000000002D50280078002F542E007D0018
:204720002D500000780032324B0000002800000000000055F401900101374B000000FA0055
:20474000AC0D00000000320090015E01F40100000A64C8009001960000050F00010F0114F3
:20476000004B3200005A140B00004B009600001400280100C8001E22002514640000000080
:20478000000000000000000032323296000019070F5A0500000264646464646464016464D8
:2047A00064004B00000000002D50280078002F542E007D002D500000780032324B0000005B
:2047C0002800000000000055F401900101374B000000FA00AC0D00000000320090015E017E
:2047E000F40100000A64C8009001960000050F00010F0114004B3200005A140B00004B00ED
:204800009600001400280100C8001E220025146400000000000000000000000032323296F4
:20482000000019070F5A05000002646464646464640164640A0013000100080044100A00DF
:2048400001010000000000000A0000010000C20100000900020100006E0A012201220200BC
:20486000000000000000000000000000000000000000000000000000000000000000000038
:20488000000000000000000000000000000000000000000000000000000000000000000018
:2048A0000000000000000000000000000000000000000000000000000000000000000000F8
:2048C0000000000000000000000000000000000000000000000000000000000000000000D8
:2048E00000000042414E44312020200042414E44322020200042414E443320202000424140
:204900004E44342020200042414E44352020200042414E44362020200042414E4437202090
:20492000200042414E4438202020003132333435363738310032003300340035003600379A
:2049400000380000000000000000000000000000000000000000000000000000004C56304D
:20496000004C5631004C5632004C5633004C5634004C5635004C5636004C5637001100014B
:20498000020000000000000200000000000009000202000000000016001B020000060000CD
:2049A00000E803000000000000000000007600150000000000000000000000000000000081
:2049C0000000000000000000000000000000000000000000000000000000000000000000D7
:2049E0000000000000000000000000000000000000000000000000000000000000000000B7
:204A0000000000000000000000000000000000000000000000000000000000000000000096
:204A200000000066002A00000000000000E803D007DC0564FF00000000E803D007DC0564D9
:204A4000FF00000000E803D007DC0564FF00000000E803D007DC0564FF00000000E803D090
:204A600007DC0564FF00000000E803D007DC0564FF00000000E803D007DC0564FF000000DF
:204A800000E803D007DC0564FF16002C000000E803D007E803D007E803D007E803D0077E48
:204AA0000029000200000000000000000000000000000000000000000000000000000000CB
:204AC0000000000000000000000000000000000000000000000000000000000000000000D6
:204AE0000000000000000000000000000000000000000000000000000000000000000000B6
:204B0000000000000000000000000000000000000000000000000000000000000014001A67
:204B20000000007E05EA05B4053200E803D00700002A002B000000001E001E001E000501A1
:204B40001E011E011E011E011E011E011E011E011E011E011E011E011E011E160019020073
:204B6000000000000000000000000000000000000022001C020000000201140000340400A6
:204B80000000008C0A01020133000022030000000008071C002800030000000200000000CB
:204BA0000000000000000000000000000000001A000A02000000004A01B400D6010000C237
:204BC000010E0196004400000008001000010000050C00F80103000101F4011400070003B0
:204BE000000000000B00190000000000280100120002000000000000000000000000000054
:204C0000001200F6010200000000000100000002020000320125000200000000000000002A
:204C2000000000000000000000000000000000000000000000000000000000000000000074
:204C4000000000000000000000000000000000000000000000000000000000000000000054
:204C6000000000000000000000000000000000000000000000000000000000000000000034
:204C8000000000000000000000000000000000000000000000000000000000000000000014
:204CA0000000000000000000000000000000000000000000000000000000000000000000F4
:204CC0000000000000000000000000000000000000000000000000000000000000000000D4
:204CE0000000000000000000000000000000000000000000000000000000000000000000B4
:204D0000000000000000000000000000000000000000000000000000000000000000000093
:204D2000000000000000000000000000000000000000000000000000000000000000000073
:204D40000000000000460029020000000000000000000000000000000000000000000000E2
:204D6000000000000000000000000000000000000000000000000000000000000000000033
:204D800000000000000000000000000A002C020000190019000A0028020000000000000A6B
:204DA0000027020000000000004500160200002002002102001001001101002601002701B6
:204DC0000018010000000000000000000000000000000000000000000000000000000000BA
:204DE000000000000000000000000000000042001A02000000000000000000000000000055
:204E0000000000000000000000000000000000000000000042454648004245544146505675
:204E2000463732320000000000000000000001004300030201000000000000000000000047
:204E4000000000000000000000000000000000000000000000000000000000000000000052
:204E600000000000000000000000000000000000000001090038000200000A078600040053
:204E8000000000000000000000000000000000000000000000000000000000000000000012
:204EA0000000000000000000000000000000000000000000000000000000000000000000F2
:204EC0000000000000000000000000000000000000000000000000000000000000000000D2
:204EE0000000000000000000000000000000000000000000000000000000000000000000B2
:204F0000000043000B0202000000000000000000000000000000000000000000000000003F
:204F2000000000000000000000000000000000000000000000000000000000000000000071
:204F400000010000001A000D02010000000000000000000000000000000000000000000C1A
:204F6000001E0200000000000000000C001D0200000000000000001E00060201002829006E
:204F800000200300000000200300000000200300000000000016001F020000FFFFFFFFFF76
:204FA000FFFFFFFFFFFFFFFFFFFFFF0A00270000002003000007001002000000000059290D
:204FC000FFFFFFFFFFFFFFFFFFFFFFFFFFFFFFFFFFFFFFFFFFFFFFFFFFFFFFFFFFFFFFFFF1
:204FE000FFFFFFFFFFFFFFFFFFFFFFFFFFFFFFFFFFFFFFFFFFFFFFFFFFFFFFFFFFFFFFFFD1
:20500000FFFFFFFFFFFFFFFFFFFFFFFFFFFFFFFFFFFFFFFFFFFFFFFFFFFFFFFFFFFFFFFFB0
:20502000FFFFFFFFFFFFFFFFFFFFFFFFFFFFFFFFFFFFFFFFFFFFFFFFFFFFFFFFFFFFFFFF90
:020000040800F2
:020000040800F2
:20800000026C03463AB11A6CD20608D50022012083F83C207047426480F83C20F3E71A6CD8
:2080200049494A4811401A6841F00201F0B419644168474D21F44031416041685C682143BF
:2080400041605168186921F48071D3F808C0DF68516054689E6A44EA0024AE42546054683E
:2080600024F040745460506840EA0C005060906820F400609060916841EA0701916054D049
:208080009068DC6A20F07060906091680E439660906820F0405090609168214391609068C4
:2080A0009C6920F002009060916841EA4401916093F82010002941D05468596A44F400644F
:2080C000481E5460516821F460415160516841EA40315160D06A0025DC6920F470005E6971
:2080E000611ED0622846D46A44EA0154D462946824F400749460946893F8301044EA412494
:208100009460946824F480649460916841EA862191605D641A6C22F0030242F001021A64B2
:20812000002283F83C20F0BC7047916821F070619160916821F040519160B0E7516821F426
:2081400000615160C6E700BFFDEEFFFF002301400100000F0129F0B42A4C4FF000062A4D44
:2081600094BF002701272368EE626662A6626763676B47EA42076763EE63EC6B002A38D1F7
:2081800044F49574EC631C6824F001041C601C68E407FCD4490289085960D8601968EAB906
:2081A00021F04001196019498B421DD018494FF47410C860196841F01E011960596941F04B
:2081C00080015961196841F00101196022B90E4AD36A43F00803D362F0BC704741F040017F
:2081E00019600A498B42E1D14FF0746041F8500CE0E744F01A04EC63EC6A44F00804EC6240
:20820000C1E700BF88190120002C0140586402400064024011480023024611780632032973
:2082200016D00133062BF8D10D49CA6D052A0ED002EB4203013200EB4303CA65032040F276
:20824000EB3140F2FF32187059809A807047704703EB430300EB4303F0E700BFC0190120C1
:2082600088190120124B30B41D6E6B6A28B943EA01430020AB6230BC7047AC6A013803EB3C
:2082800014440BD0002303F14002013305EB8202DBB25268834204EB1244F4D3403044EAF4
:2082A000014405EB80004460002030BC704700BF88190120037870B42BB30246C0F10105A5
:2082C000531912F8014FDBB2002CF9D101335B000E4C03220B8084F8643484F8652401782A
:2082E00079B1022300265A1CE518023354FA82F285F86414DBB282F8646410F8011F00298A
:20830000F1D170BC70470223E2E700BF88190120826D136A5B681B78FF2B08D090F8F030DD
:20832000013BDBB280F8F0301BB10120704700207047126A0220526813707047F0B40F4BD1
:20834000C40800F0070700221E5D03EBD005BE40F6B2C7F1080300278B4228BF0B46C3F1AA
:2083600008049A40C91A46FA04F415F8016F42EA0402EED11046F0BC704700BF2C1F0120AA
:2083800030B5EFF31181802383F312880A4AD2F85836D2F85C46D2F85806D2F85C56CAB299
:2083A00082F31188013BA84294BF4FF4006000201B1B184430BD00BF88190120012380F8D7
:2083C00051307047014BD3F8600670478819012001207047024BC3F86426C3F86816704715
:2083E00088190120024BC3F86C26C3F8701670478819012070477047212870B505D022286C
:2084000029D0202810D0002070BD0029FBD0072AF9D1184B18791C685A799B790871002007
:208420000C604A718B7170BD0029ECD0072AEAD11148104B0C680E794D79D0F8682689794E
:208440001C601E715D719971002ADCD02146D0F864069047D7E70029D5D0022AD3D1064A47
:20846000D2F87036002BCED00988D2F86C069847C9E700BF000001208819012000207047EE
:2084800003460A2201481A80704700BF080001200346642201481A80704700BF1400012088
:2084A000012901D000207047014BD3F89030184700000120012901D008F0BCB9014BD3F814
:2084C0008C30184700000120014BD3F8883018470000012010B40B780A46044603F0030337
:2084E000012B05D0022B0BD000205DF8044B70478B8843B9204611465DF8044B0CF074BB5D
:208500008B88832BF6D0034B5DF8044BD3F88030184700BF0000012038B5054B04460D464E
:20852000DB6F98472946204608F03EFF002038BD0000012038B5054B04460D469B6F98470F
:208540002946204608F068FF002038BD00000120F0B4002452004E1C2746030FB0F1204F9E
:208560004FEA001003F1300503F1370334BF0D550B5537550234A242EFD1F0BC704700BF1E
:20858000024808B5FFF796FE014808BD9C5C0608EC1D0120024808B5FFF78CFE014808BD77
:2085A000AC5C0608EC1D01200B481A220B4B00681B680A80C01801D109487047094B0822F1
:2085C000094910B51C68FFF7C3FF042207492046FFF7BEFF024810BD107AF01F187AF01F68
:2085E000B0000120147AF01FB2000120C2000120024808B5FFF75EFE014808BDB85C0608CE
:20860000EC1D0120024808B5FFF754FE014808BDC45C0608EC1D0120042301480B807047C9
:20862000CC00012000487047141F012000487047141F0120034B93F88805032894BF0020A3
:208640000120704788190120034B93F88805032894BF00200120704788190120034B93F809
:208660008805003818BF0120704700BF88190120034B93F88805003818BF0120704700BFF9
:208680008819012098B182680C4B12B107229A70704718780421DA6003281A611A750CBFF2
:2086A00080224FF480729970C3E901227047034B012241F2E4715A705A5470478C7501200A
:2086C0000378022B0FD0006908B9012070470E4B1B78032B12D080B24FF6F773984294BF07
:2086E000002001207047084941F6500243688A58B3EB422F2CBF012000207047034B984201
:2087000094BF0020012070478C750120F7FFFF0F30B40378022B13D0104A41F648014368F4
:2087200041F63C04555802F5C25100692B400968023812595B0A01FB003030BC1044704799
:20874000064B41F6300441F6340142681859595800EB410030BC00EB522070478C750120D7
:20876000826D0346126A52681278FF2A0AD190F8F020002A02F1FF3214BF0120022083F886
:20878000F02070470020704738B540F48062074C0B4640F2FF55012100F03F00A563A360B2
:2087A000E2604EF081FAA56338BD00BF002C01402DE9F843884600294FD04718461E284CF7
:2087C000802507F1FF39EFF3118185F31288D4F85826C9B2D4F85C06D4F85836D4F85CC603
:2087E00081F31188634594BF4FF400630023121A1344012B1AD1012035F0EAF9EFF3118171
:2088000085F31288D4F85826C9B2D4F85C06D4F85836D4F85C7681F31188BB4294BF4FF4BB
:2088200000630023121A1344012BE4D0EFF3118285F31288D4F85C36D2B216F8011F234451
:2088400083F87416D4F85C360133C3F30A03C4F85C3682F311884E45B5D14046BDE8F883A3
:2088600088190120F8B5002390F8505080F85030CDB10F4941F2E8028A5C032A15D10D4EFF
:2088800000F13C04B76A29462046FFF791FFB36A2D1A0444DB1B322B01D8002DF3D1B5FAB3
:2088A00085F04009F8BD0120FCE71846FAE700BF88190120802A0120002280F85120D1E7F3
:2088C00090F85020531C0244DBB280F8503082F83C1090F851200AB1132B00D9C2E7704775
:2088E000F8B5144641F2E803094A0D46D35C032B0DD1084EB76A002C09DD21462846FFF71E
:2089000057FFB36A241A0544DB1B322BF3D9F8BD88190120802A012010B5074C04F2BC50E2
:208920003BF01EFA0A2035F047F9D4F8C405BDE8104038F0DBB800BF8819012030B5002397
:208940008DB0124A082102930DF107058DF814300124099302F2BC508DF828300B9382F837
:2089600054166944CDE90733094BCDE9035406933AF0B8FF07483BF0F3F99DF80700A0F182
:20898000FF00B0FA80F040090DB030BD8819012011830008441F0120F0B503798BB0284C19
:2089A000002B14BF0122002284F8B42503D184F888350BB0F0BD04F2BC56054690F90010BE
:2089C00030463BF095F8AD7875BB01271D4B1E48C4F85036C4F8C45584F8C8753BF0C6F865
:2089E00003464FF47A70A4F8C03535F0F1F8D4F8C40538F07BF828226846002154F03EFB9C
:208A00000A236946304602933AF06CFF30463BF0A7F90E4B002284F888759B6A84F87C2583
:208A2000C4F878350BB0F0BD284637F095FE054608B11E23C3800D21284637F017FFC4E731
:208A400088190120EC1E0120801A0600802A012070B5952592B0044640F0400601AA080C1E
:208A60008DF809500D0E8DF80810090A00238DF805508DF8060006250DF103008DF80710FD
:208A800003920121174A8DF8046004938DF818308DF82C300F938DF84030119305950C921D
:208AA000CDE90733CDE90D33CDE90901FFF746FF24B180F0010010F0FF0F10D10A4C08231F
:208AC00003A904F2BC5084F854363AF00BFF04F2BC503BF045F99DF8030012B070BDFF209D
:208AE00012B070BD618700088819012030B500238DB0104A014602930DF107058DF8143087
:208B00000124099302F2BC508DF828300B9382F8541602A9CDE90733074BCDE903540693A2
:208B20003AF0E0FE05483BF01BF99DF807000DB030BD00BF8819012061870008441F012066
:208B400070B590B01C4D0024FD220DF10303012601A905F2BC508DF803200693C5F8844565
:208B60008DF81040059407948DF824408DF838400F9403960896CDE90144CDE90A44CDE977
:208B80000C443AF0AFFE05F2BC503BF0E9F83046FFF7ACFFFF2809D0084A20460923926AA8
:208BA00085F88835C5F8782510B070BD0423022085F8883510B070BD88190120802A012037
:208BC00070B5064690B008200D46FFF78FFFFF2822D0FE2802D0022010B070BD002402237C
:208BE00001A90F48089301948DF8104007948DF824408DF838400F94CDE90265CDE905442F
:208C0000CDE90A44CDE90C443AF06CFE04483BF0A7F8204610B070BD012010B070BD00BF80
:208C2000441F01202DE9F84F484B98420FD003F56853083398424DD00023454A1846A2F878
:208C40009430A2F8A030C2E92633BDE8F88F404C022300263F4F04F13005DFF80481E36286
:208C6000D7F8D0303146B34206F1010603D0D4F8B00047F033FE94F8B4302846D4F8B0208A
:208C8000414685F82430303545F8102C48F03AF8E36A9E42E4DB002384F8A230E36A012069
:208CA000E16BA28EA56B12FB03F201FB03F3B4F84060A4F89420C4F89C30E28E264BC4F873
:208CC000C010C4F89850A4F8A060A4F89620C4F89030BAE71E4C02224FF0000B1D4F04F1DC
:208CE00030054FF4806A4FF040094FF40068E262D7F8D020012659465A45B34403D0D4F8E1
:208D0000B00047F0EBFD4FF00062D4F8B0104FF4003094F8B4C0296285F824C0A5F804A0B7
:208D2000A5F81090A5F80680AE74C5E90202FFF771FA28466E7647F031FFE26A074B93456F
:208D400045F8303BD4DB84F8A260A7E71971EF00802A0120000001209CD3050870D305087F
:208D60001940EF0010B50C4647F0E8FB50B9074B93F8C430012B4FF012030CBF04480548BC
:208D8000238010BD12230448238010BD802A0120FC000120E8000120D40001202DE9F8433B
:208DA0001C4C05468946904694F888651F46042E08D0082E02D00020BDE8F883FFF7C0FE77
:208DC0000228F8D1D4F8C40537F08AFE94F87E35B3B969021120FFF73BFEB8B90E4A0523F5
:208DE0000120C4F86495926AC4F86855C4F87085C4F87475C4F8782584F88835BDE8F88320
:208E000029461120FFF724FE0028E7D0FFF784FDD1E700BF88190120802A012010B50D4C22
:208E2000002394F85626C4F8843512B10A4AC2F8C8304EF045F920B10423022084F88835FA
:208E400010BD054A0923926A84F88835C4F8782510BD00BF88190120802A012070B50F4DA2
:208E600004460E4695F88835042B0BD0082B07D1D5F8803583420ED0FFF7D0FF022801D010
:208E8000012070BD08230220C5F88465C5F8804585F8883570BD022070BD00BF88190120D8
:208EA00010B509F06FFA104C58B194F88835032B13D894F87C350133DBB2072B84F87C3567
:208EC00003D9002384F8883510BD084B01229B6A84F88825C4F8783510BD05483AF046FEF8
:208EE000A4F8C005E5E700BF88190120802A0120801A060070B51F4C06460D4694F88835E1
:208F0000042B09D0082B25D1D4F8803583422FD0FFF716FE02281DD1D4F8C40537F0E0FD20
:208F200000213720FFF794FD29461720FFF790FDC0B994F87E357BB971021920FFF788FDF6
:208F400080B908230220C4F88455C4F8806584F8883570BD012070BD31461920FFF778FD86
:208F60000028EED0FFF7D8FCFFF79AFF032070BD022070BD8819012070B50379234C002B16
:208F800014BF0123002384F8B43503D1002384F8883570BD1E4D0021032095F9CF203AF09F
:208FA000B3FB0028F2D0466830463AF0D9FB84F855060028EAD095F8CD303046003B18BF2C
:208FC000012384F856364DF013FC09F0DBF938B994F87C3584F88805013384F87C3570BD87
:208FE0004EF048F940B194F87C350022013384F8882584F87C3570BDAA6A012384F87C05B6
:20900000C4F8782584F8883570BD00BF88190120802A012010B54EF02DF958B10C4C94F82F
:209020007C350133DBB2072B84F87C3503D9002384F8883510BD09F0A5F90028F7D0054B84
:2090400001229B6A84F88825C4F8783510BD00BF88190120802A01202DE9F84F904C94F878
:20906000B455002D00F0028194F8882502278D4E531E082B3ED8DFE803F03436A73D664999
:20908000153D05004EF01CF8002840F00181D4F87835B26AFA33934229D2FFF7BBFF94F87F
:2090A0008825E5E74EF00CF80028F0D0D4F884350022012B84F87C2540F2EE80D4F880151C
:2090C000013B94F856560131C4F88435C4F8801515B1744BC3F8C8200823054684F888354D
:2090E00011E084F888754DF0EBFF00284DD194F88825531EDBB2022B3CD9082A18BF042AE9
:209100000CBF012500252846BDE8F88F236B002B37D1644B0722D4F870559B6A84F8882547
:20912000C4F87835002DEED0D4F874350120D4F86425D4F86815A847D9E7D4F87835B26A63
:20914000643393421DD2D4F82C80B8F1000FF4D14DF0B6FF0028A2D00423D4F8705584F8FF
:209160007C8584F88835002D00F090804046D4F87435DCE74B4BD4F878259B6A9B1AC82B1E
:2091800079D800252846BDE8F88F4DF02BFC0028ADD196F8D130002BA3F10203B3FA83F33F
:2091A00014BF022201225B0984F87D2584F87E354DF018FC00287FF470AFD6F820210323A4
:2091C000C4F88C2584F888354DF00CFC00288ED1344A4FF0040EC4F88405032392F804B1A4
:2091E000B2F80611D2F8080184F892B5D2F808714FEA106CD2F80861A4F890153F0CD2F897
:2092000008A1360A92F80C9192F80D5192F80D01D2F8108125FA0EF5B2F816B100F00F00D1
:20922000B2F81611B2F81621C1F30B1184F893C502F00F0C84F8947541EA1B21724684F8AB
:20924000956501F00F0184F896A584F8979501F5FA6184F89C5584F89D05C4F89885A4F863
:209260009E1584F8A0C584F888E543E7284684F88855BDE8F88FFFF7CDFE94F88855082DF5
:2092800018BF042D0CBF012500253CE705463AE7042384F8883536E7FAD1FFF7BFFD26E71A
:2092A00088190120802A01202DE9F8430546884617461E462A4C94F88805042835D0082806
:2092C00007D1D4F88035AB4206D0FFF739FC0228F1D00120BDE8F883FC22224BDFF88C909D
:2092E000214883F83021C9F838813AF02BFB002809F588711C4814BF4FF400734FF480732D
:20930000C9F840313AF0EEFA012206230020C4F86485C4F86855C4F87075C4F8746584F8CD
:209320006C2584F88835BDE8F883D4F8C40537F0D7FB94F87E3553B969021820FFF788FB4E
:2093400038B994F88835082BC6D0FE22C5E72946F3E7FFF7E1FAFFF7A3FD0320BAE700BF0B
:2093600088190120802A0120441F0120000001202DE9F04FD84C95B094F8B465002E00F03A
:20938000998194F8882504F2BC57DFF8508304F2A459531E082B00F2A080DFE813F0340020
:2093A0005E0029019E008C00AF001B009E000900FFF7C4FA002840F05482D4F87835D8F85F
:2093C0002820FA33934280F08580FFF769FD94F88825DEE7FFF7B2FA0028EED0D4F8843567
:2093E0000022012B84F87C2540F26082D4F88025013B082106460132C4F8843584F888150B
:20940000C4F8802552E1D4F8C40537F069FB00210846FFF71DFB0546FFF77EFA012D59D10A
:209420004FF0000AD4F8C40584F87DA537F058FB40F2AB110820FFF70BFB052800F09081F6
:20944000012800F05181FFF767FA94F87D35002B00F02882022384F88835D4F8C40537F0AD
:209460003FFB94F87D3500213720022B0CBF4FF080450D46FFF7ECFA29202946FFF7E8FA41
:209480000546FFF749FA2DBB94F87D35022B00F0988184F87E55D4F8C40537F021FB0021A4
:2094A0000920FFF7D5FA002871D0FFF735FA94F88825531E11E04FF40071D4F86405FFF7B6
:2094C0007FFB012800F03081022800F03581002800F0618194F88825531EDBB2022B00F228
:2094E000DF807E4BD4F878259B6A9B1AC82B00F2E7800026304615B0BDE8F08FD4F8BC3593
:2095000077481D6A3AF01EFA002800F02C81B5FA85F56D09002DDDD004A800250DF10F03A4
:2095200002224FF0010A05A9059038460792ADF8105006958DF820508DF834508DF84850A8
:209540001395CDE90B3ACDE90955CDE90E55CDE910553AF0C7F938463AF002FC9DF80F30BC
:2095600003F01F03052B00F08581FFF799FCD4F870B5BBF1000F00F0F0802A465046D4F847
:209580007435D4F86815D84794F8882501E710214846FFF715FB8246002886D101217F20CC
:2095A000FEF7CCFE012805467FF47FAF50460221FEF7C4FE002800F0358101287FF475AFD9
:2095C00016213A20FEF7BAFE01308002C4F88C05FFF7A2F9D4F8C40537F082FA00210A2039
:2095E000FFF736FA002840F01681032384F88835102105A8FFF7E4FA00287FF46BAF9DF8FB
:2096000021309DF822201B019DF815009DF8165002F00F01DBB245EA0025DDF81D0043EA5F
:2096200012139DF81C2000BA84F8A01503F5FA639DF81710C4F89805A4F89E3513099DF8BF
:20964000140002F00F0284F89C35069BA4F89055C4F8943584F89D2584F8920584F893158A
:20966000FFF75AF994F87E3573B9D4F8C40537F037FA4FF400711020FFF7EAF90546FFF74B
:209680004BF9002D7FF4A1AE16483AF06FFA00220423A4F8C005C4F884251A4684F88835FE
:2096A000082A18BF042A0CBF01260026304615B0BDE8F08F304684F8886515B0BDE8F08F34
:2096C000FFF7EEFB94F88865042E18BF082E0CBF01260026EAE700BF88190120802A0120BE
:2096E000441F012040787D01042304AA05A9774807930692CDF814A08DF820A08DF834A025
:20970000CDF838A0CDE909AACDE90BAA3AF0EAF86E483AF025FB9DF81330AB2B7FF493AE6A
:20972000022384F87D358EE6D4F87835D8F8282064339342BFF4CEAEFFF7EEF8FFF7B0FBB9
:20974000D4F870554DB10022D4F87435D4F868151046A84794F888251BE694F8882518E6E4
:2097600084F87D556FE694F86C550246D4F864154FF48073384601EB05213AF0D7FA94F81F
:209780006C250132D2B2A2F1020584F86C25B5FA85F56D09BEE60190FFF7BEF8042301989A
:2097A000D4F8705584F87C0584F88835002D3FF47DAFD4F87435D4F86425D4F86815A84754
:2097C00088E6D4F8C40537F08BF929463A20FFF73FF904AA0423824605A9384605958DF8FC
:2097E00020508DF834500E95CDE90955CDE90B55CDE906233AF076F838463AF0B1FABAF1AE
:20980000000F08D1FFF788F8049B1BBAC3F3807384F87E353FE6FFF77FF8FFF741FB94F84E
:209820008825B6E504212C20FEF788FD032182464E20FEF783FD83460C213620FEF77EFD6A
:209840000BF1020B421C05FA0AF502FA0BF2A2FB0501420A42EAC152C4F88C25FFF75CF8C5
:20986000B8E60190FFF758F80423019884F8883506461BE7164B0722D4F870659B6A84F880
:209880008825C4F87835002E3FF410AFD4F874355046D4F86425D4F86815B04794F88825B9
:2098A000531E1AE61E4684F88835FFE608D0042384F88835FFF730F894F88825531E0CE6C3
:2098C000FFF73EF902287FF405AEEEE5441F0120802A0120154BDB68C3F3022310B4C3F1F3
:2098E00007041A1D042C28BF0424062A4FF0FF328CBF033B0023A240002821EA020101FA88
:2099000003F108DB09010A4BC9B2034483F800135DF8044B704700F00F000901054BC9B292
:20992000034419765DF8044B704700BF00ED00E000E100E0FCEC00E030B5264C00222648FA
:2099400041F28731D4F8743183B0244DA0FB030304F59A70C4F83451DB0C013BC4E95012F0
:20996000C4E94E320CF098FA1D4B062137201A6C42F020021A641B6C03F020030193019B21
:20998000FFF7A8FFD4F834314FF400001549164A4860D96841F00101D96099680A40062A28
:2099A00006D0B2F5803F03D01A6842F001021A600E4B41F2041200200D499A5803F2746490
:2099C000C3F87006C2F81002C3F86806C2E9811403B030BD802A012083DE1B4300140040A3
:2099E0000038024000E100E00700010088190120F82B012038B50F4B0F4AD3F87431A2FB71
:209A000003239B09013BB3F1807F10D20B4A0024F0200B490725536081F823002146946008
:209A20004FF0FF301560FFF755FF204638BD012038BD00BF802A0120D34D621010E000E09C
:209A400000ED00E04309012200F01F0084B0013B02FA00F0032B0BD8DFE803F015021E0C53
:209A6000124B5A6C02435A645A6C10400090009B04B070470D4B1A6B02431A631A6B1040A0
:209A80000390039BF4E7094B5A6B02435A635A6B10400290029BEBE7044B1A6C02431A64F1
:209AA0001A6C10400190019BE2E700BF003802402DE9F041D0F800E00C46DFF8588084B07D
:209AC000DEF804501746DFF850C0194605EA0805DDF82880064603932C43424644EA0C0C21
:209AE000CEF804C00AF098F978B931680246039B30468F624021CDF800800AF0BDF90038AC
:209B000018BF012004B0BDE8F081012004B0BDE8F08100BF009800FC00200180F8B5134F95
:209B200004460D460AE09B69DB0602D50AF034F9D0B9D7F878395B1B0A2B08D823682A462C
:209B40000A2120469E69B606EDD50020F8BD636C2021002201200B4384F84020636484F85A
:209B6000411084F84220F8BD0120F8BD802A01202DE9F04788B0884615461F46064639F0D8
:209B8000FBFC041E30DB224BDFF890901A19B18809EB840492F858A0C4F87C895EB14FF0C4
:209BA0000042B1FA81F0C24005D01A48046824EA02040460426103EB870305F0030230687D
:209BC000C5F341149B6E0026C5F38105D1441343039103A907960695CDE9043408F0D6FD6F
:209BE00099F8BC39F02B02D808B0BDE8F0870A4AF023032112F90A0089F8BC390190FFF779
:209C000069FE01980CF020F808B0BDE8F08700BF70D30508003C01402C5D0608802A01206E
:209C200010B4B8B10D4CD4F8C439102B05D1052100205DF8044B39F06FBC03EB43022244ED
:209C400082F8C919012182F8C8090B4482F8CA19C4F8C4395DF8044B704700BF802A0120F1
:209C600020218078DCE700BF2DE9F04FC14C002387B004F6F81894F80C2AC4F8F839C8E903
:209C80000133C8E903331AB194F80D3A84F8F83994F80E3A1BB194F80F3A84F8073A94F8A0
:209CA000123A1BB194F8133A84F8023A94F8103A1BB194F8113A84F8FD3994F8143A013BBA
:209CC0005FB2DBB2019702933B46013300F04F81A94EB0220023A94802FB076106F5217A6C
:209CE000A0F128050093743106F53F7953F054F90122009B2E4602FA07FB1F46307890B3AB
:209D00009F494FF0300C03E089452CD011F808CF6045F9D14A7812EA0B0FF5D036F01CFD08
:209D2000FB1DDBB210B100218371C171032136F09DFD30780023302101E01AF83310884276
:209D400000F0B2810133102BF7D14FF0000C009A0121072086F801C0531CB270F170DBB2BD
:209D6000307100930B4601370536042FC6D194F8240A01270393FFF765FE4FF44031814ECD
:209D80000022009BC4F82C1A3046D4F8201AC4F8443AC4F8407AC4F8387A84F8587AC4F860
:209DA000302AC4F8502AC4F8542AC4F8342A84F8482AC4F84C2AC4F83C2AC4F8281AFEF78A
:209DC0001FF9019B002B40F0EF80039B002B00F0EB80A6F1080050F059FA012308F1140876
:209DE0004FF0000A9B46EA78002A40F0178105354545F8D1019B02200299234493F91C2AC6
:209E000039F082FC0546002800F0B180406839F0A7FC0022062139F0B3FC002800F0A78033
:209E20006868002739F09CFCDFF874814FF078FF009B6A68012B4FF40063A8684FF4005501
:209E40008CBF4FF480613946C4F8702A4FF40032C4F8801A4FF48071C4F8843A0323C4F863
:209E6000740A4046C4F8983AC4F8787AC4F87C7AC4F8947AC4F89C7AC4F8A07AC4F8885AE0
:209E8000C4F88C1AC4F8902A09F064FB94F8643AC4F8608A012B0597C4F8A86A67D00123D1
:209EA000D4F8285A84F8643AAB68DE0713D4D4F874313549AA68B3FBF1F342F0010203EBA5
:209EC0004303AA600593059B2BB1059B013B0593059B002BF9D1AB68D80748D5D4F8682AA8
:209EE0002A4B134043F48073C4F8683A6B68590507D5D4F8683A23F4405343F48053C4F827
:209F0000683AD4F8683A13F4805300F03881D4F86C3A23F00603C4F86C3A1D4800231D49D0
:209F20006FF02202C4F8B00A1B4884F8643AC4F8AC1A05F14C01C4F8BC0A2A606E68009B69
:209F400046F08066154A16486E60AE6846F48076AE6009F073FA134B5A68D20640F0F88000
:209F6000D4F8283A9A6812F0405F00F0038107B0BDE8F08F802A012070D30508A0340120B1
:209F8000F4D50508A834012040420F00FEF8FFFFB90C0108BD0C0108A90C0108E401002006
:209FA000F034012000230140B02200217B48482753F064F8B0220021784853F05FF8784B24
:209FC000384684F8D47AC4F8D03AFFF73BFD4FF4403000230121D4F8D02AC4F8DC0A71482C
:209FE000C4F8F01AC4F8E81A84F8081BC4F8E03AC4F8003BC4F8043BC4F8E43AC4F8F43AB2
:020000040800F2
:20A0000084F8F83AC4F8FC3AC4F8EC3AC4F8D82AFDF7F6FF614850F039F9DEE694F8640A3E
:20A020005A1C69780128D2B22F79CDF810A039D0092984F864BA52D94FF0030E6FF01D0033
:20A04000D4F828CA4FF007091EFB0100DCF80CE009FA00F907FA00F02EEA0907CCF80C70C4
:20A06000DCF80C703843CCF80C00062B4FF0050020D86FF0040710FB0373D4F8287A1F2040
:20A0800000FA03FC786B01FA03F320EA0C007863786B03437B63D4F8283A4148834234D07B
:20A0A00084F864AA1346A2E63F4A02EBC30393F888C24CE60C2B32D86FF0220710FB0373A8
:20A0C000D4F8280A1F2707FA03FC076B01FA03F327EA0C070763076B3B430363DBE7D4F867
:20A0E000280A01EB41094FF0070ED0F810C007FA09F70EFA09FE2CEA0E0CC0F810C0D0F87C
:20A1000010C047EA0C070761AFE712291AD01129C6D126494B6843F400034B60C0E76FF02A
:20A12000400710FB0373D4F8280A1F2707FA03FCC76A01FA03F327EA0C07C762C76A3B43F5
:20A14000C362A8E719494B6843F480034B60A7E7D4F8282A12498A4214D05B68DB063FF542
:20A1600006AF134B9A427FF402AF9A6812F0405F7FF4FDAE9A6842F080429A60F7E6C4F882
:20A180006C3ACAE6936813F0405F03D1936843F080439360054B5B68E9E600BF50350120CD
:20A1A000002001405835012070D3050800230140002201402DE9F041D0F800E00C46DFF861
:20A1C000588084B0DEF804501746DFF850C0194605EA0805DDF82880064603932C43424654
:20A1E00044EA0C0CCEF804C009F016FE78B931680246039B30468F628021CDF8008009F08C
:20A200003BFE003818BF012004B0BDE8F081012004B0BDE8F08100BF009800FC002001812B
:20A22000034690F83C00012800F03E810220F0B4012483F83D0083F83C40142A45D8DFE87D
:20A2400012F04D004400440044007B00440044004400DA00440044004400AA0044004400C4
:20A260004400060144004400440015001A688E68156A0F6825F48015AB4C1562106A5568F1
:20A2800020F40010D2F854C040EA0650A74E0CEA0404B24244EA072400F0088106F58066A2
:20A2A000B24200F003814E6855605465D6651062506D0C6940F400605065506D20F4806039
:20A2C0005065516D41EA0421516500220121104683F83D1083F83C20F0BC70471A68D1F81E
:20A2E00008C0156A0F6825F00105914C1562106A5668956920F002002C408C4D40EA0C006E
:20A30000AA4244EA070400F0DD8005F58065AA4200F0D8804D685660946155631062906935
:20A320000C6940F008009061906920F004009061916921439161C8E71A68D1F808C0156AF0
:20A340000F6825F010057B4C1562106A5668956920F020002C40754D40EA0C10AA4244EA2A
:20A36000072400F0C38005F58065AA4200F0BE804D68566094619563106290690C6940F41A
:20A3800000609061906920F480609061916941EA0421916199E71A688E68156A0F6825F44B
:20A3A0008055644C1562106A556820F40050D2F81CC040EA06305D4E0CEA0404B24244EA35
:20A3C000072400F08D8006F58066B24200F088804E685560D46116641062D0690C6940F41A
:20A3E0000060D061D06920F48060D061D16941EA0421D16169E71A68D1F808C0156A0F6859
:20A4000025F480754A4C1562106A5668D56920F400702C40454D40EA0C20AA4244EA0704AE
:20A4200073D005F58065AA426FD04D685660D461D5631062D0690C6940F00800D061D06935
:20A4400020F00400D061D1692143D1613DE71A688E68156A0F6825F48035374C1562106A13
:20A46000556820F40030D2F854C040EA06402F4E0CEA0404B24244EA07041DD006F5806617
:20A48000B24219D04E685560546596651062506D0C6940F008005065506D20F004005065A9
:20A4A000516D2143516510E70220704725F480254E6945EA8625F6E625F480354E6945EA15
:20A4C0000625DFE726F4407C20F008008E69CF684D693843354320F0040045EA0C0619E771
:20A4E00025F480454E6945EA861571E726F4406C20F080008E69CF684D6940EA07103543B2
:20A5000020F040004CEA850632E726F4405C20F400608E69CF684D6940EA0720354320F426
:20A5200080604CEA051680E7FF8FFFFE000001408CFFFEFFFF8CFFFE8FFFFEFFF8B53D4EE4
:20A5400096F8804B04EB4403670006EBC30393F8843B032B44D8DFE803F0461B0F023C440E
:20A5600006EBC404D4F8883B002B58D0013B0025C4F8883B2846F8BD3B1906EBC303D3F867
:20A58000882B7AB1013A0025C3F8882B2846F8BD3B1906EBC303D3F8882B002AF2D1022252
:20A5A00083F8842B3C4406EBC40494F8903B013BDBB284F8903B4BBB0323D4F88C0B84F8C6
:20A5C000843B52F0B1FEC4F8880B064652F088FE80F00100002E0CBF002500F0010525BB03
:20A5E00001252846F8BD3AF0A3FE05460028F7D03C44012342F2107006EBC40484F8843BC1
:20A6000052F092FEC4F8880B2846F8BD01254FF47A7052F089FEC4F8880B2846F8BD52F026
:20A620006BFE80F00100C5B2B0E7013EC4F8886BACE700BF802A012003689B0AA3F58013EC
:20A64000522B00D970470E4A134470B593F8044384B00D2C12D800294FF0000309494FF0F4
:20A66000010514BF1E460226427901EB84106946CDE90065CDE902330BF00EFB04B070BDA0
:20A6800070D305086436012033492DE9F84F91F8D1101C46012507460229DFF8C4A01046DB
:20A6A00019464FF00002DFF8BC9018BF7F02CAF82C50FDF74FFD294A630240F2FF5BC9F8DC
:20A6C00024204FF40075C9F828304FF48A62D9F82C30012110205E4643F09303C9F82C302D
:20A6E000C9F838B0C9F808504D46C9F80C204CF0DBFA012CC9F838B04FF00A048CBF4FF05A
:20A7000052084FF051084FF0000939464046FEF73BF8013C034640F2774201213720E4B252
:20A7200023B91846CAF82830BDE8F88FAE63C5F80890EA604CF0B8FAAE63034608B1002CBC
:20A74000E3D1002BEDD000221846CAF82C20CAF82830BDE8F88F00BF802A012000E1F50524
:20A7600088190120002C01402DE9F843DFF8748004460F46914698F888551E46042D08D03E
:20A78000082D02D00020BDE8F883FEF747FB0228F8D101233A4620460021FFF775FF68B19A
:20A7A000FEF738FCD8F87045002CEBD00022D8F87435D8F868151046A047E3E7084A05239B
:20A7C0000120C8F86475926AC8F86845C8F87095C8F87465C8F8782588F88835BDE8F8833E
:20A7E000802A0120881901202A492DE9F04F91F8D1100124DFF8A8B00746022983B0CBF8D8
:20A8000030409A4618BF4702012B4FF00A04224D40F2FF568CBF4FF059084FF058084FF090
:20A820000009009239464046FDF7AEFF013C034640F2774201213720E4B2BBB900985146B4
:20A8400001220193154CFDF785FC13494FEA4A220020019B4C628A62CA6A42F09102CA62EF
:20A86000CBF82800184603B0BDE8F08FAE63C5F80890EA604CF018FAAE63034608B1002C7B
:20A88000D0D1002BDAD000221846CBF8302003B0BDE8F08F802A0120002C014000E1F505C5
:20A8A000881901202DE9F84F05460E4690461F46394C94F8880504280CD0082807D1D4F825
:20A8C0008035AB4206D0FEF7A9FA0228F1D00120BDE8F88FDFF8C8A0C4F86465DAF8C89042
:20A8E000C4F86855C9F34F234FEA59220F2B2BD8D4F884B5BBF1000F26D094F8561619B346
:20A90000B9F5005F41D025484FF400723146484452F042FB09F50072C2F34F23CAF8C82034
:20A92000520A102B31D0BBF1010F2ED0D4F880250BF1FF33042102200132C4F8843584F8BB
:20A940008815C4F88025C3E701234FF001092846062532460021C4F87085C4F8747584F8DE
:20A960006C9584F88855FFF73FFF0028B0D0FEF751FBD4F870556DB14846D4F87435D4F8E2
:20A9800068150022A8470320A2E792B2034E013AAD1ADAE703209BE7881901208C550120BC
:20A9A000802A012070B50D4C1346D4F8A45F2A78022A07D00A46014604F6A470BDE8704087
:20A9C0003AF030B82A6A0AB1002070BD0A46014604F6A47039F02AF9012070BD802A0120BF
:20A9E00003681878012801D00020704793F90430074A03EB430302EB431313F8332C202A4F
:20AA0000F3D153F8743C9869C0F3C030704700BF783B0120036801221B78022B01D03AF040
:20AA20002BBA39F05BB910B50B4CD4F8A43F1B78022B10D1D4F8AC0F36F058F8D4F8AC0F04
:20AA400008B12123C380012135F010FF034839F08DF8A4F8A80F10BD802A012080969800CE
:20AA600038B505460A460C460648294639F00EF945F08001034839F08DF8231A58425841F0
:20AA800038BD00BF243A012030B5044683B001230D460DF107020848214639F0C3FF9DF86C
:20AAA000072035EA020304D02A43214602483AF097FA03B030BD00BF243A012013B53A4C72
:20AAC0000023D4F804218DF80730137803F0FD01012905D194F8081111B90C2184F80811F9
:20AAE000022B1ED0032B2ED001220B212F484BF055FD042033F06CF801230DF107020021C5
:20AB00002A484BF06DFD002839D09DF80730482B35D1274BC4F8F830264BC4F8FC3002B047
:20AB200010BDD4F80C0135F0E1FFD4F80C0108B13523C380012135F099FE1F4839F016F8C1
:20AB4000A4F80801D0E7D4F8B43546F2A8115068122219610023372180F888304BF0F1FCBA
:20AB6000D4F804310D22242158684BF0EAFCD4F8043130226A2158684BF0E3FCB4E7D4F860
:20AB800004311A78022A03D0032A07D00020C6E7D4F80C0138F086FE0020C0E71022372148
:20ABA00058684BF0CEFCF1E7783B01207C3C01203F660508C166050880969800F8B55E4C60
:20ABC00000234FF4F07206460F4604F63810202184F8343984F8353952F050FA4FF4F07285
:20ABE000202104F6183052F049FA322032F0F0FF94F8F93C002B00F0948094F8FA1C04F65E
:20AC0000FC4038F075FF002800F08B8094F8F90C35F0A2FD0546C4F8040D35F069FE002818
:20AC20007FD00DB12323EB800D21284635F01EFED4F8040D35F05AFF404838F097FF03468F
:20AC4000FF213F48A4F8003D39F052F88C213C4838F0A0FF1B2867D10122D4F8043D84F8E2
:20AC600034290BB12322DA8040220A21344839F00DF88A21324838F08DFF94F8F83CC0F399
:20AC8000801584F8945D002B44D0022B3BD12D4838F06CFF0346A4F8960D94F8982D182A17
:20ACA00011D1294A2949D2F87421A4F89C7D5208A4F89E5DA4F8A03DB2FBF3F2A1FB02120D
:20ACC000520BA4F8A22D1E4802220021A4F8003D38F0DCFFC8201A4D32F06EFF8021284638
:20ACE00038F058FF10F00200F8D17278B3783178C2F12002C3F1100384F8A52D84F8A63D03
:20AD000084F8A41DF8BD124838F030FF0346A4F8960DC2E7094838F029FF0346A4F8960D36
:20AD2000BBE76FF00100F8BDD4F8040D202135F09DFD4FF0FF30F8BD783B0120404B4C00B1
:20AD400074480120002D3101802A01205917B7D1809698000146014838F01CBF2049012029
:20AD600030B40023314D32494CF25034C5F8583E304AD1F8780904E0D1F878391B1AA34282
:20AD80000FD8D368DB03F7D4D16811F4F9710BD1D06810F0010002D001230846D36030BCC8
:20ADA0007047032030BC7047D3689B0705D5D5F8583E43F02003C5F8583E1E4BDB68DC06C5
:20ADC00005D5D5F8583E43F01003C5F8583E194BDB68980605D5D5F8583E43F00803C5F820
:20ADE000583E144BDB68590605D5D5F8583E43F00403C5F8583E0F4BDB681A0605D5D5F88E
:20AE0000583E43F00203C5F8583E0A4BDB68DB0505D5D5F8583E43F04003C5F8583E054B43
:20AE20004FF4F9720120DA6030BC7047783B0120802A0120003C0240014488420ED0034613
:20AE4000074810B4074C13F8012B04FB00F0994280EA0200F7D15DF8044B704700487047FD
:20AE6000C59D1C8193010001094B93F85E3E042B08D9053B032B08D801231A4600B10370BD
:20AE80001046704700230122F8E700231A46F5E7783B01202DE9F04FDFF8DC81DFF8DC9180
:20AEA000D8ED037A08F5B06399F8802EF8EE677A2DED028BC3ED007A83B0002A4ED1614E3E
:20AEC000C8F8882598F88C153278D9B1B9F8863E0024DFED5D5A07EE103ADFED5C6A5C4B0C
:20AEE000B8EE477A67EEA66A03EBC10085EE876A36EE266A86EE867A1C60083303ED017A29
:20AF00009842F9D199F87E3E9FED525A06EE103A96F8583B9FED507A1A44B8EEC66A27EE0A
:20AF2000877ADFED4E6A12FB01F14D4AC5EE065AC9B207EE901AF8EEE77AE7EE876AF7EED7
:20AF4000667AFCEEE77AC2ED005A17EE903A88F8DC3603B0BDEC028BBDE8F08FFCEEE77A04
:20AF60009FED404A99F8811EB9F8843EF8EE674A06EE101A002107EE103A324EB8EE466A2D
:20AF8000C4EE245A0191B9F8821E01239FED365A06EE901AC6ED057A98F88C15B8EEC77A76
:20AFA0009FED328AF8EE666AC8F88865327067EE057A86ED016A88F88435C6ED036AC6ED86
:20AFC000047AC6ED025A89B3294B4FF0000B019903EB010A12B3AAF118045746002507EE24
:20AFE000905A01223846B0EE481AB8EEE70AD6ED017AD6ED040A15447169283720EE270A4F
:20B00000283452F0A5F984ED028A84ED018A84ED048A84ED038A32789542E0DB0BF1010BBA
:20B0200098F88C150AF1780A8B45D3DB019B03F57073B3F5346F0193C5D10E4BD3ED007A65
:20B0400043E700BFD034002083F9223EBD378635004A0120555555406E12833A48E1FA3E10
:20B06000BC0800200060EA480AD7233C00000000E834002064070020E4010020783B01207A
:20B0800007EE900ADFEDAF5AAF4B0022B8EE677ADFEDAE4AB3F8C81E85EE874A06EE101AF2
:20B0A000B3F8CC1EDFEDAA5A07EE901AB3F8CA1EB8EE466A06EE901AF8EEE77AF8EEE66A88
:20B0C00036EE065A67EEA47A2DE9F04FC6FE856AA04D2DED048BB4EEE54A05F5DC6993F840
:20B0E000CE4E85B0C5F83007F1EE10FA89ED016AC5F8EC46C5F8F026C9ED026AC9ED007A2D
:20B1000002D51446C5F8EC26F6EE004A9FED925AF7EE003A914927EE055A9FED912A64EE83
:20B12000247A0B46F0EE002A9FED8E3A143381ED045A87EEA67A01F5A677039301F12C064F
:20B1400091ED055A884A12F8542C87FE237ABDEEC77AF8EEC77A17EE103A012BC5F88C3984
:20B16000C4EE275AB8BF0123029383EEA74A65EE825A86EE257AA1EC014AC1ED005AC6EE34
:20B18000A57A37EE247A87FE227ABDEEC77A77EEA47A17EE101AC7FEC37AFDEEE77A01F1CE
:20B1A000FF38C5F8981917EE901AB8F1230F01F10100A8BF4FF02308C5F89C192328834616
:20B1C00028EAE878A8BF4FF0230B5B468045C8BF43460093A3EB0803019362BB624B934650
:20B1E000DFED629AA3F1500A9FED619A07EE90BA0BF1010B0AF1080AF8EEE78A68EEA98ADE
:20B20000B0EE680A44F036FFB0EE408AB0EE680A45F04EF9B0EE680A45F04AF928EE098A90
:20B2200020EE090ABBF1240F0AED028A0AED010ADCD19FED505A019A00234F489446029ADB
:20B240009FED4E7A9CFBF2FA0AF10101A24614468E460099324646F80C1C46E9053846E9F2
:20B2600002E4A2EC017A9742FBD13A4606F5107BD0EDD67AD0F85CC3C2ED007A083242F8A3
:20B2800004CC5A45F8D106F515763D4A07F515779642DFD1039BB6EE008A5446012283ED60
:20B2A000005A4FF0000A374B4FF0000800932E4B03F8542C002C35DD09EB0A06DDF800B0D4
:20B2C000002707EE907AD9ED016A99ED027A06EE104AF8EEE77A012237EE667AD5F8301744
:20B2E000B8EEC66A06F1540077EE887A1744B7EE001A283667EE877A87EE860A30EE260AA5
:20B30000ABEC010AD9ED000A52F022F8D5F8EC46C6F84480BC42C6F84080C6F84C80C6F81A
:20B320004880CEDC009B0AF1C80A1433BAF5167F009302D0D5F8EC46BCE705B0BDEC048BB4
:20B34000BDE8F08F00247449783B01200AD7233C0000FA44E40100209C534937740B002083
:20B36000398E633C00000C42DC120020C3B8B23D72F97F3FBC297E3F70D305080000000086
:20B380009C120020D808002008480023024611780632022904D00133062BF8D1002070475F
:20B3A00003EB430300EB4300704700BFC01901200021094B00B5084683B0C3F8D01E2AF04D
:20B3C00027F80422054B06200DEB020101932AF013F803B05DF804FB783B01205475C52A6B
:20B3E00070B5461E00F13105344614F8011F601EFF29A0EB060002D0C0B22AF009F8AC4273
:20B40000F3D1A02040F2E93446F02AF80121022029F0FEFF01E0013C04D04220FFF79AFCC7
:20B420000028F8D16220FFF795FC1321242029F0EFFF2520092129F0EBFFA020BDE870400C
:20B4400046F00EB830B54CF205028DB0002304460321ADF8002001AD01228DF802300B930D
:20B460008DF814208DF82820CDF808D0CDE90633CDE90833CDE9035138F072FC204602A918
:20B4800038F030FA204638F06BFC9DF806000DB030BD00BF2DE9F043734E83B0734C24221F
:20B4A000002106F1380051F0E9FD002394F8D55EF365002D37D16E4FD7F8903043B39B6A5F
:20B4C00033B36C489847836813B3038800246A4F013BBC4639469BB20878063103281BD003
:20B4E0000134062CF8D1002239780637022900F09D800132062AF7D1F16D052908D002FB48
:20B5000001C20131F16502200021938010705180284603B0BDE8F083062303FB0464638F7F
:20B52000013B9BB2DFE704F6DC6794F8D40EC4F8D87E10B900254E4FBEE735F00DF9C4F8E8
:20B54000E40E35F0D5F90028F4D02946384638F0CFFA05460028EDD0D4F8D83E454A98689B
:20B56000C3F8942008B12023C3800D21404F35F07DF9D4F8D83E4FF00109986835F0B6FAC5
:20B580003E4838F0F3FAD4F8D83E024632209A80C7F8B03087F8B49032F01AFB04234FF07B
:20B5A000000C9F21D4F8D80E0DEB0302CDF804C038F03CFB9DF805809DF8043007F19000BD
:20B5C0004FEA08289DF8061048EA034848EA0108414645F097FB00287FF46EAF4046FDF71F
:20B5E00021FB034600287FF467AF9DF806009DF8052000029DF8071040EA0240204A084311
:20B60000904217D0A7F89430A7F8A030C7E92633FDF708FB034600287FF44EAF94F8D40E50
:20B620001D4635F099F838F03DF945E7062101FB02C268E7134B4FF400314FF0006287F83F
:20B64000A290C7F894304023C7E92612A7F8A030FCF7E0FD07F1900087F8A99045F09EFA9E
:20B66000094BC7F8903027E788190120783B0120802A0120102B0120C0190120404B4C005B
:20B6800021AAEF000004000870D305082DE9F04F0423BE4C402141F21C1504F6746704F17F
:20B6A00060064FF0A042636661670023022194F81D048BB0C4F8607466512266C4F89030F9
:20B6C0002367C4F88C30C4F88430A167E166C4E91F33002800F0628103211F46164684F84E
:20B6E0001D14936823F001039360F368304643F04003F36008F090F9B36B012F054643F429
:20B700008033B36317D005B3022384F81D34A04B93F8C450012D00F0FD80236E8021012057
:20B7200059625A6A42F480029A62FCF79BFD00200BB0BDE8F08FB36843F00603B360B368C7
:20B7400043F02003B360002DDED1236E3220DA6822F0C042DA60DA6842F08042DA600AF0C7
:20B7600081FA606E50B32A4601272946C2EBC203561C04EB830383F89C20A3F8A220F2B2E5
:20B7800083F89D70824283F89F10C3F8B010C3E92911EBD300221146C2EBC203561C04EBC8
:20B7A000830383F85C22F2B283F85D12824283F85F12C3F87012C3E99911EDD30022236EC6
:20B7C000D4F86CC01646D4F87080D4F88CE0D4E91E71019102F14001013203EB81010F2A33
:20B7E0004E60F7D19A6BBEF1000F40F0438122F400129A631A6842F040021A601A6842F0D3
:20B8000080021A600022012F03F50066C3F8002ED3F80028C3F80028D3F8002800F0218138
:20B82000032F00F01E8142F00302C3F800284FF48461584A196102E0013A00F032811969A7
:20B840008F06F9D41021534A196102E0013A00F026811969C906F9D4002131617161F16195
:20B86000E0B103F510624FF0904A4FF0006B0F464FF67F399C4607E0176001311761C2F814
:20B8800008902032814261D01368002BF4DA11B1C2F800A0F1E7C2F800B0EEE73269B8F1DF
:20B8A000010F22F48072326100F0ED8000216FF0804299615A61B8F1000F03D19A6942F0C8
:20B8C00010029A619969344A0A439A61019A1AB19A6942F008029A61BEF1010F00F0CE80F6
:20B8E000002D7FF411AF0121D4F8842084F898508A4284F81D1400F0D6807368032043F002
:20B90000020373600AF0AEF9214B93F8C450012D7FF403AF44F012FE00287FF4FEAE236E34
:20B920008022284640215A625A6A42F400129A62FCF798FC20210220FCF794FC40210320E1
:20B94000FCF790FC00200BB0BDE8F08F002163460CF530624FF0904A4FF0006B0F464FF6AF
:20B960007F39844607E0176001311761C2F808902032614592D010680028F4DA11B1C2F8A7
:20B9800000A0F1E7C2F800B0EEE700BF88190120802A0120400D030000383C8000F0FF056C
:20B9A0004C4B03204FF4C05684F81C541A6B42F001021A630A221B6B069105A903F0010363
:20B9C000089045480493049B07950596099206F0DDFED4F88C30012B72D03E4B0621432060
:20B9E0005A6B42F080025A635A6B02F080020292029A5A6C42F480425A645B6C03F48043AB
:20BA00000393039BFDF766FF266E0323334A0821916084F81D34A26FB368012A276F23F07B
:20BA20000103B3607FF461AEB26B2D4B22F48032D4F89410B2630129F26803EA0203F360C2
:20BA4000F36823F44013F36003D1F36843F48013F360304607F0E0FF012F05467FF453AE47
:20BA600069E6BCF1000F3FF4E0AE42F00102C3F80028DCE642F400129A63C3E69969194ACD
:20BA80000A439A612CE718490020184A31636FF08041376B3A4332639861596112E701252E
:20BAA000DAE60125CEE684F854549969C4F85C2441F000610E4A9961596D0A435A651CE7D1
:20BAC0004FF4007305A904480593CDE9065506F05DFE82E7003802400000024000E100E0D6
:20BAE000BFFFBDFF0400004000018000030001000300001010B51A4C94F8750FC0B9194BD8
:20BB000083F8B505C3F8B80594F8783F012B05D0022B21D0D4F87C3F1BB910BD124BC4F8D5
:20BB20007C3F12495B68A1F10C00BDE81040184734F012FE94F8772F0A49003AC1F8B805D1
:20BB400018BF012281F8B5250028DDD01F222021C28034F08BFED7E7054BC4F87C3FE0E706
:20BB6000783B01208819012084010120F84A01206001012099B10A6B824216D9154BD3F807
:20BB8000C42F914221D34C3991421ED30B6B9842F9D38B6B9842F6D80B46184670470D4B2A
:20BBA000D3F8C41F0A6B904212D30B680BB9F4E70A6B90420B4602D38A6B9042EDD951F856
:20BBC0004C3F002BF4D1184670470023184670470A46D8E7783B01202DE9F047CC0143D18C
:20BBE000034622494FF0FF32022443F8081B7E2642601846DFF878802644051D6FF0704788
:20BC0000D8F8C89F4FF0010A013E494608E0A3421CD0631C45F8043C321B1C460435CAB1BD
:20BC20000B6BA34202D88B6BA34204D22046FFF7A1FF014690B10A794B6B002AE7D1A3429A
:20BC400004D0E6D2631C45F8042CE5E7631C45F8047CE1E7C8F8C81FBDE8F087321B631C0D
:20BC6000494645F804ACD8E78026C3E7F8FFFF0F783B01200A44914219D0013910B4541EE6
:20BC800011F8012F0823504002E0013BD0B209D010F0800F4FEA4002F7D082F0D500013BE3
:20BCA000C0B2F5D1A142EBD15DF8044B70477047194A00232DE9F04702F6DC7484B0054601
:20BCC00092F9D58F1F46461804F5287A4FF0B609D4F800C0204600226946E034BCF1000F86
:20BCE00014D09CF838C0BCF1140F0FD018F1020F01D0C4450AD1CDE90277CDE90056ADF876
:20BD000008908DF80D702AF0CDFA0346A245DFD1184604B0BDE8F087783B01202DE9F04779
:20BD20009AB004460D4617469846DDF89090DDE9226A02E0206831F0BDFF206831F0C2FFE9
:20BD40000028F7D10146642201A851F097F9264B8DF80450CDF85CA00293002D3FD0AB1E07
:20BD6000012B3ED9042D14BF002303231F4A8DF805300123926A039616448DF85B30CDE937
:20BD80000594049637B14246394607A851F004F98DF85A80164E002396F8C6911893B9F174
:20BDA000000F19D196F8C501642201A902FB006000F5E47051F0F0F8012386F8C59186F8C1
:20BDC000C631236843B143463A46294620461AB0BDE8F04717F080B81AB0BDE8F08705231C
:20BDE000C4E70223C2E700BFF44D0120802A0120704C01200C480D4BD0F8481210B48A1EC7
:20BE00000B4C2231C0F83832B0F866321B01A4FB03C3DB08A3F5B06322F8023F9142F3D115
:20BE20005DF8044B704700BF704C01201D700208CDCCCCCC70B5084C251D2E4614F8010BFC
:20BE40002AF004FC28B10378B44205F8013BF5D170BDFF23F8E700BFFC4E01202DE9F047DA
:20BE60001C4F01264FF03C094FF0000807F10805B24617F8010B34F06FFC044690B180F8BB
:20BE80000690C671FB7803F07F02012A17D013F0800F20460CD185F8048034F021FE85F846
:20BEA00005802C6001360835052EE2D1BDE8F08785F804A034F01AFE85F805A0F1E71B0683
:20BEC00005D40121204634F0D1FCFB78DFE734F00DFEF6E7044F01202DE9F047204E82B06A
:20BEE00000244FF00409DFF87C8006F10C05A6F5307716F801AB5046BAF1000F2CD034F08B
:20BF00002BFC0134034604215046E4B26B6113B183F80690DC71224631F0EEFB02218246E0
:20BF2000D0B168699AF8082034F068FCB7F8BE32B7F8BCC2002051460A4A01902846CDF8D2
:20BF400000C01835B8FBF3F39BB229F07BFA0123082C05F8073CCCD102B0BDE8F08700BF9E
:20BF6000304F012040420F002DE9F041204C00234FF0050894F8932304F5647704F5657585
:20BF800084F88C2317F8010B5E1C20BB2860032E05F104053346F5D194F88C13D4F8940381
:20BFA000C94301F0010134F055FE94F88C13D4F8980381F00201C1F3400134F04BFE94F817
:20BFC0008C13D4F89C0381F00401BDE8F041C1F3800134F03FBE34F0BFFB0121F3B2286088
:20BFE00010B180F80680C371286834F03FFCCEE7704C0120F0B5294C83B0B4F8A453A4F841
:020000040800F2
:20C00000A653EDB994F8A00334F0A6FB94F8A123C4F8A803003A18BF012284F8AC2348B15E
:20C0200094F8A2132B220029C28014BF1121012134F01CFC002003B0BDE8F04034F012BE08
:20C0400094F8A07300222B21384631F055FB0646384634F081FB00B10EB903B0F0BD2B2255
:20C06000C4F8C40302210027C280327A34F0C6FB0B4AA4F8C853314604F56C700197B2FB83
:20C08000F5F3C3F34F059BB2009529F0DBF9D4F8B0331F6084F8C173DFE700BF704C01209F
:20C0A00040420F002DE9F84F264B002693F8D42303F2CB3703F57A7483F8CA235FFA86FB5A
:20C0C0004FF0010917F8010F01360BEB090A49464FF000085FFA8AFA524631F00DFB0546F9
:20C0E00048B3387804F80E8C04F80D8C04F80FBC04F8109C44F8045C34F02EFB022118B126
:20C1000080F8069080F807A02A7A34F077FB0E4A002128464CF090F90C4B221D214623608C
:20C1200028460B4BC4E901384CF052F842466979286829F0D5F8082E04F11C04BED1BDE870
:20C14000F88F00BF704C012040420F0095530308D1FB020870B52C4C00222C4B022194F87D
:20C160000005C4F8F834C4F8B824C4F8BC24C4F8C024C4F8F424A4F8FC2431F0BDFA00286E
:20C1800041D0234B0546026803F1C000597C11B159688A422CD018338342F7D1002394F810
:20C1A0000005C4F8E45384F8D83334F0D5FA08B10223C38000262A7A022134F01FFB31464A
:20C1C0002846144A4CF038F9134B144A2846C4F8E833134B111FC4F8F063C4F8EC334BF072
:20C1E000F7FF324669792868BDE8704029F078B8926A0C4801320C49D0F87431B3FBF2F3E9
:20C2000081F8A831CAE770BD704C012000FFFF00AC13002040420F00F9FB02085C500120D8
:20C2200095FD0208802A0120000001202DE9F04FDFF878B180460B46DFF874A10BF1D00052
:20C24000C02200212DED068B97B0CDE9023850F015FF9AF80185B8F1000F00F095829AF83C
:20C2600002350893002B00F0CE82DFF8489199F86C3E012B00F0ED82022B00F0E5820BF587
:20C28000FC73444D99F8626E1C460F930FCD0FC40FCD0FC4311E404A99F85E3E18BF0121DC
:20C2A000CBF81022072B8BF8301295E8070084E8070000F25D83042B0ED999F8613E374A02
:20C2C000012BCBF8382205D09A1E53425341002E18BF00238BF83C320023DFF8DCA003933A
:20C2E0002F4B04932F4B0593DDE90232934240F3B081059B032113F8015B059309EB050329
:20C30000013593F8636EEDB230462A4631F0F4F90446002800F02283304634F01DFA049BA1
:20C32000586110B10323C571837199F85E2E99F85F3EE77906920BB187F00107204637F028
:20C34000A7F90346002800F006839BF83C220792002A40F01883D0F80480B8F1000F00F0E0
:20C36000FD829B6840460B9337F0FAF92A4603210A9037F005FA002800F0F0829BF84062EA
:20C3800025680948CAF89480002E00F027830023024617E020D80508398E05086D4104082C
:20C3A000AC130020E649012020150020DC120020704C0120783B0120A02600200133B3422B
:20C3C00000F00C831168B8328D42F7D1DEB2B8239BF84022039906FB0303013A8AF8111003
:20C3E000CAF898302079099234F0B6F907F001019BF8303201310BB187F001074901CAF845
:20C40000084041F00E01CAF81410227A34F0F6F9099B9E4200F01E84069B063B0C93002345
:20C4200060220AF16401CAF8803008EE101ACAF86420CAE91A33CAE91C33CAE91E3317F035
:20C4400002034FEA47070D9300F0E082012307F00207CAF86C30CAF87870002702234FF4A3
:20C4600080310A22CAF87070CAF88420CAF89030CAE9221763790C2B00F2BE82CB4A9BF87C
:20C480003C1202EB8302D2F80874CAF85470002900F0F982DAF89830C3F8A880CAF8948029
:20C4A000079B002B00F073830AF118000E9007F0F1F89BF83C320E98002B00F08E83BC4960
:20C4C0004FF4907322684FF0030C03FB0613DAF898104C32C1F8B030CAF81C300B9BCAF820
:20C4E0001820CAF83C30CAF848C0069B40214FF4806C082B4FF00403CAF820104FF480515C
:20C50000CAF844304FF000030CBF06221222CAE91333CAE909334FF40033CAF838204FF4C1
:20C520008042CAF84030079BCAF83420CAE90BC1002B00F040839DF83030CAF89480022BFA
:20C5400000F25582994A9B4902EB8303069AD3F8FC33082AB1FBF3F308BF5F2203F1230318
:20C5600018BF1322CAF85C30DAF8983050469A804CF0D2FB9BF83C32002B00F02782079BA7
:20C58000002B00F0238218EE102A3946284605F02FFF012F00F0EC82042F00F05383102FC5
:20C5A00000F08682402F00F0AB83B7F5807F00F0B583B7F5806F00F0B983B7F5805F00F0E1
:20C5C000BD83B7F5803F00F0C1836A6D05F11800082342F400626A6577490422DFF800C286
:20C5E000C95C1CF803C00B5802FA0CF223EA02030B502B6843F001032B600D9B002B00F05D
:20C60000B3822B6A43EA87072F62099B9E420BD16B6C43F400436B642B6843F080032B60B0
:20C620002B6843F001032B609BF83032002B40F0A782039A012304990AF1A00A01320AF8F4
:20C64000913C4B7401F11803082A039204937FF44BAE0F9B89E1DFED598A594AB0EE688A81
:20C66000584BCBF8AC210022CBF8A831564BCDF81080039238EE887ADFED547AF5EE006A2F
:20C68000534C28EE278ADFF85CA1B0EE67AA0027C6EE879A9FED4F9ACBF8B431CDF814803F
:20C6A000029BBB426DD01AF8015B032109EB0503013593F8638EEDB240462A4631F01CF899
:20C6C0000646002800F0B782404634F045F8606110B10323C5718371327A022134F08EF88B
:20C6E000049B002B00F0EE81B9F85C3E4FF6FF7107EE903A384BF8EEE77AD3F87421FCEE3E
:20C70000E77A17EE903AB2FBF3F00144090CB2FBF1F2B2FBF3F399F85E1E042900F0E4814D
:20C7200007EE902AF8EE676A26EE887A69EE477A99F85F0E03999BB201902046E6EEA87A91
:20C740000091314684ED027AC4ED037A28F07AFE002F40F3B58161681D4B02E09C4200F0AD
:20C76000AF815A6818338A42F8D1059B013783F0010301221834082F04F8083C04F8072C83
:20C780008ED1164ECBF82C62DBF82C3263B300220121029883F82D1083F82C001A6383F809
:20C7A0002E2017B0BDEC068BBDE8F08F70D30508E01A002000D0121368D80508000000005A
:20C7C000A50203080DC4030801C403086F12833AAC13002000007A44802A01206C140020B5
:20C7E0005CD80508E6490120C54DC64C0FCD0FC40FCD0FC495E80700A4F1200384E8070077
:20C80000CBF82C32CDE7C04D0BF5C874DFF854930FCD0FC40FCD0FC495E8070099F85E3E2D
:20C8200099F8606E84E80700042B00F23C8101A252F823F051CA0008A7CA000847CA000893
:20C8400025CA000857C6000899F85E3E082B00F00281029B0026AD4DCBF83432AC4C99F87A
:20C860005E7E8AF804658AF83C750FCD0FC40FCD0FC499F8623EA4F58A729B1B049295E8D1
:20C88000070018BF0123354684E8070031464FF44C72A0488BF8303250F0F0FB9E4BDDF87A
:20C8A00010809E4E0393CDF810900AE034F018F9F368082D06F1200608F1180848F8043C9C
:20C8C0005DD0DBF83432AB4259DD039A12F8013B0392049A134493F8637E384630F094FFC5
:20C8E0000446384633F038FF049A8146E77992F85F2E0AB187F0010707F001049BF830221F
:20C9000001348AF803450AB187F00107484633F0EFFF002800F084814846013536F02CFE0E
:20C92000C6F80C9061017060EAB2377441F001017161B9F1000F05D04FF0030389F80720A4
:20C9400089F80630484633F091FFF9074846ADD434F0CCF8ACE79BF83C32A3B9704900231C
:20C96000704ACBF81412CBF81C22CBF82C320BE7082B7FF4B1AC6C4BCBF83832ACE46448DD
:20C98000CBF82C0200E7D4F81480B8F1000FE5D0A36940460B9336F0E3FE644B2422451E63
:20C9A0000A9002FB053595F8C831392B00F02C8120684BF0AFFD024639210A98D2B236F0C2
:20C9C000DFFE0028CAD000230793D7E40A9890229AF8113056494DF07DF9D4E5B823721CA5
:20C9E00003FB06B38BF84022C3F84452EFE48D231322CAF85C30B7E59BF83C32CAF8547021
:20CA0000002B7FF447AD1F461A4641E001224FF4807307F00207CAF86820CAF87C30CAF8CB
:20CA200074701AE59FED438ADFED438A002E3D4A424B16BF414600211346414A049141495F
:20CA4000CBE96A2116E69FED408AF0EE488AEDE7DFED3E8A01E60BF5FC733D4D99F8626EEC
:20CA60001C460F93003E0FCD0FC40FCD18BF01260FC4384B8BF83062CBF8103295E80700F7
:20CA800084E8070077E7344A02EB4303B3F83C24DAF89810AAF80C20B1F8B43023EA020322
:20CAA000A1F8B430FCE49FED2D8AF0EE488ABDE7AA6905F11800022342F40062AA618BE529
:20CAC000002353E6FAFE697AFCEEE77A244B17EE901AD3F874214FF6FF73B2FBF1F11944B3
:20CAE000090CB2FBF1F216E607EE903AB8EE677A07EE902AF8EE676A27EE0A7A16E600BF95
:20CB0000C8D7050878510120D0D60508F4D70508A0140020A02B0020E6490120D02E0020C7
:20CB200009C4030801C40308394104080000012095370000ACC5A737ACC5A73601FE020834
:20CB40000DC40308A5020308282930386F12833A20D80508398E050870D305086F1203396A
:20CB6000802A0120783B01202B6A1F432F624CE5AA6905F11800002342F00802AA612BE5C2
:20CB800023684FF6FF7162793433995051E5D8F800205FFA88F3182128F0FF0022F00102CB
:20CBA000103BC8F80020B3FBF1F106F0CBFD0A984DF0B6F878E45FFA88F31821024628F0A6
:20CBC000FF00103BB3FBF1F106F076FDD8F8003043F01003C8F80030ADE40B9A5821DFF856
:20CBE000A0C1CAF83C20039A01FB02C12268CAF84830CAF89C1002F13403CAF81C10627935
:20CC00001344CAF8183070E420684BF083FC95F8C93183427FF4CCAE089B0793FFF7AEBB48
:20CC20004E4B01224E498AF80425CBE977314D4BCBF8E831A4E64C4A4A4BCBF8AC21CBF81E
:20CC4000B4319FE5AA6905F11800012342F00802AA61C1E400224FF0FF311346ADF8442047
:20CC6000129214928DF854201391404A52F8332095424DD001330E2BF7D10020069B9A1F03
:20CC80000C92FCF7DFFE2B6839499DF8302023F00103D1ED5D7A022A2B60F8EE677A22D808
:20CCA0003449DFED356A01EB820292EDFF7AB8EE477A87EE870A30EE260A4EF0FBFE069B91
:20CCC0000138082BADF8440014BF13225F22002311A92846139214938DF85430129305F03C
:20CCE000D9FCFFF79CBB9FED257A9FED230AA7EE870A4EF0DFFE01381322ADF84400E6E7C9
:20CD0000AA6905F11800032342F00802AA6163E4184A02EBC30393F89003AFE7EA6905F12C
:20CD20001800042342F00802EA6155E4EA6905F11800052342F00802EA614DE4EA6905F16A
:20CD40001800062342F40062EA6145E46A6D05F11800072342F008026A653DE40DC403086F
:20CD600009C4030801C403080DFF0208FCD60508802A012070D305080AD7233CFCF4B234E5
:20CD8000E023002070B5524E96F8600233F0E4FC96F8615260B12D2304462021C38033F025
:20CDA00065FD0A2030F008FF204636F0DBFB18B9D6F84035DA0000D570BD013D092DFBD827
:20CDC00096F85F42CCB940202BF052FA0028F3D090F9043096F83112092BC8BF143B0A2922
:20CDE000334493F8444566D093F8503596F85E22002A08BF1C46002CDED0204633F0ACFCF6
:20CE0000054608B12D23C3800121284633F02EFD0121084633F068FF0121284633F01AFFD7
:20CE20003C2030F0D5FE0021012033F05DFF96F861321BB3002400210134084633F054FFB5
:20CE40000021022033F050FF0021284633F002FF782030F0B1FE0121002033F045FF012138
:20CE6000022033F041FF0121284633F0F3FE782030F0A2FE96F861329C42DCDB96F85F325C
:20CE80008BB9D6F8603203F0FF13B3F5803F93D1D6F8403513F080538ED186F86132BDE8F0
:20CEA000704043F02FBA322030F092FE2846002133F0DCFCE5E7D6F868355B057FF57CAFE4
:20CEC0000EF072FC00287FF477AF002C95D173E7704C012030B40438043A0C1F01F10805D4
:20CEE00054F8043F52F8041FAC42A3EB010340F8043FF5D130BC704738B5041E0D4611DB84
:20CF0000092C1FDC0846134B0021134AA3FB04C34170DB0803EB8303A4EB4303D35C0370D3
:20CF2000284638BD64422D230846092C00F8013BE9D9084B01460A22A3FB0430C00842F08D
:20CF400009F9E0E703480A22A0FB0430C00842F001F9D8E7CDCCCCCCDC5C0608344870B4F8
:20CF600090F86C35A3F13001092958D800F26C5400F27B50224612F8015FA5F13001092927
:20CF800004D88242F7D1002070BC7047141B022C4BDD2848002101E010F8013B01EB81017D
:20CFA000161A044603EB4103022EA3F1300303F0FF01F1DC204B03FB01F1A2424FF000038D
:20CFC0000ED903EB830314F8016B5B00A242A3F13003334403F0FF03F3D1184800FB03F3F7
:20CFE0002E2D06D01648A0FB032370BC01EB9300704701320425002404EB84041078013DC2
:20D00000303864000928A4B2204401D8013284B215F0FF05F0D1642202FB0433E2E70021A9
:20D020001D4600F26C520B46DAE70021054CC4E7704C0120DD5101208096980040420F0043
:20D04000ABAAAAAADC51012038B50D460446FF2100682A4650F012F822682A44226038BD9E
:20D060000C461646054683B529F07CFB204629F079FB0021204B0846002E08BF1E4633F0A6
:20D0800033FE0021012033F02FFE284630F01AFEB0B10121002033F027FE284630F00AFEA6
:20D0A0000746204630F00AFE0028FAD03946204630F02EFE3846B0470021084633F014FE59
:20D0C000204630F0FFFD0028DFD00121002033F00BFE204630F0EEFD01462846019130F0B1
:20D0E000EDFD01990028F8D0284630F011FE0021084633F0F9FDC8E7B5570308F0B500220A
:20D1000089B0234E04AF13460A61BC46C1E90022C1E902220268C2F3855040FA03F4654682
:20D12000E40703D59C5D05F8014BAC460133062BF3D1184DC2F303240023C2F305302C5DF8
:20D140000DF119068CF80030DFF850C08DF8184040FA03F43546E40704D513F80C4005F876
:20D16000014B2E460133062BF2D10023C2F3834506AC0846337002F00F030749C2F3031266
:20D180000097CDE9014542F0E9FD09B0F0BD00BF245D06081C5D0608045D0608145D0608BB
:20D1A00070B5094C0546D4F87C2562B1002601362D21D4F87C0538F02FF8AE42F7DBBDE87C
:20D1C000704038F0D3BA70BD704C012038B50546084641F06DFE041E0D4B0FDB93F88C251E
:20D1E000944205DA21460B4839F0F0FD204638BDFF2C03D1084839F0E9FDF7E793F88C25D7
:20D20000284606494FF0FF34013A38F075FAEDE7E4010020345D0608455D0608585D060822
:20D2200030B583B04D1C0093002304688572C272A469A04703B030BD03685B6C0BB102217B
:20D240001847704770B5104ED6F82C3293F82E20CAB19B699847B0B1D6F82C3293F82C206E
:20D260006AB10A4D0024DB69E0B2B5EC010A01349847D6F82C3293F82C209442F3DB5B6A16
:20D28000BDE87040184770BDDC1200206030002038B51E4C0968D4F884550068491B1C4D4D
:20D2A000DFED1C6A00EE901AD4F88015D5EDFB7A1C46F8EEE00A401A60EEA70A07EE900AD2
:20D2C000F8EEE77A20EEA07AB1EE670AA7EEA77AF1EEC77A67EEA67AFCEEE77AC2ED007A10
:20D2E00042F06AFE9FED0C7ADFED0C7AE0EE077AFDEEE77A17EE902A002A02DBC4ED007AA4
:20D3000038BD48F6A0431344236038BD704C0120000001202C7D8E3FA00CB34500A00C461E
:20D3200038B50F4C034694F89F1504F5B36084F89B3501F03F0101F10A058B1C083184F836
:20D340009A55254484F89D351FF0C4FC85F8960594F89A35000A1C4484F8970538BD00BFAF
:20D36000704C012038B50A4C00250122802120462AF06AFF30B194F904002AF099FF08B1DE
:20D38000006838BD01350C34092DEED10020F8E73052012038B5041F00F1080554F8043F86
:20D3A000D81780EA430018F065FCA542F6D138BD074B4FF6FF70002103F6AC4210B40024CF
:20D3C000C3F8280D5167C3F8244D5DF8044B7047D4230020F8B5794CDFED797AD4F8302DAD
:20D3E00094F8103D07EE102AB4F8127D2DED028BB8EE478A28EE278A002B68D1D4F81C6D4C
:20D4000094F82D1D304626F097FC0F2894F8113DB8BF0F2085B2A4F8125D002B00F0BB80C8
:20D42000AF4258D094F8AC6CB4F8143D07EE905ADFED645A002206EE103AF8EE677A6249F7
:20D440000020B8EE466AC5EEA76A0B4685EE867A76EE886AC8EE267A37EE087AC8EE076A54
:20D4600096BB58609860D860C3ED047A01321033032AF5D1002E34D094F8163DB4F8185DAA
:20D48000C1ED106AC1ED147AC1ED187A002B7CD194F82D1DD4F81C0D26F04EFC0F28B8BF97
:20D4A0000F2080B28542A4F8180D6ED000286CD007EE900ADFED436A444BF8EE677A86EE0F
:20D4C000A77AD3ED006A56E0C3ED047ACEE794F8113D002B5CD094F8AC6C002E66D13D462B
:20D4E000A2E7002394F8162DB4F8185DC1ED106AC1ED147AC1ED187A4B638B63CB634B6473
:20D500008B64CB644B658B65CB6562B994F82D1DD4F81C0D26F010FC0F28B8BF0F2080B206
:20D520000546A4F8180D41F26D0394F82C2DE2545DB307EE905A254BDFED226A0022F8EE62
:20D54000677A41F26C010120C3F80823C3F80C2386EEA77AD3ED006AC3F81023C3F81823B6
:20D56000C3F81C23C3F82023C3F82823C3F82C23C3F83023605437EE267AC6EE877AC3EDB7
:20D58000C57AC3EDC97AC3EDCD7ABDEC028BF8BDD4F81C6D3D46304694F82E1D26F0CCFB75
:20D5A0000F28B8BF0F20A4F8140D39E794F8163DB4F8185D002B3FF46BAFE6E7D423002055
:20D5C000BD3786354E2DA63D8030002008310020012817D0304A41F29303D35C012B2DD06A
:20D5E0002E4BF6EE006ABEEE007ADFED2D7A03EB800090ED000A80FE660A80FE070A20EE4B
:20D60000270A7047274A41F294032349F6EE006A02F5C960BEEE007ADFED217A90ED010AF8
:20D62000CB5C80FE660A80FE070A20EE270A23B1B5EEC00AF1EE10FA03DC70479FED1A0A97
:20D64000704707EE903AB2F93216B2F94636DFED176AF8EEE77ACB1A07EE103AB8EEC77A9B
:20D6600027EE267AB4EEE77AF1EE10FAE6DA77EEC77AB2EE047AF4EEC77AF1EE10FADCD8C5
:20D68000B1EE047A67EEA67A30EE470AA7EE807AB0EE470A704700BFD4230020B852012053
:20D6A00000004843704C012000000000CDCCCC3DF8B5744B40F60301B3F854260A402DED31
:20D6C000048BB0EE408A04D0B0EE480ABDEC048BF8BD03EB4003B5EEC00ADFED6B7A00F162
:20D6E000D40EB3F93016B3F94436F1EE10FA674DA1EB030305EB8E0CC8BF012600EE103A91
:20D70000D8BF4FF0FF36DCF8344D05F63457B8EEC00A20EE270AB5EEC00AF0EEC07AF1EE10
:20D7200010FACCBF01214FF0FF31A31B18BF0123002C08BF0023002B49D197EDCF7AF4EE00
:20D74000C77AF1EE10FA07DD8E4208BF002C0CBF0123002300F08180002C42D007EE901A18
:20D76000B0EE408AD7EDD25AF8EEE77A9FED486ADFED486ADFED488A97EE878A28EE258A55
:20D7800088FE468A88FE268A002B58D141F27803EB5C984298D1414D95F8983D262B93D1CC
:20D7A000B2EE049A20EE090A4EF084F9B0EE480AA5F89E4DA5F89C0D4EF07CF928EE890A35
:20D7C000A5F8A00D4EF076F9A5F8A20D7CE797EDCF7ACCF8342DF4EEC77AF1EE10FA3ADC8F
:20D7E00013462F4A9FED2F6A02EB8002D2ED097AF0EEE76AF4EEC66AF1EE10FA28DC9FEDC7
:20D800002A6A66EE866A97EDD06AF0EE408A67EE867AE6EEA78AF5EEC08AF0EEE87AF1EE24
:20D8200010FAF4EE477ACCBF01224FF0FF32F1EE10FA01DD964217D00024002BA6D01B4A6D
:20D8400000EB8003002102EB830343F8341C9DE7F7EE006AD7E78E42C2D105EB8E0E0C4669
:20D860000123CEF8341D77E707EE902AB0EE688AD7EDD26A0024F8EEE77A97EE878A28EEB9
:20D88000268ADCE7704C0120CDCCCC3DD423002000007A4400007AC400000000783B0120AF
:20D8A000E4010020FFFFF9436F12033BCC34002070B504466F4EC0B22DED048BF0EE408A5B
:20D8C0000D7820F07FFB6C4A06EB8403694207EE905AD3F8583607EE101AF8EEE76A82FB55
:20D8E0000312DB17B8EEC77AC3EB621307EE903AF8EEE77AE6EE807AF4EEC77AF1EE10FA37
:20D9000005D407EE105AB8EE477A87FE677A06EB4404DFED5A9A40F60100B6F85426B4F9FD
:20D920003036B4F944161040A3EB010307EE903AF8EEE77AA7EEE97AB0EE478A07D0504BB9
:20D94000BDEC048B93ED7C0A27EE000A70BD20F039FB0120B0EE409A20F034FBB6F930360C
:20D96000B0EEC00AB6F93216002B464AB0EEC99AB8BF5B42002992F8380FB8BF49429BB22F
:20D9800089FE009A89B28B42B8BF0B4607EE903A02F63453F8EEE77A67EEA97A50BBF7EEA9
:20D9A000006A93ED807AB4EEE67AF1EE10FA50D493ED7E7ADFED347AB4EEE77AF1EE10FA96
:20D9C00044D9DFED325AB7EE006AC5EE876AB0EE467AA9EE667AC7FE466AC6FEA76AD3ED40
:20D9E0007D7AB0EE680A68EE277ABDEC048BA7EEA60A70BD9FED246A93ED7E7AB4EEC67A0B
:20DA0000F1EE10FA1FDDD3ED7F5AF4EEC65AF1EE10FA18DDDFED1E6A75EEE77AB7EE005A91
:20DA200029EE269AC7EEA56AC9EE077AC6FEC56AC6FE866A77EE857A66EEA76AC6FEC56AB0
:20DA4000C6FE866ACBE7F0EE466AC8E7F0EE676AC5E776EEC76A9FED0F5A9FED0F6AD3ED79
:20DA60007E5A66EE856A76EE677AA6EEA77A27EE257A9FE7704C01201F85EB51CDCCCC3DF8
:20DA800008310020D4230020000000000000C8420000C8C2610BB63B000034431C4991F8C0
:20DAA0006C259AB3F0B4002605463346304637461BB991F86C452D2C22D02E2A18D0CA188C
:20DAC00000EB800092F86C454000A4F13002092A02D8A0F13002A0180E2B14D80133CA18D6
:20DAE00092F86C25002AE3D106B14042F0BC70470133002DF8D0CA182A4482F86C75DEE7F8
:20DB000001231E46EBE70020F0BC704700207047704C01202DE9F041A02301240B4F1825AE
:20DB2000E6B2FF2B0BDCC5F11B0103F101083246DBB2C9B2D7F86006FFF772FB4346013D8E
:20DB4000EFD10134052CEAD1BDE8F081704C01201FB503AC8DF80C30002300948DF80D3034
:20DB60000EF0F0FC04B010BDF8B50546262023F0F3FF144C014608BBD4F8640690F8383067
:20DB80001E3B012B02D894F871360BB130F0C0F80D4F0026AE4209DBB4F892360133A4F8C5
:20DBA00092360A4B9B6AC4F8A436F8BD17F8011B0136D4F8640630F0ABF8EBE7002384F82C
:20DBC000A036EEE7704C0120E2520120802A012010B51C2032F0C0FD0446112132F046FEDB
:20DBE000204632F07DFFC8202FF0F2FF2046BDE8104032F07BBF00BF08B5002032F0ACFD0B
:20DC0000054BC3F8A80608B12A23C3804021BDE8084032F02BBE00BF704C0120F8B56A4CAA
:20DC2000D4F834110B699E0702D5CB689D074BD40B69580702D5CB685A073DD40B691B0708
:20DC400002D5CB681F072FD40B69DE0602D5CB68DD0621D40B69D80702D5CB68DA073FD406
:20DC60000B691B0603D5CB681F0600F191800B69DE0503D5CB681D0600F18E800B695C0683
:20DC800003D5CB68580600F18B800B699A0602D5CB689B0620D4F8BD6FF0100200230A61B8
:20DCA000CA6984F85031D5E76FF0080200230A61CA6984F85031C7E76FF0040200230A61B0
:20DCC0008A6984F85031B9E76FF0020200230A618A6984F85031ABE76FF020030B61F8BD9E
:20DCE0003A4B6FF0010299420A61B9D141F204133748C558D5F81432002BB1D1354FD7F874
:20DD0000AC2692B1D0F858C602F03F066244C0F85826D0F85826B2F5006F01D1C0F8583681
:20DD20000023C7F8AC36002E44D0D0F85826D0F85C369A4294D0D0F85826D0F85C369A4281
:20DD400032D9D0F85866C6F50066D0F858C6B6F5007F214A28BF4FF40076D5F8143262443D
:20DD6000C5F81062C5F80822002B7FF479AF012341F21C11C0F8A46EC5F814323346405865
:20DD8000812106F035F9D4F83411C7F8AC6667E76FF080030B616AE76FF480730B616DE7D8
:20DDA0006FF040030B6170E7D0F85C66D0F85836F61ACAE7D0F85826074BC5F8106213443F
:20DDC000C5F808324CE700BF802A01200014004088190120704C0120FC1F012070B5D0F873
:20DDE000A852C1EBC1000C46002605EB80001C21C0F80822C0F8103280F8FC41C0F81462D8
:20DE000080F8FD612B6901FB0451012B01F5FE7108BFC0F80C22DAB228681CB905F042FEE3
:20DE2000002070BD05F0CAFE002070BD0E4841F20413C35810B5A3B190F8844E00F6746093
:20DE4000D3F8042234B1002440230121FFF7C6FF204610BD4FF400730121FFF7BFFF204663
:20DE600010BD0224204610BD8819012010B50C4CD4F8603663B10B49013BD1F8B026C4F83C
:20DE8000603612F8014BC1F8B026047013B10123184610BDFFF7CAFF0123184610BD00BFB3
:20DEA00088190120704C012013B5074CD4F8B03603B9FEE701A8FFF7D9FF0028F6D09DF85B
:20DEC000040002B010BD00BF704C012010B50B68064C074AC4F86036C2F8B0060BB10020AA
:20DEE00010BDFFF7A3FF002010BD00BF88190120704C012038B5D0F8A84201F00F03626806
:20DF000093422BD80A062BD41C25C1EBC102002005FB014104EB820201F5FE7182F8FD01B8
:20DF200001220B708A7094F8BC03904216D084F8BC234A782068012A09781DD000F5306281
:20DF400002EB41121568002D00DBF1B9116841F4001111601BB3002384F8BC33002038BDB1
:20DF60001C21C3EBC302012001FB034104EB82023C3182F83D00D3E700F5106202EB411298
:20DF800015680029E2D0002DE0DB116821F080411160116841F400111160002BDBD104F585
:20DFA0007172217C05F052FDD5E700BF10B504468021FFF79FFF00212046BDE8104099E7E2
:20DFC00011F0800F01F00F01F0B4D0F8A8424FF01C0042D1C1EBC10500FB0140002604EB29
:20DFE000850500F5FE7085F8FD61457801708360C27005B1C180022A01D10023037194F8FE
:020000040800F2
:20E00000BC33012B1AD00122236884F8BC234178057891422CD003F5006605F00F0103F592
:20E0200030638A40F16903EB451341EA0242F2611A68120405D5002384F8BC330020F0BC55
:20E04000704782681D68C2F30A02C07818492A4342EA804211431960EDE7C1EBC1050126AB
:20E0600000FB014004EB85053C3085F83D60BCE705F00F06D3F81CC803F5106203F5006740
:20E08000B14002EB451241EA0C01F96113681904D1D483681668C3F30A03C0780449334355
:20E0A00043EA804343EA855319431160C3E700BF008000102DE9F04F854D83B02C6E6369E5
:20E0C00013F0010B02D003B0BDE8F08F6269A3691A42F8D06369A26913409E0703D563691A
:20E0E00003F0020363616369A2691340180379D42046436982691340590300F1D480426936
:20E1000083691A4200F1B9804369826913401A0508D5D4F80838DB0700F15383436903F44F
:20E12000006343614369826913401F0110D5436903F00063436195F85434002B40F04A8207
:20E14000012385F85434436DC3F38303C5F85834436982691340DE0400F1D38143698269B9
:20E1600013409A0400F17681436982691340DB0612D5836923F010038361236AC3F3434256
:20E1800003F00F01022A00F0E582062A00F05E82836943F0100383614369826913401F07D3
:20E1A00000F10D82436982691340DE0200F102824369826913409C0200F1F7814369826918
:20E1C0001340590000F1EC814369826913405A077FF579AF4468630700F1E78243681C43D4
:20E1E000446070E7D4F81868D4F81C381E40360C3FF47EAF374B20460027CDF800B0994655
:20E2000006E0760807F1010709F11C0900F03282F107F6D5F9B200F5306A0AEB4112926898
:20E22000D0F8143802EA030818F0010F40F0288218F0080F40F05C8218F0100F05D004F5BF
:20E240003063102203EB47139A6018F0200F09D0296F012900F0568304F53063202203EB60
:20E2600047139A6018F4005FCBD004F530634FF4005203EB47139A60C3E7D4F8043823F01C
:20E280000103C4F8043895F85434012B00F0B781D5F8603493F8752283F87422436903F0E6
:20E2A0000043436130E7D0F81838D0F81C2803EA02081FFA88F8B8F1000F3FF420AF054E9F
:20E2C0004FF0000A04F51067CDE9004B0CE000BF88190120E81901205FEA58080AF1010A46
:20E2E00006F11C0600F0C98118F0010FF4D05FFA8AF9D0F81028D0F8344800F5106309F06E
:20E300000F0103EB4913CC409B68E401E4B214431C40E20732D54FF0010E009B0AF00F0C78
:20E3200007EB4A12D3F834180EFA0CFC21EA0C01D5F870C0F445C3F83418C2F808E003D19D
:20E34000D6E911231344B364D5F860B4B9F1000F40F0E681DBF86C32022B00F0D88233F020
:20E36000040300F01A839BF87832012B02D100238BF87832BCF1010F00F0F182230703D55B
:20E3800007EB4A1308229A60E10603D507EB4A1310229A60620603D507EB4A1340229A60E5
:20E3A000A30703D507EB4A1302229A60210693D5D6E91441A1428FD8621A736C00EB4A1CD5
:20E3C00093420CF5106C28BF1346DCF81820033392B2B2EB930F2ED309F10109864600EB2A
:20E3E00009393CB3A14280F0C682621A736C95F870009A4228BF1A46B36C02F1030B4FEA7D
:20E400009B0B70B990B2033080080AD003EB800153F8040B8B42C9F80000F9D1B36CD6E957
:20E420001441DCF818001344114480B2B36471658345D6D97046A142FFF44EAF0AF00F01C6
:20E440000124D0F8342804FA01F122EA0102C0F8342841E7D0F8001900F50063B84A0A40B3
:20E46000C0F800299A6802F00602042A00F0CB805A6842F480725A609B6813F0060340F073
:20E48000AA81C268EB6622F47052C260C36843F41053C3604FF00009D5F860644FF0400894
:20E4A00000220127434630461146FFF789FD4346002230468021C6F84471C6F85081FFF786
:20E4C0007FFD0023D6F8A022B761C6F8248086F87472C6F86C327360C6F87C32002A00F07A
:20E4E000EC81D6F88C32304600215B689847D5F86034286E83F81090436903F4005343613E
:20E5000032E6D4F804284FF4846104F500678D4B22F001027A60016101E0013B02D00269E0
:20E520009106FAD4D5F864C0BCF1000F16D004F510634FF67F3199600BF1010B1A682033AC
:20E54000E34522F4001243F8202CC3F8E811D3F8E02122F40012C3F8E021ECD1FB69D5F892
:20E56000902043F00113FB61002A3DD17A6942F22B0313437B613B6943F00B033B61D4F84C
:20E58000003895F8701023F4FE636F4AC4F8003805F05CFA286E436903F480534361DDE554
:20E5A000436903F0804343610EE6436903F40013436103E6436903F480134361F8E5D5F89A
:20E5C000603493F87422032A37D0436903F008034361E7E5D5F86034042193F8742283F816
:20E5E000741283F87522B3E5D7F8843043F00B03C7F884307B6C43F00B037B64BFE70023E4
:20E6000085F854344AE6D0F8002942F00302C0F800295A6842F480725A609B6813F0060309
:20E6200040F0D980C368002223F47053EA66C360C36843F41053C3602CE7D3F88C22D26908
:20E64000002AC2D018469047286EBEE7C1EBC10104F58054C3F30A1305EB81022668D2F8B5
:20E660007412C5F824640B442168C2F87432C5F828148DE5DDF800B03BE5DDE9004B3EE553
:20E6800004F530634FF0010C2A6F0AEB471A03EB471B6245CBF808C0D0F840E0DAF808303F
:20E6A00000F01681294A964540F0FB801A0440F1F3804FF4004218F0080FCAF808203FF457
:20E6C000BBAD026CDAF80800204B9A4200F0D0801D49D5F86004019206F080FB1C4B019A66
:20E6E0009A4200F2D0800822286ECBF80820A3E57B01296F026C03F5306A012904F5306101
:20E70000824401EB030BDAF80800DDD1104B9A4200F2AE800C49D5F8600406F05FFBE2E7BB
:20E72000DBF88C325B69002B3FF428AE9BF87422032A7FF423AE584649469847286E1DE611
:20E7400000F8FFFF400D0300AC1D01200A31544F0A30544F47F6F07213423FF419ADC3F32B
:20E760000A16C1EBC1024FEAC10C3346033605EB8202B608D2F8682208D004F5805402EB3A
:20E780008607266842F8046BBA42FAD1ACEB010205EB8202D2F86842D2F874121C440B446D
:20E7A000C2F86842C2F87432F2E4D5F860040122D0F88C3280F8742201795B689847286E25
:20E7C0000CE5D5F86034042193F8742283F8741283F87522A2E423F00403002B3FF422AFBF
:20E7E000A74A0326A74BD2F87421A7491344EE668B4240F2C280A54BA54913448B4240F29E
:20E80000D480A44BA44913448B4240F2F380A34BA34913448B42C0F02481A24BA24913447D
:20E820008B4240F22181A14BA14913448B42C0F01E81A04BA04913448B42C0F01E819F4BBD
:20E840009F4913448B42C0F015819E4B9E4913448B4234BF4FF4E0534FF4C053C2684FF04A
:20E86000010922F47052C260C2681343C36013E6000403D54FF40042CAF808209349D5F804
:20E88000600406F0ABFA296F01297FF42CAF8F4A286E05F0DBF826E79B0602D52023CAF8A8
:20E8A0000830C1EBC103D5F8600405EB8303D3F8682206F07FF8286EBAE4D6F89032002B58
:20E8C0007FF40FAED6F89832002B7FF40AAE0EE61A0755D57E4A964505D9190403D54FF422
:20E8E0000043CAF808307949D5F8600406F076FA764A0121286E05F0A9F80823286ECAF8F1
:20E90000083095E4714A05F0A1F8286EA4E4DBE908239A4259D8DBF81C10B1FBF3F203FB55
:20E9200012120AB98B4268D9DBF88C32DB682BB19BF87422032A01D158469847802158464E
:20E94000FFF7D8FA0023052258461946CBF86C221A46FFF743FAD5F870C0286E03E5D5F87C
:20E96000B0305AEA03037FF409AD6146574A05F06DF8286E02E5704660E54FF470536DE7D0
:20E980009A0615D52022CAF8082018F0080F3FF453AC026CDAF80800B8E680215846FFF755
:20E9A000A9FAD5F870C0286EDDE44FF4605355E713F0280FE9D1464A96452CD91B042AD5AC
:20E9C0004FF40042CAF80820DFE7D31A4946D5F8A820DBF8A802CBF820309BB205F008FB1C
:20E9E0004B464A4649465846FFF7F8F9D5F870C0286EB8E44FF4505330E7DBF87032994266
:20EA000092D24B464A464946DBF8A80205F0F0FACBF87092E4E7DAF81020C1EBC100D9F8B6
:20EA20000432C2F3120CD9F8082205EB80001A44A3EB0C03C9F80822D0F86822D5F86004F9
:20EA4000C9F8143205F0B6FFD5F870323B437FF432AF1E4A0121286E04F0F8FF286EFFF72D
:20EA6000E7BB4FF44053F9E64FF43053F6E64FF42053F3E64FF40053F0E64FF41053EDE629
:20EA8000802A0120405327FFFF340C00401E1BFF3F420F0000DC0BFF7F4F1200808CF9FEE2
:20EAA00020D6130060B6E5FE5FE3160000D3CEFE40771B00C05BB3FEC091210000CA91FEF4
:20EAC00020753800E05459FEE09C4100AC1D01200A30544F2DE9F0414FF0FF35324A002301
:20EAE00032482C4603E0013310320B2B14D0917A0429F8D103F5B17100EB0111C979CF0787
:20EB0000F1D4661C116801D0A942ECD21C4601330D4610320B2BEAD1631C02D10120BDE887
:20EB2000F081224D04F5B17705EB07139988E9B92601DFF88480AA19D8F87C3F41F218600C
:20EB40001B491E690023105801EB4421194AB047E0B1022817D141F2CC6205EB0717012160
:20EB60000020AB58B971013BAB50D8E7DFF8488005EB041241F218602601D8F87C3F1058E8
:20EB8000DB689847D7E70020BDE8F08141F2CC62032405EB071741F2D061AB58BC71012410
:20EBA000013B6C54AB50BAE7A88B01208C750120A4750120D5EB0008783B0120044B41F2EF
:20EBC000E472995C09B90121995401225A7070478C75012070B50024164D41F2D066164BDD
:20EBE0002046AC5503E0013010330B2814D053F80E4C8C42F7D11C78032CF4D16AB10F4B08
:20EC000003EB40239A4201D0FFF7D8FF00F5B170012305EB0010837170BD41F2CC6100F579
:20EC2000B17304206A5805EB0313013298716A5070BD00BF8C750120B28B0120A475012028
:20EC400038B50020114B9C7B14B11D688D4204D0013010330B28F6D138BD82B10C4B03EB6C
:20EC600040239A4201D1022C01D0FFF7A7FF00F5B170084B012203EB0010827138BD00F581
:20EC8000B170044B03EB0010827138BDA48B0120A47501208C7501202DE9F04F83B002F0F8
:20ECA000020C019310B9BCF1000F60D1844C41F638056559002D61D14FF0FF36814F002532
:20ECC000B146B046B2463B68984200F0BE8097F80EE0BEF1000F62D0BEF1010F15D105F598
:20ECE000B17E04EB0E1E9EF807E01EF0010F0CD11EF07E0F09D15FEADE1340F0B080D7F874
:20ED000008E0F24501D9F246A946013510370B2DD9D1751C04D1B8F1FF3F00F0A780464684
:20ED200041F2C86806F5B17704EB061E41F21C6A54F808504FEA071941F2186B01354EF852
:20ED40000B0044F8085004EB07184EF80A5044F809500025C8F8045004EB0715AD79042D36
:20ED600000F2A980DFE805F02139163955000225FFF724FF284603B0BDE8F08F04F5C25727
:20ED800041F63C063F68A65907FB0565A84293D3FFF714FF0025284603B0BDE8F08F2E46B1
:20EDA000013510370B2D8ED1B3E712F0010E6FD104EB0710019BD51090F80780032B65F338
:20EDC000C71880F8078061D94FF6FF70834228BF03469BB204EB07108380BCF1000F18D078
:20EDE00004EB061041F218630344987B042810D041F2C86C41F2CC654FF0040E54F80C0086
:20EE0000013044F80C00586083F80EE0635901336351500705D504EB0710C37943F001030A
:20EE2000C371D30608D504EB0714E379C3F34502013262F34603E371234B012503EB462672
:20EE400028460E6003B0BDE8F08F05F5B17704EB07164FEA071EB6796EB92E4660E7A84674
:20EE6000013510370B2D7FF42EAF52E7B9F1FF3F90D04E4654E741F2C8682E4654F80850C2
:20EE8000013544F8085044F80E5065E77346A1E70E4A00230C49D2F87CCF01EB46210C4AF3
:20EEA000DCF80860B04700283FF474AF04EB07140223A3715EE70225FFF780FE5AE700BF7E
:20EEC0008C750120A48B0120A4750120783B012041EC0008F0B5154D83B00E462B78022B1F
:20EEE0000FD14FEA102CC4B241F630070023012201A9E8596044FFF7CFFE012806D003B08F
:20EF0000F0BDC0F3D41C00F07F04EDE72B78022B019B04D133F81430336003B0F0BD53F86C
:20EF2000243023F07043336003B0F0BD8C75012010B5144602070B4610D50B4941F2C47287
:20EF4000581C8B58834204D305D100230120236010BDFFF733FE2060012010BD21461846FA
:20EF6000BDE81040B6E700BF8C7501202DE9F0410D46416882B00446C1F308032B44B3F589
:20EF8000007F58D390F91A30591C0AD0304A03F5B173FF2102EB0313DA796FF30002DA71EA
:20EFA000817694F91B305A1C0FD0294A03F5B173FF2002EB0313DA79C2F34501013921EAE9
:20EFC000E17161F34602DA71E0762378022B38D01F4A02F5C2531B68B5EB432F4FEA432824
:20EFE00025DC41F648036768D6583E407242AA421DDCAB19434512D301AA2169207EFFF780
:20F0000097FF012813D16768A5EB0805206908EB0703019A354460619F1B2261676020461C
:20F02000F9F74EFB20B93D440120656000E0002002B0BDE8F08129440120616002B0BDE8E9
:20F04000F081616801202944616002B0BDE8F0818C75012070B5154604460E46FFF786FFA4
:20F0600050B994F8280028B90223C4E90B5684F8283070BD022070BD1DB12046A84701202B
:20F0800070BD012070BD00BFD0E9011310B48B4290F91A2038BF0B46511C83600AD0144B44
:20F0A00002F5B172FF2103EB0212D3796FF30003D371817690F91B305A1C0FD00C4A03F5B1
:20F0C000B173FF2402EB0313DA79C2F34501013921EAE17161F34602DA71C4760022436A11
:20F0E0005DF8044B1146426142600361B2E700BF8C75012070B544220021114841F60204B0
:20F100004DF0BCFF0F4B032141F64C001A784FF6FF761D5803F5C050022A1E5341F2E876FF
:20F1200041F60C0418BF0A4600F8181941F601011D519A5510225A54FFF7A6FF012070BDD9
:20F14000748D01208C750120B1F904300F2B2DE9F0410C4682B01646054633D02846F9F780
:20F16000D7FA95F91B800746B8F1FF3F34D02D4B41F2186203EB08118A58904212D118334F
:20F1800003EB4823A1882846013109B203EB4113A1803360F9F7BCFA03460120236002B057
:20F1A000BDE8F081FFF70AFD2846F9F789FA28B100230120336002B0BDE8F081002002B011
:20F1C000BDE8F0814FF40071FFF7D0FE0028F5D04FF6FF73A380C1E72846F9F771FA002841
:20F1E000E2D10FB9FFF7EAFC38460023112201A9FFF752FD0128D7D1019B0B4A9A1A48BF78
:20F2000002F2FF12B2F5B05F4FEA622106D24FFA81F885F81B80002BB4D1C5E7FFF7CEFCA9
:20F22000019BF6E78C750120A475012030B50446C06983B010B9012003B030BD0D4600236E
:20F24000032201A9FFF728FD0128F5D1B4F92030002B03DAFFF7B2FC0220EDE7019A012D6D
:20F260004FEA431102EB431303D0022D12D1E5255554A268DA612278032A04D100221A7792
:20F280005A779A77DA77626AC2F30F415A83998203B030BDE268DA61EDE700BF10B503787A
:20F2A0000446023B012B037E02D913F0060F5AD198063AD494F91A30591C0AD02D4A03F5BB
:20F2C000B173FF2102EB0313DA796FF30002DA71A17694F91B305A1C0FD0264A03F5B17315
:20F2E000FF2002EB0313DA79C2F34501013921EAE17161F34602DA71E076237E1B070BD527
:20F300001C4841F2C873C35C072B01D0FFF756FC41F2C8730022C2540023E26A237084F88D
:20F320002830FAB1BDE81040104700231249E0691A018A58904206D001330B2BBAD01A0103
:20F340008A589042F8D10B4A03F5B17302EB0313DA79C2F34501013921EAE17161F346023B
:20F36000DA71A7E710BD0121FFF760FF0128F9D1237E9DE78C750120A48B0120B8B138B590
:20F38000027822B190F828201AB1002038BD012038BD826803244568C162AA4280F82840AD
:20F3A00038BF2A468260FFF779FF012038BD0120704700BF2DE9F04FDFF84C91174683B050
:20F3C0008A4699F800300A68022B7BD1D6B241F630044FF48071A6EB020859F80450B8444E
:20F3E00005EB12258844BA4208F1FF38B8FBF1F864D200F0010BA844032B06EB0704A8EB77
:20F4000005030CBF80214FF48071A41A8C4228BF0C460EB98C4235D20B2201A92846FFF7A8
:20F420003BFC012802D003B0BDE8F08F99F80010DAF80020022902F1010325D0A64210D24F
:20F44000019A6FF04040111F304401EB840102EB800242F8043F914203F10103F9D1DAF8CA
:20F460000020A61B3244BA42CAF8002002D1BBF1000F39D1BA4205F101051FD299F8003015
:20F480000026B9E70A22C8E7A642EAD201996FF0004C881EB44400EB440001EB4C0121F8C3
:20F4A000023F884203F10103F9D1DAE76FF00043019A4FF6FF71234422F81310012003B054
:20F4C000BDE8F08F41F6300102F07F06032BC2F3D41559F80140A6EB020814BF4FF4807129
:20F4E0008021B84425447DE799F80030022BDDD06FF04043019A4FF0FF31234442F8231047
:20F50000DAF80020B6E700BF8C750120F8B590F838300446032B4ED8DFE803F002303944D7
:20F520002B4B41F2A87EC56841F2C47C187803F5C25153F80C2041F2AC770328096853F80D
:20F540000E000CBF80264FF48076226101FB06F105EB4125A0EB4120E560951943F80E00FF
:20F56000D85943F80C50A0EB4121E06AD951C4E90C2548BB6262012384F838300021154837
:20F58000FFF754FE012811D1022384F83830626B04F130010120FFF70DFF012806D10323D3
:20F5A00084F8383000212046FFF740FE431EDBB2012B01D9F8BD022094F82830062BF9D102
:20F5C000002384F82830F8BD921B2263D3E700BF8C7501202C8D01202DE9F04FDFF8248107
:20F5E000012887B00C4698F800608CBF002301231546032E02930B6839D0022E62D14FF494
:20F6000080724FEA1329DFB201920138012823D8012203929D421AD9384E06F1880A06F172
:20F620001C0B32681AB1DBF8001099424ED0DAF800000023092205A94844FFF72DFB0128C1
:20F640001FD002280FD020B123689D42E9D80320256007B0BDE8F08F87B1FFF7AFFA02203A
:20F6600007B0BDE8F08F022007B0BDE8F08F80220192C3F3D41903F07F07C6E7019A039284
:20F68000C8E7059ADDF804E0DDE902C198F80030022B14D0032BE6D152F8273023F07043BD
:20F6A000B3FA83F30F445B096345236823D00B4477452360EAD309F101090027C5E732F8FE
:20F6C0001730EDE74FF480720192D2E70C49013A096802EB41224902B2FBF1F2039913446F
:20F6E000B3FBF1F201FB12320AB10B449B1A9D42236096D8ABE7AB42ABD3A8E7348D01203C
:20F70000CC8D01208C750120F0B5114D83B00E462B78022B17D14FEA102CC4B241F63007B2
:20F720000023032201A9E8596044FFF7B5FA012807D12B78022B019B0CBF23F8146043F84B
:20F74000246003B0F0BDC0F3D41C00F07F04E5E78C7501202DE9F043002990F83C3083B028
:20F76000044614BF02210021042B7BD8DFE803F0030C3C476900FFF759FD012870D1626B6E
:20F78000002A75D184F83C00404E4FF6F777DFF804813F4D1BE0B94594BF4FF000094FF045
:20F7A000010901A9B9F1000F48D1FFF793FB0128494652D1206BFFF7A7FF01284DD1019A5B
:20F7C0002B68511E22638B4228BF0B462B603378206B032B1FFA80F9DDD1404594BF4FF057
:20F7E00000094FF00109DCE7426B04F130010020FFF7E0FD012833D1032384F83C30234B85
:20F8000041F2C470E16A41F2A8771A5803F5C255195041F2AC76511A2A68D85902FB01F287
:20F82000995900EB422503F5BD5001EB42220021DD519A51FFF7FAFC012811D1042384F85B
:20F840003C3094F82830042B02D1002384F82830A36B8BB120469847012003B0BDE8F083E4
:20F860000228FAD194F82830042B09D00220F4E7022384F83C30B8E7012003B0BDE8F08312
:20F880000023022084F82830E7E700BF8C750120D08D0120F7FFFF0F38B590F834300446FB
:20F8A000052B42D8DFE803F01E033B0F1868006B4FF0FF31FFF728FF012836D1E06AB0BB7D
:20F8C000032384F8343000212046FFF7AFFC01282BD1042384F8343094F82830082B2AD0BD
:20F8E000012038BD41F63803244D00F130010120EA580232FFF770FE01282AD00238C0B223
:20F90000012812D8052384F8343094F82830082B16D041F2E57301220220EA5438BDC06AA2
:20F92000216BFFF7F1FE0128CAD0002038BD022384F83430F4E70023012084F8283038BD91
:20F9400000230122022084F8283041F2E573EA54E4E705F5C252E368206B41F644011268FD
:20F96000685003EB4223E26AC4E9033002B96062012384F834309BE7004DC6E78C75012031
:20F9800043682DE9F04F164683B0C3F30808002A00F0DF80704B054689464FF0000AA3F1E7
:20F9A000180BC8F5007495F91A702846B44228BF3446791C2ED0F8F7ABFE41F218620BEB48
:20F9C00007139B58984205D0FFF7F8F8504603B0BDE8F08F604B03EB47202246494640449D
:20F9E000A2444DF0D9FA002221462846FFF732FB0028EBD02B7E1B0706D5584B2A691B68B5
:20FA00009A4201D3FFF7DAF8361BA1444FF00008C7D1DBE7F8F754FE002846D12846F8F7BA
:20FA200077FE6968C1F308031BBB4D4AAB680A4002F500729A422CBF062207222B7E03F0DA
:20FA40000C030C2B1BD0002301A9FFF725F90128BCD10198404BC31A48BF03F2FF13B3F527
:20FA6000B05F4FEA63224CD257B2AF760028B4D1ACE72B7E072203F00C030C2BE3D19BF8DB
:20FA800000C0384BBCF1030F1B680CBF4FF0800C4FF4807C03FB0CF34FEA432C0CF1FF3C2F
:20FAA0000CEA0101A3EB5123CEE72B7E1A072CD59BF800202B4B032A95F828201B680CBF53
:20FAC00080214FF48071062A03FB01F34FEA43233FF47CAF24490868834231D891F83D3091
:20FAE000002B7FF473AF002A7FF470AF06216B69284685F8382085F82810EB62FFF706FD51
:20FB00001AE0FFF75BF80198AFE795F82830002B7FF45CAF154B1A78002A7FF457AF082127
:20FB200085F834206A69284685F82810D3F85F30C5E90B23FFF7B0FE01283FF46FAF45E77E
:20FB400041F2E573012250460BF8032003B0BDE8F08F92463AE700BFA4750120508D012074
:20FB600000FEFFFFCC8D0120348D0120718D01202DE9F04790F8384082B00546032C00F223
:20FB80009980DFE804F00218600BFFF785FE01280FD0022809D1032385F8383000202B6CC5
:20FBA000022485F8280003B19847204602B0BDE8F08785F838002B78022B50D03E4941F650
:20FBC00048026B688A5803EA0208C8F34F282846DFF8E890F8F79CFD0646A8EB00080222AD
:20FBE00001A930460023FFF757F808EB060701284FF40072BFB24FF00001044606F10106A6
:20FC0000D3D101984DF03AFAEB694FF4007128460BB16B684BB3D9F80030013B9F4206D23D
:20FC2000FFF7A4F90028DAD1FEF7C8FFD7E7C3EBC35328465902FFF799F908B9FEF7BEFF5C
:20FC4000022385F8383000222B6C85F8282053B1012428469847204602B0BDE8F0876B689F
:20FC6000C3F34F28B3E701249FE7019B4FF020322E244FF0100C1A605A601C70C3F8072096
:20FC8000D5F824E01A625A62CEF30F4A83F8204083F82140C3F8272083F80BC0EA6BA3F852
:20FCA0001AE0C2F30F44A3F814A05A879C8683F82BC0B0E7002478E78C750120CC8D0120D4
:20FCC0002DE9F04F90F8303089B00446042B00F2A780DFE813F0A800B10005008900E70084
:20FCE000B54D41F61003EB5C002B40F09980B34F04F11C0901AEB84607F1380BBA46324681
:20FD000049464046FFF720FA012840F016810198002800F0F98003780BB1E52BEFD1A84AAB
:20FD2000821A48BF02F2FF12B2F5B05F4FEA622380F03B811B01A34A13449A7B042A0CD0FC
:20FD400041F2C86641F2CC610427AA590132AA515A609F736B5801336B5041F60202AB56CC
:20FD60005E1C09D003F5B173FF2105EB0313A954DA796FF30002DA7141F603016B565A1C7D
:20FD80000ED003F5B173FF2605EB0313DA796E54C2F34501013921EAE17161F34602DA71B0
:20FDA000202200214DF06AF92346019A05A853F8315F59681560516019899B7A118193727F
:20FDC000019B627EDA723FF013FABDF81430002B40F02E8144F28172019903200A82CB815E
:20FDE0000A83CB8284F83000237E980600F1A8802046FFF749F92369002B00F0AD80237E12
:20FE000003F0F70213F00403227640F0B380122A00F0B9800022E36A204684F82820984714
:20FE200009B0BDE8F08F6548FFF72EF94FF6FF720123228484F8303004F11C0801AE5F4F49
:20FE400004F13109324641463846FFF77DF901282FD00228E4D1584D41F60202AB56591C2D
:20FE600009D003F5B173FF2105EB0313A954DA796FF30002DA7141F603016B565F1C0ED013
:20FE800003F5B173FF2005EB0313DA796854C2F34501013921EAE17161F34602DA71042372
:20FEA00084F830300020E36A2070984709B0BDE8F08F019D0B2249462846002D00F08680C2
:20FEC0002B78002B00F0828095F80BA01AF0080FB8D14DF0B9F90028B4D1637E8AEA030389
:20FEE000DB0640F1C680344D41F60202AB565F1CC1D003F5B173FF2105EB0313A954DA794F
:20FF000060F30002DA71B6E73B78092250462E49022BC4D00B78002BC1D10A708BF800308B
:20FF20004A6B0B73C1E9053351F8143CC1E90132FFF71EFE01283FF4E2AE0228AFD06FE739
:20FF40000023112205A9E069FEF7A6FE01283FF44FAF09B0BDE8F08F237E19077FF55AAF46
:20FF6000154A41F2C873D15C00297FF459AF0721D1544FE70023E26AA168204684F82830AE
:20FF8000FFF768F84CE7E56A0421626A204684F83C306363A56384F828106362C4E9023321
:20FFA000C4E90B22FFF770F83AE7FEF707FE01986FF00F03BFE600BF8C750120748D01203C
:20FFC000A4750120A48B01209C8D0120474D41F60202AB565E1C09D003F5B173FF2105EBFE
:20FFE0000313A954DA796FF30002DA7141F603016B56581C0ED003F5B173FF2005EB03135D
:020000040801F1
:20000000DA796854C2F34501013921EAE17161F34602DA71237EDA067FF541AF3448FFF701
:2000200033F84FF6FF720223228484F8303058E6304B05A902A8B3F9B4263FF0F9F89DF8EC
:200040000C309DF80D00DB029DF80A509DF80B20BDF8081043EA401342EA45129DF80E00C3
:20006000A1F2BC7143EA500342EA41229BB292B2B2E6A98A6A8B204B42EA01421B6862623F
:200080005A02EB69B3FBF2F102FB1131A36009B113445B1A154D41F60202E36084F819A042
:2000A000AB565E1C09D003F5B173FF2105EB0313A954DA796FF30002DA7141F603016B56AF
:2000C000581C0ED003F5B173FF2005EB0313DA796854C2F34501013921EAE17161F3460250
:2000E000DA71032384F830307EE600BF8C750120748D0120704C0120CC8D01202DE9F041AE
:2001000090F8283084B00446013B082B41D8DFE803F048054D525865406A4300394B41F6EE
:20012000480241689F5803F5C253056B0F401B68EA194FEA4328B2EB432F16D258E0216926
:20014000207EFEF7F5FE012823D1256B6168A5EB080522694144039B3D446261C91B2361AC
:20016000A84537466160256342D82046F8F7A8FA03AA06460028E2D06168A3680020E26AA8
:20018000994284F8280038BF1946A1600AB12046904704B0BDE8F081FFF7EAFC04B0BDE892
:2001A000F081FFF78DFD04B0BDE8F081FFF776F804B0BDE8F0810021FFF7CCFA04B0BDE820
:2001C000F0810121FFF7C6FA0128E2D10023216C204684F82830FFF7D1F8DAE7FFF796F90B
:2001E00004B0BDE8F081FFF757FB04B0BDE8F08120460191F8F764FA01990028BDD1294421
:200200006160BAE78C7501202DE9F04782B0054618461C4602AF0E4690464AF03DFC08304A
:20022000013C20F00700ADEB000D0DF1080AD14614F8013F5BB94246314689F80030284620
:20024000CDF800A033F0E2FABD46BDE8F08718463EF07AFDC3B2A3F120023F2A88BF2023FA
:2002600009F8013BE4E700BF2DE9F0470D4690460021442204461E46089F4CF0FFFE012308
:200280004FF6FF722676628384F828302B782E2B42D004F1310A04F139092E46327820237D
:2002A00010462AB12E2A03D03EF04EFD0136C3B20AF8013BCA45F1D130782E2801D17078F6
:2002C000013604F1380904F13B0A202318B13EF03BFD0136C3B209F8013FD14507D0307883
:2002E00020230028F3D109F8013FD145F7D118F0100F84F81980E76214BF0323012323707B
:200300002B782E2B24D00023204684F83030FFF7D7FC2046BDE8F0876B78002BB9D1124B48
:2003200041F60C0041F2F47141F2F0721E589A58585841F601016662C4E9022041F2E872D8
:20034000595C61769B5CE76223702B782E2BDAD16B78002BD7D10323204684F83030FFF783
:20036000AFFC2046BDE8F0878C7501200121032008B549F07BF872B640F0FEF82DE9F04FDD
:20038000CF4C8DB04FF00008DFF84893CD4D009054F80B0C002800F0FE802DF093FC064671
:2003A000002800F0DC81D9F82830E026A4F10B0BC54F44F8073C002306FB08F604F8033CFE
:2003C00054F80B0C2DF07EFC002800F0E48054F80B0C2DF06FFC14F8023C82465A1E0B2AFD
:2003E0000DD8DFE812F01F003A004600530083009B00E20016013601410179019101242875
:200400000CD0009A3AB995F82E26824240F08281012204F8032C0D2BD2D186E0012304F8EC
:20042000023CCDE700234D28C4F8C53084F8CD3084F8CE3004D0582808D004F8023CBFE782
:20044000022284F8C43004F8022CB9E7032304F8023C022384F8C430B2E704233C2804F829
:20046000023C0BD0BAF13E0F0CD0002304F8023CA6E70A233C2804F8023CF3D1002304F8F7
:20048000013C9DE7012304F8013C99E7D4F8C500BB19421C0344C4F8C520022A83F8E7AFD6
:2004A00094F8CD008AEA000184F8CD1088D12378C02BDAD86278FF2A08D1052BD5D90123A6
:2004C00084F8C430072304F8023C79E7A4F8C1200022C4F8C930934284F8C320C4F8C520BF
:2004E00014BF0523062304F8023C69E7D4F8C500BB19421C0344C4F8C52083F8E7AF94F806
:20050000CD00D4F8C9308AEA00019A4284F8CD107FF456AF062304F8023C51E794F8CD3003
:200520008342A2D10D2304F8023C14F8017C002F40F0F780654B04AE0894ADF82A700397E3
:200540000FCB86E80F00D4F8C930324608A9D4F8D10023440993B4F8C130ADF8283094F890
:20056000C3308DF82C3001238DF82D3003AB28F0B7FB48B1049B314694F8C4205846059374
:20058000534B049325F08EFE0023039E04F8023C002E40F0DC8008F10108E034B8F1030FFC
:2005A0007FF4F6AE0DB0BDE8F08FD4F8C500BA195146431C0244C4F8C53082F8E7AF94F856
:2005C000CD2094F8CE008AEA0202019384F8CD20D5223EF077FE019B84F8CE00072B7FF43A
:2005E000EFAEB4F80530C02B3FF63FAFB4F80320C4F8C930A4F8C120A27884F8C3200022D3
:200600009342C4F8C52014BF0823092304F8023CD6E6D522014694F8CE003EF053FE94F8A1
:20062000CD3084F8CE008AEA0303D4F8C50084F8CD30BB19421C0344C4F8C52083F8E7AFC4
:20064000D4F8C9309A427FF4BBAE092304F8023CB6E694F8CD30434084F8CD3094F8CE300C
:2006600083427FF402AF55E7D4F8C500BA195146431C0244C4F8C53082F8E7AFD52294F871
:20068000CE0001933EF01EFE019B84F8CE00052B7FF496AEB4F80120B4F80330A4F8C120B8
:2006A0002278C4F8C93084F8C32000229342C4F8C52014BF0B230C2304F8023C80E600BF65
:2006C0005F4B0120704C0120783B01204CD8050850190220802A0120D522014694F8CE007F
:2006E0003EF0F0FDBB1984F8CE00D4F8C500421C0344C4F8C52083F8E7AFD4F8C9309A4238
:200700007FF45EAE0C2398E694F8CE3083427FF4ACAE07E723287FF47EAE022204F8032C6A
:2007200079E6012F4FF0000602D004F8026C32E7D4F8C93008A8089423440993B4F8C130DF
:20074000CDE90A66ADF8283025F074FAEDE754F80B0C26F007F854F80B0CB0471BE714F83F
:20076000033C002B3FF417AFD9F8282054F8071C521A632A7FF60FAF012B29D0022B7FF49D
:200780000AAF54F80B3C012285F8C906C5F8B836C5F8BC36C5F8C436402385F8B62685F854
:2007A000C8360C4A0C4B0D48C5F8C026C5F87C35C5F80C3734F0DEFF4FF4005028F0EEF896
:2007C000074834F0CDFF85F8106785F81167E2E6FFF7CCFD0DDD0308305301207E5D0608E8
:2007E000B45D060803460A2201481A80704700BFF00301200346202201481A80704700BF14
:20080000FC0301200346202201481A80704700BF1C0401200346202201481A80704700BFAF
:200820003C04012003460A2201481A80704700BF5C0401200023D0F89822184613737047C8
:200840000346222201481A80704700BF680401200346222201481A80704700BF8C0401208E
:200860000346222201481A80704700BFB004012003460A2201481A80704700BFD4040120F6
:200880000346432201481A80704700BFE00401200346432201481A80704700BF24050120FB
:2008A0000346432201481A80704700BF68050120D0F8943283B110B5D0F8904294F80002F4
:2008C000FF2807D09B68214694F801229847FF2384F80032002010BD0020704701F00F018D
:2008E000D0F8A822C1EBC10102EB810238B5D0F89032D0F89452D2F8144203F50371EA6885
:20090000D3F80402C3F80C429047002038BD00BF08B5D0F88C325B689847002008BD00BFC9
:2009200008B5D0F88C321BB11B68984700B908BD022008BD0022836BA3F85A20A3F85220AF
:20094000704700BF836B1A6810B45C6F986F9168090601D5212C1AD09168490601D522289E
:2009600006D0DA6F5DF8044B42F01002DA67704700202024A3F85A00116821F4907111601F
:20098000916821F00101916018669C67E9E700212024A3F85210116821F0C00111605C6728
:2009A000DAE700BF704700BF704700BFC369B3F5807F12D0826B002120201368A2F85A1049
:2009C000196821F480711960996821F001019960996821F04001996090677047C369B3F53C
:2009E000807F0CD0826B00211368A2F852109A6822F080029A601A6842F040021A607047E0
:200A000011F0010307D090F8413003F02803282B0CBF4223F2238A0709D590F8412002F001
:200A20002802282A0CBF43F0440343F0F4034A07016848BF43F0B8030A6822EA03030B602D
:200A4000704700BFC16838B5022903689A699C699A68DD680DD1C2F3C21282EA144212F0FA
:200A6000060206D1816C01318164816C022907D038BD0421FFF7C4FF002380F8403038BDD1
:200A800008218264D96180F8402038BD836B0022D3E90E0102650A6593F84120602A02D146
:200AA000202283F8412070470023202210B5134C4363C462036380F8412080F842304B0791
:200AC00012D50268436A526A1A70436A028D013343624AB1438D013A013B02859BB24385DF
:200AE000436C43F0040343640721FFF789FF102102680023D16180F8403010BD0000FFFF1D
:200B000038B5002580F8425090F84130292B04D090F841302A2B0BD038BD282221230121CA
:200B200080F841200363FFF76BFF80F8405038BD28222223022180F841200363FFF760FFD3
:200B400080F8405038BD00BF38B50025202280F8425090F8413080F84120212B0BBF11235F
:200B60001223012102210CBF456345630363FFF747FF80F8405038BD90F8BC33012B29D0A5
:200B8000012380F8BC330B060ED402681021124B116101E0013B02D01169C906FAD4002344
:200BA00080F8BC331846704701F00F010A4B890110B441F020010468216101E0013B02D0E6
:200BC00022699206FAD4002380F8BC3318465DF8044B704702207047400D030011F0800F28
:200BE0004FF01C0301F00F0170B432D103FB0103C1EBC102002400EB820203F5FE7382F888
:200C0000FD41197090F8BC23012A31D00121026880F8BC135C781D7802F500638C422AD01C
:200C200005F00F04DE6B02F53062A1401C4C02EB451226EA0146DE63DD6925EA0141D961E4
:200C400013681C401460002380F8BC33184670BC704703FB0103C1EBC102012400EB820279
:200C60003C3382F83D40197090F8BC23012ACDD1022070BC704705F00F01DE6B02F5106299
:200C80008C40084902EB451226EA0406DE63DD6925EA0404DC61136819401160D3E700BF40
:200CA0000078F3EF007833EC836B40221A645A6C42F004025A647047704700BF836B1A6C18
:200CC00012F0500F1A6C20D142F4007219681A648A6812F0405F1AD19A69C2B9CA6A12F45F
:200CE000700F02D08A68500511D44A6822F020024A601A6C22F480721A641A6CD10406D4A6
:200D00001A6C42F001021A647047D20600D570479B6BDB6C184700BF836B0121002283F867
:200D20003D101A77704700BF0122836B83F83D20704700207047114A1068A8B153689BB1B5
:200D400088420FD88B4234BF00230123DBB243B1D368916099421FBF094B1420D16083F841
:200D6000BB0170470023F1E7A1F59C53083BB3F57A7F2CBF00230123E9E700BFE08D01204D
:200D8000F0030120054B5A7C19748A421FBF044A1420597482F8BB01704700BFE08D012059
:200DA000F0030120704728B1034B987C012894BF00200120704700BFE08D012008B5FFF7B9
:200DC000F2FF50B1054AD37C127C5B0003F00203002A18BF43F001030B6008BDE08D0120AC
:200DE00008B5FFF7E0FF10B1014B5B690B8008BDE08D012070B5FFF7D6FF50B10A4A158BCD
:200E000035B1D6690023B3421C4603DB002000E00D7070BD02EB44040133248CDBB2AC4217
:200E2000F1D10B70F5E700BFE08D012008B5FFF7BAFF10B100230B70137008BD042070475E
:200E400028B1034B93F9BC01003818BF01207047F003012008B5FFF7F3FF50B1054B93F9A5
:200E6000BC21012AC9BF93F8BF310020C3F340030B6008BDF003012008B5FFF7E1FF18B1AE
:200E8000024B93F8BE310B7008BD00BFF003012070B5FFF7D5FF38B10E4C94F8BF31DB07E8
:200EA00003D500230B70137070BD0B4D94F9BD3195F8306093FBF6F301330B7094F9BD416B
:200EC00095F8301094FBF1F301FB134301331370EAE700BFF0030120E08D012003207047BD
:200EE0000A4A70B592F8343006255E1CB6FBF5F405FB146492F83550AC421EBF02EBC30347
:200F000082F83440C3E90E0170BD00BFE08D0120002230B504461046914200DC30BDA35C6C
:200F20000825584010F0800F4FEA400318BF83F0D503013DD8B2F5D10132EDE710B5D9B1DB
:200F40000E4B986E814217DCB2B11B6B9A4213DC013A01390A4C03FB012104F5E37084F815
:200F6000CA110521FFF7D4FF062184F8CB0104F5E370BDE81040B3E710BD00BFE08D012043
:200F8000F00301200023038083708380C3800381704700BF074A084992F86C3009780133E7
:200FA000DBB2994282F86C3004BF002382F86C30704700BFE08D012070070020F8B5774CAC
:200FC000236F83B1764B1B6893F82E305BB1754B94F87420A3FB0013012A4FEA93132FD078
:200FE000022A08D002B1F8BD6F4B9842FBD9012384F87430F8BDA26F64329A423DD894F800
:201000006C3004EB031393F88C20FF2A06D001326649012083F88C2081F8CC01FFF7BAFFDA
:20102000634B01221B7884F87420092BDBD1B4F80E31604A01339BB2A4F80E315380F8BDE3
:2010400094F86C1004F180055B48002701EB8106A367E567022500EB461355480A2684F8C7
:201060008A7000789A70092884F88B6084F87450B9D101314F4B1980F8BD94F88A2094F8B6
:201080008B309A42AFD104F17F0004F18805002310F8011F08224B4013F0800F4FEA430134
:2010A0000B4616BF81F00703CBB2DBB2013AF3D18542EDD194F88910994238D1B4F8836069
:2010C000012794F86C5076BA94F887C004EB0511B4F88500B6B294F8883040BA81F88C209C
:2010E00043EA0C23C1F8906094F881C080B294F882601BB2C1F89400032D46EA0C2294F949
:201100008000A1F89830A1F88E20284A81F88D0082F8CC7108D8264A12780C2A29D00D2A38
:2011200002D1244B23F81500FFF734FF5FE794F86C3004EB031393F88C20FF2A06D0013238
:201140001A49012083F88C2081F8CC01FFF722FF174B01221B7884F87420092B7FF443AFC6
:20116000B4F80C31134A01339BB2A4F80C319380F8BD03EB83031149114A03EB830391F8E1
:2011800022100C48F9409B0093FBF1F382FB0312DB17C3EBA20320F81530C5E7E08D012015
:2011A00008150020D34D62103F4B4C00F00301201049012014490120A0260020D44901205A
:2011C000676666660A4B93F88A1093F88B2091420DD0C0B210B493F88A20DC6F511CD2B26F
:2011E000C9B283F88A10A0545DF8044B70477047E08D01200F4B104AD3F81031B2F9000060
:201200005B0707D400EB8000400080B200F5C87080B27047094B0A4AD3F8C430323382FB55
:201220000312D817C0EBA20080B200F5C87080B2704700BFE08D0120844B0020243A01205A
:201240006766666680F08003042B70B520D941281ED0FD2806D0F0281DD0EF281FD0022432
:20126000204670BD0B2004260F4D2E4400240135FFF7E8FF2044AE42C4B2F1D015F8010BDD
:20128000FFF7E0FF2044AE42C4B2F7D1204670BD0424204670BD03200526044DE5E70C2002
:2012A0000626034DE1E700BF085E0608005E0608F85D060870B5D0F8A052044695F81832E8
:2012C00013B9D5F814323BB981212046FCF712FE6B7A022B07D070BD6B7A002BF4D1012123
:2012E000FCF708FEF0E705F5037220461F230121BDE87040FCF772BD70B5037C044601255A
:201300007BBB4FF4007302222946FCF759FE4FF40073C4F85851174E812102222046FCF765
:201320004FFE321DE5620025D4F8A432C4F8A0222846B581A6F860521B6898470121D4F841
:20134000A802FFF719FC8121D4F8A802FFF714FC06F5047220461F230121FCF73FFD2846E2
:2013600070BD402302222946FCF72AFE4023C4F85851D0E7844B002038B504460025012143
:20138000D0F8A802FFF72AFC8121D4F8A802C4F85851FFF723FCD4F8A002E5624BF03EFE01
:2013A0002846C4F8A05238BD38B504468321D0F8A8020025FFF712FCD4F89802656518B1AD
:2013C0004BF02CFEC4F89852002038BD38B5044600258121D0F8A802FFF700FC0121D4F89D
:2013E000A802E562FFF7FAFBD4F8A8028221C4F85851FFF7F3FBD4F8903225644BB1D4F8D0
:2014000094325B689847D4F890024BF007FEC4F89052002038BD00BF10B50823032283219B
:201420000446FCF7CDFD0123102063654BF0EEFDC4F8980218B103460020187310BD022061
:2014400010BD00BF2DE9F041037C04460125BBBB4FF4007302228121FCF7B2FD29464FF484
:20146000007302222046E562FCF7AAFDC4F858514FF001080823032282212046FCF7A0FDF8
:201480004FF40770C4F840804BF0C0FD0546C4F8900258B3D4F8943200271B689847267CBD
:2014A000C5F814724146D5F804222046C5F81872AEB140233E46FCF791FC3046BDE8F08170
:2014C000402302228121FCF77BFD2946402302222046E562FCF774FDC4F85851C8E74FF41A
:2014E0000073FCF77BFC3046BDE8F0814646E4E707B50DF1060212F06BFA68B1084BBDF8E2
:201500000620B3F814111A8391421FBF05491420A3F8142181F8BB0103B05DF804FB00BF3A
:20152000E08D0120F003012013B50446FFF788FC00B300230DF106022046ADF8063012F05E
:2015400047FAB8B10C4C9DF8062094F9BC1184F8D121032909484FF0050104BF62F07F02AE
:2015600084F8D121FFF7D4FC062184F8D2010348FFF7B6FC02B010BDF0030120BD05012058
:201580002DE9FF47002304461E200193ADF80C301D4B93F8009093F801A09D78B3F80480DC
:2015A000DF881E7A20F0D8FA28B1002F1EBFB84601254FF00009154A92F81631D9070AD40B
:2015C00092F81B213AB9012E1BD0022E03D113F0020F08BF012501AB8DF80C608DF804907D
:2015E0008DF805A08DF80650ADF80880ADF80A7003CB1B88206020466160238104B0BDE885
:20160000F0873546E7E700BFD8520120E08D0120144B30B4D3F8404114B383F84611090A37
:2016200000220F2583F8450103F5A27083F847110121C3F84821C3F84C21C3F8502183F8A1
:20164000445110F8015F01312A440E29D2B2F8D183F8522120461022034930BC2CF036BB9E
:2016600030BC7047E08D0120248F0120034B002183F85411C3F85811CAE700BFE08D0120F4
:2016800013B504462620019120F066FA019920B9204602B0BDE81040BAE702B010BD2DE93A
:2016A000F743B74C0D46D4F840314BB14FF0020800264FF00109D4F840012CF003FB58B971
:2016C0000027A37C042B00F25781DFE813F08F00E400F7003D014601D4F840012CF0EAFA05
:2016E000D4F858315A1C234483F85C0194F85431C4F85821012B0AD0022B11D0002B70D11A
:201700000F280CBF84F85491C4F85831D3E7A0F17203012B01D9762863D184F85481CAE787
:20172000102AC8D197490023012211F8010F013203440E2ADBB2F8D194F86A2184F8546147
:201740009A42C4F85861B6D194F86B31002BB2D194F85D71732F37D0762F0DD0722FAAD13A
:2017600094F85F2194F85E3153EA0223A3D02360B4F860316360A4E794F85F2194F85E3138
:2017800053EA022397D094F8611194F8602194F8650142EA012294F862116361E17494F890
:2017A0006311A4F86C2184F86E1194F8641141EA0021A4F87011A16801B9A360238B002B88
:2017C0007FF47FAF22837CE794F8632194F8623143EA02231AB2002B3FF46DAFA4F872216A
:2017E0006FE784F85461C4F8586164E7722F44D101230022A374644B1B78402B2FD1634E31
:20180000A37C94F86EC1208B33804FEA0C330502B4F86CE103F44053217C05F4706577802C
:201820006769704514BF042000202B434FEA0E1543EA8133614514BF02210021EDB22B4397
:20184000A5681BB2BD4214BF0825002513432B4318434F4B014393F8BB31B180F380A36E61
:201860001BB1E369002B40F09D801F2249494A4803B0BDE8F0434BF0F9BCD4F87431474AF6
:20188000EB1A934201DC0022B5E77220FFF7EEFEC4F87451F7E7762F03D102230022A37429
:2018A000A9E7D4F874313D4AEB1A9342EBDD7620FFF7DCFE0022C4F874519CE7344ED4F824
:2018C000743196F8BB21EB1A82B3344A934230DDE27CD2071BD4A168626991420ED089B279
:2018E0004620FFF7CDFE96F8BB310122C4F87451013B86F8BB310423A3747CE7218BB4F804
:201900006C218A4203D05020FFF7BAFEEBE7217C94F86E218A4206D0B1FA81F14920490979
:20192000FFF7AEFEDFE7142286F8BB211C4A9342BDDC762FA7D17320FFF798FE0323002257
:20194000C4F87451A37456E7732F9CD0D4F87411124B691A9942A0DC95E7D4F874310F4AD6
:20196000EB1A93428FDD7620FFF780FE02230022C4F87451A3743EE700231A46A3743AE758
:20198000E08D01203C8F01201049012014490120F0030120B95D0608C30501203F0D030065
:2019A0003F420F00334D2A23D4F878610DF1020285F8D33120230DF10101304685F8D43167
:2019C00012F09DF830B19DF801109DF8027051EA070339D1552385F8D531462385F8D631AB
:2019E000202301A9304685F8D73112F082F80346214813B1BDF804209ABB20493EF0AEF9A1
:201A0000B4F870711E4D87B30DF10301304612F073F850B30DF106029DF80310304611F087
:201A2000D7FF10B3BDF806203B4616492846BA420CBF20222A223EF091F9B4F87231A4F8EC
:201A40007C3103B0BDE8F083304612F03DF8394685F8D501304612F023F8037885F8D631FD
:201A6000BEE709493EF07AF9CAE7084928463EF075F9E2E7F0030120C8050120DB5D0608B1
:201A8000CC050120D35D06083A9D0608DA5D060838B50B680C460E4D5A1C20460A60052272
:201AA0001A700B6895F8BC21591C21601A70236895F8BF21591C21601A70B5F8C2113DF01A
:201AC000C7F8236895F8C421591C21601A7038BDF00301202DE9F0472DED028BFFF7B0F92E
:201AE000C8B31E4B93F9BC01012834DD93F8F24115461B4F8E1E02EB44089FED1A8A4FF0A8
:201B00003209454504D12046BDEC028BBDE8F08737F802ABB2EE040A07EE90AA26F802AFEB
:201B2000F8EEE70A60EE880A4AF06EF8BCEEC00ABAF10E0F10EE103A9BB209D91933B3FBA1
:201B4000F9F39BB203EB830303EB83035B009BB225F8023BD5E70024D5E700BFF0030120F3
:201B60005E8F0120CDCCCC3D38B50D46FFF768F9044638B10C4890F8BF31DB0704D5B0F8BC
:201B8000C0012880204638BD084A00F5FA7010F9373C92F8302093FBF2F102FB1132013197
:201BA000013211F029FFECE7F0030120E08D012038B5134C94F8353094F834209A4219D072
:201BC00004EBC3030F49D3E90E200023984212DC93780D4A5B08C4F890011370FBF7C4FFD9
:201BE00094F8353006210133B3FBF1F201FB123384F8353038BDD55C013301F8015BE5E76B
:201C0000E08D0120E252012010530120AA4B1B782DE9F04F81468BB0002B40F0B680A74EF8
:201C2000D6F87851002D00F0B080A54AD2F8F84104F0F021B1F1E02F6CD1C2F8F831D6F82A
:201C40009421944266D004930DF11008C8F804300DF11C0EA8F808309A4BC6F894419A8888
:201C60001F78ADF8142093F801C01A7A93F802A08DF810708DF811C08DF812A08DF8182098
:201C800098E80700AEE803008F49AEF80020C4F34252895CC4F303428F4202F101021F462E
:201CA00001D1944508D028468DF81C108DF81D2011F0A2FEADF82000284604F0070B12F0E4
:201CC000EEF8032833D0042835D000239A4501A9284618BF8DF81E3011F008FF48B1019B5E
:201CE000C4F3001103F001038B4202D0284611F0ADFF0A2207A940464BF098F950B19DF8A7
:201D00001E30BDF81C20BB70BDF820303A80BB803EF0F8FA96F898A104AFDFF8A8B196F807
:201D20009831032B7BD8DFE803F00A3376A3674B13F80B30CAE7664B13F80B30C6E739467D
:201D4000284611F0D9FE044658B107A8FFF718FC9DF81E109DF810308B4260D0284612F02C
:201D600001F896F89831013303F0030386F898310CB99A45D3D196F81631DB0700D524B1F6
:201D80002B68494628461B6898470BB0BDE8F08F01A8FFF7F5FB96F816819DF8044008F0ED
:201DA0000108ECB1B8F1000F39D13A460DF10301284611F0A4FE044688B307A8FFF7E0FB23
:201DC0009DF81C109DF803309DF81D208B4203D19DF81030934222D0284611F0CDFFC0E789
:201DE000B8F1000FBDD13946284611F082FE0446A8B107A8FFF7C4FBBDF82010BDF810304E
:201E00008B420CD086F89981284686F89A812B689B699847A5E796F81631D80701D50024CA
:201E20009FE707A9284611F061FE04460028F6D01E201FF091FE96F89B3180468342EED0E7
:201E400086F89B0160B1BBF80630002BE7D1079BD907E4D401212846444611F0F7FE80E7DA
:201E6000079BDA07DBD50146284611F0EFFE78E73846FFF785FB07AB97E8070003C31A80A1
:201E80009DF810309BB10DF11D0207A9284611F036FE0DF11E01284611F02EFE0A2207A91D
:201EA00038464BF0C3F8041E18BF012459E708A9284611F01EFEECE726530120E08D012019
:201EC000F0030120D8520120285E06081C5E0608105E0608FD292DE9F041044684B000F030
:201EE000D880F02900F0BC80EF2900F02B814AB10346861803AD002003F8010B9E4205F8FB
:201F0000010BF9D19B4B0B2003F1090501E013F8010F814200F0C280AB42F8D14B1E832B1A
:201F200000F29280DFE813F01E01340184003E01AA01B001450150015C01900090006201E9
:201F4000620162017801780178015C019000900082018A0190009000900090009000900065
:201F6000900090009000900090009000900090009000900090009000900090009000900061
:201F8000900090009000900090009000900090009000900090009000900090009000900041
:201FA00090009000900090009F019000900090009000900090009000900090009000900011
:201FC000900090009000900090009000900090009000900090009000900090009000900001
:201FE0009000900090009000900090009000900090009000900090009000900090009000E1
:020000040801F1
:202000009000900090009000900090009000900090009000900090009000900090009000C0
:2020200090009000900090009000900019011901514B93F8AB11002900F05D81019223F08C
:2020400035FB019AADF80C003AB103AB224413F8011B04F8011BA242F9D104B0BDE8F0814E
:2020600003214FF00508454FB8440025013701E017F8011B0846FFF7E5F806466019324699
:20208000FFF728FF7019B845C5B2F1D104B0BDE8F0810B214FF00408394FE5E7364BD3F883
:2020A000100180060CD4002AD7D003AB224413F8011B04F8011B9442F9D104B0BDE8F0811B
:2020C00093F89C01870742D52E4D287D052834BF02260326142917D97C39C8B20628E2D85E
:2020E0000629E0D801A050F821F000BFCF220108CF220108B9220108A7200108DF2201088E
:20210000D9220108E52201080929CCD90A390A29C9D801A757F821F09F220108EB220108D5
:20212000A7200108A7200108A7200108A7200108A7200108A7200108A7200108B122010813
:20214000CF2201080C214FF006080F4F8CE70D4B0B29187DA7D10126C8E00C4BD3F8C030C0
:20216000039371E70192FFF745F8019AADF80C006AE700BFEC5D0608E08D0120005E0608FE
:20218000085E0608F0510120F85D0608243A0120684BD3ED767AFDEEE77A17EE903AADF864
:2021A0000C3051E7019223F081FA019AADF80C004AE7604D95F81631DE0700F1A580B5F8E4
:2021C000E831ADF80C303FE75B4B5C49B3F9043081FB0301DB17C3EBA103ADF80C3033E7F5
:2021E000544BB3F80432ADF80C302DE70C39544B9FED547AC9B2D3ED9C7A03EB810367EE14
:20220000877A93EDAE7A67EE877AFDEEE77A17EE903AADF80C3017E70F39474B33F811307F
:2022200003EB83035B00ADF80C300DE7414B93F8163103F00103ADF80C3005E7424B1988AA
:20224000CD0556BFCB43032303F0010311F0440F18BF042311F0020F18BF072311F4806F13
:2022600018BF0923ADE70192FEF7C4FF374B019AD3F8C83043EAC0400390E5E62D4BD3F8CE
:20228000F831ADF80C30DFE62A4BB3F8E811002934D0019223F022FA019A80B2D2E62B8A2D
:2022A00003EB830303EB83039B00ADF80C30FAE6EB89ADF80C30F6E6EB89254903EBC30313
:2022C0009B00A1FB03135B09ADF80C30EBE6B3F89E31ADF80C30E6E66B680393E3E62B68AF
:2022E0000393E0E6AB680393DDE6F6B28DF80C608DF80D00D7E6B3F8C401A3E6D3F8000268
:2023000080F3100080B29DE6019221F05BF8D5ED767A019AFCEEE77A17EE903A9BB20028B2
:202320007FF44FAF0B49096811F0100F18BF002347E700BFE08D0120A05201206766666626
:20234000844B002000007A44C4520120243A01201F85EB51D8510120014B1B681B6A18473D
:20236000F44A0120024B186808B1836918477047F44A0120024B186808B1436918477047CF
:20238000F44A012010B5074C606D40B131F0EAF894F8513013B180F00100C0B210BD012063
:2023A00010BD00BFEC1E01200368042201F01F01186A02FA01F120EA010010B418621A6A87
:2023C0000A4C114319625A6C42F400425A649A681440062C06D0B4F5803F03D01A6842F08F
:2023E00001021A6000205DF8044B704707000100B1F5805FF0B400F0D4802AD8102900F045
:20240000F580B1F5807F4ED1046A166924F4807457689A4B0462016A446821F40071C569B5
:2024200041EA0621964E2B40156821F48071B04245EA030541EA072173D0924B984270D0C2
:20244000D26800234460C561C26301621846F0BC7047B1F5803F00F08180B1F5801F48D158
:20246000046A156924F480145668874B0462016A446D21F400112340146841EA0551804D5F
:2024800043EA042421F48011A84241EA06515DD07C4B98425AD0D26800234465C26501624D
:2024A0001846F0BC7047012923D1046A166924F001045768714B0462016A446821F002012B
:2024C000856931436E4E2B40156821F00101B04245EA030541EA07010FD06A4B98420CD03D
:2024E000D268002344608561426301621846F0BC70470123F0BC18467047D2E9056321F013
:20250000080124F4807441EA86011C439668D36921F0040124F4007441EA860144EA430492
:20252000DEE7D2E9056321F4006124F4805441EA8621966844EA0314D36921F4806124F4F2
:20254000005441EA862144EA431479E74368956923F4802343EA852343609CE7046A156926
:2025600024F480345668494B0462016A446D21F400312340146841EA0541414D1C4321F423
:202580008031A84241EA064155D03E4B984252D0D26800234465846D826501621846F0BC39
:2025A0007047046A166924F480545768384B0462016A456821F40051C46941EA0631304E58
:2025C0002340146821F48051B04243EA042441EA073138D02B4B984235D0D268002345602D
:2025E000C461026401621846F0BC7047046A166924F010045768264B0462016A446821F059
:202600002001856941EA06111D4E2B40156821F01001B04243EA052541EA071119D0194B1B
:20262000984216D0D268002344608561826301621846F0BC70474368956923F4803343EA4A
:2026400005234360A4E725F48045936945EA8315C3E7D2E9056321F0800124F4806441EAFD
:202660008611966844EA8304D36921F0400124F4006441EA861144EAC304D3E78CFFFEFF0D
:202680000000014000040140FF8FFFFE8FFFFEFFFF8CFFFE70B4344CB0F1804F0368A0EB0C
:2026A0000404B4FA84F44FEA541406D02CB92F4D2F4A904218BFA8421DD12E4A23F070031C
:2026C0004D68821A2B43B2FA82F2520923F44073D1E902652B430D880360C66285623CB96B
:2026E00032B9436943F0010370BC4361002070470B7C0363F5E702F58062904220D002F50A
:20270000784290421CD01C4A1C4DA84218BF90420CBF0122002224D0194EA5F59635A84225
:2027200018BFB042D2D0174A90421AD002F58062904216D08C680A880360C4628262D0E7D6
:202740000C4A23F07003104D821A4E68A842B2FA82F243EA06034FEA5212B7D0002AB5D1DA
:20276000D1E70022B2E700BF0000014000040040000800400004014000400140004401400F
:2027800000480140001C0040000C00402DE9F04F002383B0DFF810820D68DFF810E203E0D3
:2027A0000133102B00F0B88001229A4032EA050405EA020CF4D14C6824F01007022F40F05E
:2027C000AE80DF0803F0070A4FF00F0B0E6900EB87074FEA8A0AD7F820900BFA0AFB06FA41
:2027E0000AF64FEA430A29EA0B094FF0030B46EA09090BFA0AF604EA0B0BC7F820906FEACC
:20280000060907680BFA0AFB27EA06064BEA060606608768C4F3001607EA090BCF689E4096
:2028200007FA0AF747EA0B078760476827EA020216434660C668E7008A6806EA090902FAA4
:202840000AF242EA0902C260AAD5D8F8447023F0030903F003020F2647F4804709F180490F
:202860009200C8F8447009F59C39D8F8447006FA02FA07F480470197444F019EB842D9F8A8
:20288000086026EA0A061AD007F58067B8425ED03F4FB84260D03F4FB84262D03E4FB842C2
:2028A00064D03E4FB84266D03D4FB84268D03D4FB8420CBF0727082707FA02F21643C9F8AC
:2028C00008606FEA0C07DEF80020E60303F1010354BF3A404CEA0202CEF80020A203DEF825
:2028E000046054BF3E404CEA0606E202CEF80460DEF8086054BF3E404CEA0606A402CEF816
:202900000860DEF80C2054BF3A404CEA0202102BCEF80C207FF448AF03B0BDE8F08F4FEADF
:20292000430A4FF00309D0F800B0013F04EA090609FA0AF9012F2BEA090B06FA0AF66FEA92
:20294000090946EA0B0606603FF674AF61E7012707FA02F21643B2E7022707FA02F2164398
:20296000ADE7032707FA02F21643A8E7042707FA02F21643A3E7052707FA02F216439EE7BA
:20298000062707FA02F2164399E700BF0000024000080240000C02400010024000140240FB
:2029A00000180240001C024000380240003C014030B40023154C0168C36725680B681B074B
:2029C00009D4002220231446436780F870208367204630BC7047CB6913F40013F1D122681C
:2029E000521BB2F1007FF6D30A682025032422F4D0720A608A6822F001028A60456780F8CA
:202A000070308567204630BC704700BFF8330120436ADA0710B406D50168846A4A6822F4CA
:202A2000003222434A609C0706D50168C46A4A6822F4803222434A60590706D50168046BA4
:202A40004A6822F4802222434A601A0706D50168446B4A6822F4004222434A60DC0606D513
:202A60000168846B8A6822F4805222438A60990606D50168C46B8A6822F4005222438A601A
:202A80005A060AD50168046C4A68B4F5801F22F4801242EA04024A600BD01B0606D502685F
:202AA000816C536823F400230B4353605DF8044B70474A68446C22F4C00222434A60ECE7BC
:202AC000754B002108222DE9F0411D6882B080460191D0E9166334689A40224204D001684C
:202AE0000F68780700F18A8001229A40224204D0D8F800104969090678D404229A4022425F
:202B000004D0D8F8001009688F0767D410229A40224204D0D8F800100F68380749D4202286
:202B20009A40224217D0D8F800100C68E00612D5B26098F83520052A73D00B6813F4802FBD
:202B40000B6800F09080190340F19B80D8F83C300BB140469847D8F854303BB3D8F85430A7
:202B6000DA071BD5D8F8002005214C4B88F83510A3FB0535136823F00103AD0A136002E09C
:202B80001368DB0704D5019B0133AB420193F7D90022012388F8342088F83530D8F84C3093
:202BA00023B1404602B0BDE8F041184702B0BDE8F081B2600A6812F4802F0A682AD1D7058A
:202BC00003D40A6822F008020A60D8F84020002AA5D040469047D8F85C30A0E7B260D8F835
:202BE000542042F00402C8F854208FE7B260D8F8542042F00202C8F854207EE70F6827F0CC
:202C000004070F60B260D8F8542042F00102C8F8542069E71203D8D5D8F84820002AD8D15E
:202C20007DE70A68D8F8404022F016020A604A6922F080024A6154B30A6822F008020A60E9
:202C40003F220024012102FA03F3D8F85020B36088F8344088F83510002AA7D0404602B0F6
:202C6000BDE8F041104713F480737FF46FAF0A68012422F010020A6088F8343088F835409E
:202C800064E7D8F84430002B7FF463AF63E7D8F84820002AD0D1D3E7F42B0120B5814E1B0F
:202CA00090F835200346022A03D0802201205A65704702680521002083F83510136823F0B8
:202CC00001031360704700BF70B5324A002590F84130044680F84250283BC2624585426CF5
:202CE000022B41EA020141642BD80321FDF788FE2822294B80F84120436305632268136889
:202D000013F4804312D01368A06B23F480431360B0B1224A0023026584F84030FFF7C0FF3C
:202D200070B1A06BBDE87040036D1847116811F4004114D194F84130602B24D084F8401057
:202D400070BD0721FDF75CFE90F84130602B02D0202380F84130002323636363CEE71168B1
:202D6000E06B21F4004111600028E9D00B4A026584F84030FFF794FF0028E1D0E06BBDE866
:202D80007040036D1847202384F8401084F8413070BD00BF0000FFFF8D2E01088D0A01086A
:202DA0000368202270B51E680D46DA6107210446FDF726FE03683348596841F400415960CD
:202DC0005A6802405A609A69910701D500229A629A69D20703D49A6942F001029A6170044C
:202DE0002BD5A26B1AB11268526892B262856A0709D55A6A25F00405636A1A70636A228D98
:202E0000013363624ABB638D9BB21BB1636C43F0040363640023236384F84230666C6363AC
:202E200016BBE36A184DAB420DD194F84130202384F8406084F8413070BD3104D7D5E26BA0
:202E4000002AD0D1D3E72046FDF75AFE2023E56284F8406084F8413070BD638D013A013B14
:202E600022859BB26385CEE7616C2046FFF72CFF94F84130282BDFD129462046BDE8704043
:202E8000FDF712BE00E800FE0000FFFFF8B590F84030C66A012B00F0848017460123CA0644
:202EA00004460D4680F8403020D5FB061ED5438D9BB2002B62D190F84130B6F1007FDBB27D
:202EC00002D1282B00F0848094F841301021292B2368D96102D116F5803F68D1AA0601D535
:202EE000BB0659D4002084F84000F8BD680710D42A072ED53B072CD594F8413003F028036E
:202F0000282B61D0216808200023C86184F84030E4E77907ECD5638D9BB27BB1216825F031
:202F20000405636A496A1970638D606A218D013B01309BB20139606263852185638D9BB296
:202F4000002BCBD116F5803FC8D02046FDF7D8FDC4E7A807C2D5B907C0D5638D9BB213B3D0
:202F6000606A236810F8016B218D9E62638D01396062013B21859BB26385AFE703681021A5
:202F8000D961436C43F00403436436F08073A5D1416CFFF799FEA1E729462046FFF700FF4C
:202FA000A0E70220F8BD36F0807397D1CDE799698A0701D5002199629969CE07C5D4996987
:202FC00041F001019961C0E72046FDF73BFD85E7FDF76AFD82E700BF38B520220368204D95
:202FE0000024DA615A682A401E4D5A6004634463CC06C56205D51022DA61426C42F00402ED
:2030000042649A69910701D500229A629A69D20703D49A6942F001029A610321FDF7F0FC91
:20302000436C90F84120602A0CD01A1E18BF012243B990F84130212B08D090F84130222B01
:2030400004D038BD416CBDE838403DE6202380F8402080F8413090F8423080F8422038BDED
:2030600000E800FE0000FFFF38B590F840300446C06A012B71D0012384F84030CB0615D5DB
:20308000D50613D5D30BC2F3803543EA9232D20729D5E26B5AB3DB0729D513685B6833BBF7
:2030A000A36B53B34DB31B685B6826E00B0707D4880601D5930612D4002084F8400038BD0F
:2030C0001507F5D594F8413003F02803282B46D0236808220020DA6184F84000EFE720467E
:2030E000FFF75EFEE8E723681022DA61E4E7A36B23B31DB31B685B6803BB94F84130282BE4
:2031000002D1B0F1007F2ED094F841301022292B2368DA61D0D110F5803FCDD09A699107D8
:2031200001D500229A629A69D20703D49A6942F001029A612046FDF7E3FCBDE7236810221B
:20314000DA61636C43F00403636430F08073B3D1616C2046FFF7B8FDAEE7022038BD2046DD
:20316000FDF770FCA8E72046FDF79EFCA4E700BFF8B590F84030012B7BD00123CD060446C5
:2031800080F8403023D5D00621D510222368616B4548DA61626C814242F00402626466D06D
:2031A000424A914263D0F4211A680A431A609A69910701D500229A629A69D20703D49A69DA
:2031C00042F001029A61002084F84000F8BD0B0631D5570643D523681A6822F040021A60C7
:2031E000628D92B2002A46D05868618DC0F309008AB2FF2A4BD8628DE56A91B215F5803F20
:203200002185CDB24BD0E76A2D045A68284E324002433A432A435A60628D521A92B26285D3
:2032200094F84120222A1A680CBF42F4004242F480421A60C7E74D0611D550060FD5638D0D
:203240009BB2FBB923685A689101BCD4E26A12F5803F13D15A6842F480425A60B3E78B0669
:20326000B1D59206AFD52046FFF7B6FEABE760219AE70220F8BD5B689E0103D42046FDF79E
:2032800063FCA0E740212046FFF71EFD9BE7FF224FF47F054FF0807711462285B5E74FF0F7
:2032A00000772D04B1E700BF6930010871310108009C00FC90F84030012B00F09C800123D6
:2032C0002DE9F041044680F84030C8060D4690461BD512F0100F18D023681021D961616CC2
:2032E00041F0040161649969890701D5002199629969CA0764D5AB0602D518F0200F71D142
:20330000002084F84000BDE8F0816B0712D4AF0724D518F0020F21D0606A236810F8016BE1
:20332000218D9E62638D01396062013B21859BB26385E0E718F0040FE9D0216825F004059A
:20334000636A496A1970638D606A218D013B01309BB20139606263852185CCE72E0615D4E8
:203360006906C8D518F0400FC5D0638D9BB2002B33D1236859688A01BDD4E16A11F5803F71
:2033800027D1596841F480415960B4E718F0400FB1D0638D9BB2C3B1238DB3B92068416854
:2033A000638DC1F309019BB2FF2B26D94368FF27204E27853340204E19430E4346609AE749
:2033C000996941F00101996195E723685B68980103D42046FDF7B8FB8DE740212046FFF746
:2033E00073FC88E720462946FFF7F6FD002084F84000BDE8F08102207047638DE66A9BB2D9
:2034000016F5803F23850AD0E76ADBB24668094A16403E4346EA0343194341606BE7466837
:20342000DBB2044F3E40314341EA034343F00073436060E7009C00FC0000FF01F0B4044633
:2034400090F834000128A66D38D0012594F83500A84284F8345005D00023022084F83430A1
:20346000F0BC704725680227002084F83570A76860652868402F20F4802028606B601AD02E
:20348000A960EA60E16D3F23226C8B40B3602B6843F016032B606B6943F080036B611AB132
:2034A0002B6843F008032B602B68002043F001032B60F0BC7047AA60E960E3E70220F0BCED
:2034C000704700BFF0B490F83530022B37D0036800221D492126DCB21D68103C25F00105FD
:2034E0005F2CA1FB04711D60184F4FEA11111A605A609A60DA601A618CBFA2F58062144AEC
:203500005E6188BF1A407D5C98BF1A404FF03F014FF0000388BF0432C565A9401C46826527
:203520009160436580F8343080F83530C0E90F33C0E91133C0E913332046F0BC7047DCB21B
:203540002046F0BC704700BFABAAAAAA8CD8050800FCFFFF0246F0B4494C2068002A56D076
:2035600002231168002582F8353082F834500B6823F001030B6003E023681B1A052B3ED8CD
:203580000B68DD07F8D4D2E90130D56803430F68D2E904402B432343146AD2E90665034365
:2035A0003848334338402B43556A2343042D40EA03002FD008604B6923F007031D43CBB297
:2035C00031484D61103B314CA0FB03505F2B304B4FF001054FEA101003EA01034FF03F01FB
:2035E000205C4FF0000488BF04338140D065204693659960546582F83550F0BC7047032300
:2036000020211846516582F83530F0BC70470120F0BC7047D2E90B74936A3C43204308600E
:203620004D6925F007051D4345F00405002FC6D07EB1B6F5005F12D0022B03D9032BBED16F
:20364000FB01BCD5012340211846516582F83530D3E7012B10D033F00203B0D1F0E7032BF1
:20366000ADD801A050F823F045360108413601084536010879360108B7F1C07F9FD1E1E76A
:20368000F83301203F8010E0ABAAAAAA8CD8050800FCFFFF0023C0E90033C0E90233C0E995
:2036A0000433C0E90633C0E90833C0E90A33C0E90C338363704700BF1F4BF0B4595C0446D6
:2036C000D2E9023645181069334356696758034390693343D6690343906A3343174E0343D8
:2036E0003E40D06A3343635090B16E69176B26F00706536B3843976B30436861605820F0ED
:20370000C07018436050635823F4C0033B436350566800201368EE60AB60094E6B681E406E
:20372000D2E908321E436E60635823F0F05313436350F0BC704700BFE05D06081F80FCFF44
:203740000000FFFF30B4614C0346614A655C0C1E18BF0124821A405918BF012220F00100BF
:20376000585192B98CB95B4A00212120116051609160D160116150615A5922F0F0525A51F0
:203780003F2200209A6030BC70475348181A18BF012014B908B9514AE6E74C1E18BF0124EA
:2037A0001ABB14BB4E4A00202124106050609060D060106154615A5922F0F0525A51012926
:2037C0000DD0022915D0032924D0042927D0052914D006292BD0072935D00120D3E74FF429
:2037E0007462002030BC9A60704760B95CB93D4AD9E74FF47C1200209A60C4E74FF4746212
:203800000020DA60BFE78C1E18BF01245AB954B9354AC8E74FF0746200209A60B3E73F228A
:203820000020DA60AFE738B934B9304ABBE74FF47C120020DA60A6E7CC1E18BF01243AB90D
:2038400034B92B4AAFE74FF074620020DA609AE710B90CB9274AA6E70C1F18BF012412B902
:203860000CB9254A9FE710B90CB9244A9BE74C1F18BF012412B90CB9214A94E710B90CB9A5
:20388000204A90E78C1F18BF012412B90CB91E4A89E710B90CB91D4A85E70D4A934203D1D7
:2038A000072901D11A4A7EE71A4A00202124106050609060D060106154615A5922F0F05207
:2038C0005A5100297FF47BAF5AE700BFE05D0608006002401060024000640240106402407C
:2038E000286002402864024040600240406402405860024058640240706002407064024048
:203900008860024088640240A0600240A0640240B8600240B86402402DE9F8433C4E337D84
:20392000012B6DD0012380460F463375F7F718FA054600285FD14FF0FF333B60D8F8003088
:20394000012B3DD0D8E901934B444B4553D9314C2DE0022B0CBF4FF400734FF440732269D5
:2039600022F440722261226913432361236923F0F8032361236943EAC90343F00203236138
:20398000236943F480332361BFF34F8FF7F7E8F9236923F07A032361002835D1D8F80830F8
:2039A00009F10109D8F8042013444B4523D998F80C30002BD3D0012BCBD14FF48073CEE7DF
:2039C000144CD8F80C3022691B0222F440729BB22261226942F0040222612269134343F4DD
:2039E00080332361BFF34F8FF7F7BAF92369054623F004032361002328463375BDE8F88391
:203A000002252846BDE8F8830546C7F80090F2E7B8490120003C02400B4B01E0013B10D08B
:203A20000269002AFADA0369074A43F00103036101E0013A05D0036913F00103F9D1184639
:203A400070470320704700BF400D0300144B10B4046C9C421AD800F530600023012903612D
:203A6000036943F400230361036943F018030361036943F0C043036104D14261036843F0E2
:203A80008023036000205DF8044B7047D0F8003B00F53060002BE0DA00205DF8044B7047BD
:203AA0000A30544F4B78012BF0B50D7826D000F53060404C404B00EB45104D6906693440A5
:203AC00004610469234003618B6805B14B610469C3F31203012A44F400240461046943EA3A
:203AE0000403036105D0036843F0044303600020F0BDCB68002BF6D04361F4E74B6993B3D4
:203B000000F510642B4FD1F808C004EB45142A4E6345D4F810E00EEA07072761276906EAFF
:203B200007062661266938D946F40026C1F814C0CCF31203012A2661266943EA0603236195
:203B400026D0BCF1000F08D005F00F020125D0F8343895401D43C0F834582368002043F024
:203B600004432360F0BD00F51060134EA3F50023012A00EB4514206906EA0006266120694F
:203B800040F400202061206903EA00032361E4D10B69002BE1D06361DFE746F40026C3F3AE
:203BA0001203012A2661266943EA06032361CBD1EEE700BF0000F8FFFFFF07E02DE9F043A0
:203BC0004D780F78012D4DD000F530636F4E4C6903EB47136E4D1F693E401E611E693540D0
:203BE0001D616CB38D68012A6A4E2C441F6904F1FF34B4FBF5F41FFA84FC06EAC44405FB07
:203C00000CF544EA0704C5F312051C611C6945EA04051D6121D0CA78012A0AD1D0F80828B2
:203C200012F4807F1A680CBF42F0005242F080521A601A6842F004421A600020BDE8F08384
:203C40008C68012A1D69C4F3120444EA05041C611C6944F400241C61DDD1CA68002ADAD02C
:203C60005A61D8E74B6900F51064002B37D104EB4714474E454D012AD4F810C00CEA060640
:203C80002661266946F400262661266905EA06052561CE7872D0012E59D1D0F8085815F406
:203CA000807F25680CBF45F0005545F080552560256845F004452560002ABED19BB20333C8
:203CC0009C08BAD0CA6800F5805302EB840403EB073352F8041BA2421960FAD1ADE704EB0B
:203CE0004714D1F808E0DFF8A490C3F31206D4F8108003EB0E0C08EA09090CF1FF3CDFF868
:203D00009080C4F81090D4F81090BCFBFEFE09EA0808DFF880C0C4F810800CEACE4CD4F8D6
:203D200010E04CEA0E0CC4F810C0D4F810C046EA0C062661CE78012E10D0012A22D007F0E9
:203D40000F03D0F834789D403D43C0F834582368002043F004432360BDE8F0832569012AC3
:203D600025F0C0452561256945F00055256194D10D69002D91D0164665618CE70D69002D64
:203D800089D0F9E70D69002DF6D1E0E70000F8FFFFFF07E00000F81F70B41D4E056803E0E7
:203DA0003468A41AA14226D3AB6913F02003F7D010222023EA61EB61AB699A0701D5002312
:203DC000AB62AB69DB0703D4AB6943F00103AB616B6800220F4C202123406B60436C80F8CC
:203DE000402043F00403436480F8411080F84220012070BC7047426C202180F840300A43B7
:203E0000426480F8411080F84230012070BC7047F833012000E800FE2DE9F041DFF8548021
:203E200004460E4615460AE09B69DB0602D5FFF7B3FFE0B9D8F800305B1BB34209D82368CB
:203E40002A46314620469F69BF07EDD50020BDE8F081636C2021002201200B4384F84020D2
:203E6000636484F8411084F84220BDE8F0810120BDE8F081F8330120F0B484460568049FB9
:203E8000104E03E03468E41B9C420AD8AC6931EA04000CBF012400249442F3D00020F0BCD9
:203EA0007047DCF844302021002201200B438CF84020CCF844308CF841108CF84220F0BCAE
:203EC000704700BFF833012003689A69196810B4D4052FD50C061FD5416C4FF4807441F075
:203EE000010141645105DC6129D5416C4FF48064920541F008014164DC6106D5426C4FF437
:203F0000007142F002024264D961416C11F00B0F0CD15DF8044B70475405F6D49405F4D595
:203F20000906EBD4416C11F00B0FF2D05DF8044BFEF7CABE5405F1D50906D6D4E5E79205CD
:203F4000DCD4E2E70268436B9169126803B11847704700BFF0B490F841200346002A40D0C3
:203F60002420DC68D3E9002183F84100012C106821F0706120F0010010601161916821F498
:203F800000419160996828D041F40441022C916002D14FF40061516051680020134C2026B7
:203FA0009F690C43D3E9041554602943DC69D56841EA07211F6A25F400453C43D560D16014
:203FC0001460116841F001011160586483F84160186383F84200F0BC704741F40041916076
:203FE000DAE702F0FF0180F84010B9E700800002F8B501F00F05012600271C21C5EBC5046E
:020000040801F1
:2040000001FB050100EB84043C31A264236584F83C50676584F83D600369B34208BFE264D5
:20402000DAB200681DB9FFF73DFD0020F8BDFFF7C5FD0020F8BD00BF2DE9F0410A46D0F806
:20404000A05200270B4E044685F838222F7205F50B720D238121C5F82C62D0F8A802FFF730
:20406000C7FF05F5037220461F230121BDE8F041F9F7B4BE555342532DE9F047137882B0C2
:20408000914604468A465A2B5CD8DFE813F0D0005B005B0080005B005B005B005B005B00DF
:2040A0005B005B005B005B005B005B005B005B005B00B5005B005B005B005B005B005B00F6
:2040C0005B00AB0177005B005B0077005B005B005B005B00CE015B00F8015B005B003D01B2
:2040E0005B00E2005B005B005B005B002A015B005B005B005B005B005B005B005B005B00B9
:204100005B005B005B005B005B005B005B005B005B005B005B005B005B005B005B005B00EF
:204120005B005B005B005B005B005B005B005B005B005B005B005B005B005B005B005B00CF
:204140005B001902D0F8A0120524002091F85D325A1C01EBC303D2B283F83C4283F84002AC
:20416000042A15BF4FF0FF354FF0FF3581F85D2281F85D02284602B0BDE8F087D0F8A032B1
:20418000002005465881284602B0BDE8F087D0F8A042002104F10B0304F11D0003F8011FA4
:2041A0008342FBD1702094F85C320C25207394F85D02E574984213D004EBC300013390F891
:2041C0003C52DBB2A573042B90F84152257690F8400218BF84F85C32607608BF84F85C1295
:2041E0001223638199F80430122B98BF63810025284602B0BDE8F08799F80130D0F8A002DC
:20420000DB0740F18081072100F1120300F10B0583224181C3F10604D44900E0127A03F8B2
:204220000129E218AB4211FA82F2F7D1DFE7D0F8A062D6F81472002F40F02582D0F8A4329E
:2042400008469B6898470546002840F05282708190E7D0F8A062357A002D40F0898196F9E0
:204260001832002BC0F26E81D0F8A43208469B6898470746002840F07B82D4F8A432504680
:20428000DB6898470546002840F05F82D9F80210D4F8A00209BAD0F86072C6F86412B9F8E5
:2042A00007305BBA9BB21944C6F86832B94200F27082B6F85E12D6F8142203FB01F39342E8
:2042C00040F09781B3F5007F4FF00101204606F10C0228BF4FF4007331729BB2F9F77EFDCB
:2042E00048E799F80150D0F8A03215F0020040F01A82D3F86012D3E9992422448A4200F266
:20430000E7810546588135E7D0F8A08298F80860002E40F0298198F91832002B80F2C6814C
:20432000D0F8A43208469B6898470546002840F04282D9F80200D4F8A06200BAD6F860724D
:20434000C8F86402B9F807305BBA9BB21844C8F86832B84200F2F680B8F85E22022003FB85
:2043600002F3D8F8142288F808009A4240F0EA80B6F85E324FF4007CD6F8687206F10C0597
:20438000D4F8A422504607FB03F72946A8F80AC06745D2F81080D6F8642228BF6746B7FB80
:2043A000F3F39BB2C0470028C0F259812A463B46D4F8A8028121FFF71BFEB6F85E52D6F8CB
:2043C0003432B7FBF5F5D6E99920DF1B2A44451BC6F83472C6E99925002D7FF408AF03234D
:2043E0003372C7E6D0F8A072082000225F4E07F11303788107F10B05C3F1070000E0127C62
:2044000003F80129C2189D4216FA82F2F7D1D4F8A4325046DB68984700283FF4E8AEBB7BF1
:20442000002563F07F03BB73A4E6D0F8A062002506F10B0306F1170203F8015F9342FBD1CA
:20444000D4F8A43250460DF1020201A95B689847002840F0DE80019B0821BDF80220022062
:20446000013BF17352BA0C211C0EF374F2821A0C1B0A34747274B374B0827181B7E6D0F8D5
:20448000A0620846D4F8A43206F25E2206F518715B6898470546002840F0CE80D6F860323B
:2044A0000821B6F85E22013B308252BA7181180EF373190C72821B0A30737173B37359E603
:2044C000D0F8A07208200022284E07F11303788107F10B05C3F1070000E0127E03F80129E3
:2044E000C218AB4216FA82F2F7D1D4F8A4325046DB68984700283FF47AAEFB7B002563F0DE
:204500007F03FB7336E6D4F8A44201EBC10199F80430E46904EB810422790532934228BF1B
:2045200013464381002B3FF462AE013B9AB2531C0C322344024413F8011D9C4202F80119F3
:20454000F9D154E696F85D3205211A460133DBB206EBC202042B82F8405282F83C1200F04B
:20456000A28086F85D3242E6464601E78CD80508B6F85E5206F10C08D6F868720846D4F8D4
:20458000A432414607FB05F7D6F86422D3F81490B7F5007F28BF4FF40077B7FBF5F39BB24A
:2045A000C8470028C0F22A81B6F85E02D6F83432B7FBF0F1D6E99925DB1B0A446D1AC6F88C
:2045C0003432C6E9992525B920462946FFF734FDD0E505FB00F3424620460121B3F5007F4F
:2045E0004FF0000528BF4FF400739BB2F9F7F6FBC0E590F85D3205215A1C00EBC303D2B21F
:2046000083F8405283F83C12042A39D080F85D22EDE5D4F8A022022092F85D32591C02EB99
:20462000C303C9B283F8405283F83C02042900F0D68082F85D12DAE5D4F8A0220220002583
:2046400092F85D32591C02EBC303C9B283F83C0283F840520429ECD182F85D528AE5D4F88A
:20466000A0220420002592F85D32591C02EBC303C9B283F83C0283F840528142D9D1EBE76E
:2046800080F85D5276E596F85D32052100251A460133DBB206EBC202042B82F83C1282F8E9
:2046A00040527FF45EAF86F85D5263E598F85D3205211A460133DBB208EBC202042B82F8AD
:2046C000406282F83C1200F08D8088F85D328EE593F85D22052411460132D2B203EBC10100
:2046E000042A81F8400281F83C427FD083F85D227DE5D4F8A0220220002592F85D321946E2
:204700000133DBB202EBC101042B81F8407281F83C0218BF82F85D324FF0050308BF82F8B0
:204720005D72337226E593F85D220520002511460132D2B203EBC101042A81F83C0281F88A
:204740004052D3D183F85D5214E5D4F8A022022092F85D3219460133DBB202EBC101042B39
:2047600081F8407281F83C0244D082F85D323EE5D4F8A022022092F85D3219460133DBB22E
:2047800002EBC101042B81F8405281F83C02ECD162E790F85D3205211A460133DBB200EB2A
:2047A000C202042B82F8405282F83C123FF468AF80F85D321BE5D4F8A022022092F85D3218
:2047C00019460133DBB202EBC101042B81F8406281F83C02C9D1354682F85D62CAE482F893
:2047E0005D5204E5354688F85D62C3E4054683F85D02BFE43D4682F85D72BBE4D4F8A022FF
:204800000420002592F85D3219460133DBB202EBC101834281F83C0281F84052A5D11BE768
:20482000D0F8A01210B50B7A022B07D0033B012B02D80021FFF700FC002010BD01F21B223C
:2048400091F819120446FFF717FC0028F4DA20460121FFF7F1FBEFE7F8B5D0F8A042054679
:20486000267A5EB1012E07D104F21B2294F81912FFF702FC00282FDB0020F8BDD0F8A832FB
:20488000D4F81012D3F83032D4F814221F2BC4E98C1208D12D4BD4F80C229A4203D194F8DF
:2048A000191201291DD994F85D32002105205A1C04EBC303D2B283F83C0283F840120223F2
:2048C000042A2846637214BF84F85D2284F85D12FCF7F0FC0020F8BD28460121FFF7ACFBCD
:2048E000CAE794F81A32013B0F2BDCD804F21B22FFF7C2FB0028237A1DDB013B022BBBD965
:204900006189F1B1D5F8A07204F10C020420D7F83432D7F814425B1A87F83862A142387290
:20492000D5F8A802C7F834320B4628BF23468121FFF75EFBA0E7052BCED02846FCF7BAFCDD
:204940009AE72846FFF778FB96E700BF5553424370B5D0F89062E6B101EB810500EB850539
:20496000EB695BB1D0F8A802C1EBC10400EB8404626CB3FBF2F402FB14341CB10020C6F82F
:20498000140270BD23462246EC61FFF731FB204670BD022070BD00BF002310B504241A4683
:2049A0001946C0F86C42D0F8A802FFF721FB002010BD00BF70B5054641B9D0F86C320C46E0
:2049C000032B10D0052B1FD0002070BDD0F88C329B6933B190F87422032A02D198470020D2
:2049E00070BD022070BDD0E953639E4212D8D0F88C321B6923B190F87422032A00D1984729
:204A00002846FFF7C9FFDFE7C5F86C12F9F772FA204670BDF61AB342C0F84C6128BF3346B0
:204A20009BB2F9F7DBF9204670BD00BF10B5134602240A460021C0F86C42C0E90733D0F84D
:204A4000A802FFF7D5FA002010BD00BFF0B5002383B00E460446ADF806300B78D0F8A0726A
:204A600013F0600522D0202D19D14A78FE2A11D0FF2A14D14A8892B9CD8885B91B060ED419
:204A80004FF4807107F503721F2339810121F9F7A5F908E04D8815B9CE88012E73D020460C
:204AA0000225F9F783FA284603B0F0BD4B780B2BF5D801A252F823F0F74A01081F4B010811
:204AC0009F4A01089F4A01089F4A01089F4A01089F4A01089F4A01089F4A01089F4A010846
:204AE0000D4B0108E94A010890F87432032BD6D18B787B60D7E790F87422032ACFD102226B
:204B00000DF106011D46FFF791FFCCE790F87432032BC4D1391D0122FFF788FFC3E70979E1
:204B2000D0F8A802FCF728F83179D4F8A802FCF755F8B38896F9042003F00F03002A4FF034
:204B4000000203EB830304EB83032ADBC3F84421237C9BBB4FF40073022201212046F9F7FE
:204B60002FFA0123C4F85831D4F8A0727B7A022B32D03279D20996D0012B94D0204601219D
:204B8000FFF75AFA8FE71A0689D5D0F8A4329B69984703463246204639463B60FFF746FFDA
:204BA00081E79A61237C83B94FF40073022281212046F9F705FA0123E362D5E7402302223A
:204BC00001212046F9F7FCF9CBE74023022281212046F9F7F5F9EEE720468121F9F78AF9F9
:204BE00000237B725FE700BF10B50C7882B00023D0F8982214F06004ADF8063016D0202C0B
:204C00000ED14B78023B092B0AD8DFE803F033390909090909093F2F90F87432032B5AD04F
:204C20000224F9F7C3F9204602B010BD4B780B2BF6D80FF2080C5CF823F000BFC14C0108A5
:204C4000214C0108214C0108214C0108214C0108214C0108974C0108214C0108214C01082E
:204C6000214C0108194C0108B34C01088B7800241360D8E7111D01220024FFF7D7FED2E7F6
:204C8000114601220024FFF7D1FECCE74B8800241B0A5360C7E74B881B0A222B1FD0212B01
:204CA000BED1CA881149092A28BF0922FFF7BEFEB9E790F87432032BB2D18B789360B2E7B4
:204CC00090F87422032AABD102220DF106011C46FFF7ACFEA7E702F108010122E6E7CA8816
:204CE0000349362A28BF3622E0E700BF24060120EC0501202DE9F0410A7884B000270D466F
:204D000012F060060446D0F890328DF80D70ADF80E7016D0202E1AD1CE8806B3120643D5D4
:204D200019460193D4F89432324668783E46D3F80880C047019BEA8820461946FFF776FE7B
:204D400009E04B780A2B20D00B2B28D08BB120460226F9F72BF9304604B0BDE8F081D0F86E
:204D60009432324648789B689847304604B0BDE8F08190F87432032B29D002262046F9F740
:204D800015F9304604B0BDE8F08190F87432032BF3D101220DF10D01FFF748FEDBE790F8F0
:204DA0007432032BD7D0E8E74A78032583F80162394683F800221A46C0F848613346C0F8D3
:204DC0004C613E46C0F86C52F9F708F8C3E702220DF10E01FFF72AFEBDE700BF2DE9F04397
:204DE0000D784FF0010883B0044680F8805205F01F0C4F7800F5207EC44580F88172CB78EE
:204E00008E7806EB0326B6B2A0F882624A790B7903EB02239BB2A0F8843291F807908A7976
:204E2000C0F86C8202EB092292B2A0F88622C0F870220DD0BCF1020F3ED0BCF1000F19D098
:204E400005F08001F9F756F8002003B0BDE8F08305F06002402A67D06A0665D5802120460A
:204E6000F9F748F820460021F9F744F8002003B0BDE8F08305F06005202D6FD0402D6DD0D4
:204E8000002DEBD1092FE9D801A151F827F000BFA94F0108D74F01085D4E0108F54F01083E
:204EA0005D4E010805500108655001085D4E010891500108714F010805F06005202D4DD0F7
:204EC000402D4BD0002DC9D1012FD9B200F00481032F00F0EF80002FC0D190F87422022AB8
:204EE00000F0CC81032AB9D113F0800F01F00F0303EB830300EB830340F0D881D3F844317B
:204F0000002BABD001F07F03142202FB030202F5A072002B40F00D820023136011462046FA
:204F20000222FFF783FD8FE794F87422013A022A94D8DBB2032B91D8D4F88C3271462046A1
:204F40009B689847B4F88632002B7FF47DAF00287FF47AAF2046FFF71FFD75E7D4F88C321F
:204F6000714620469B689847002003B0BDE8F083F1B2C14D012985F806123FF66FAF90F8FC
:204F80007432022B00F0BE81032B00F0A9818021F8F7B0FF00212046F8F7ACFF95F80612C2
:204FA0002046FBF7B5FC4FE790F87432013B022B3FF654AF022A7FF451AF0122D0F87C32AB
:204FC000C2600BB10323C360022204F10C012046FFF72CFD38E790F87432013B022B3FF614
:204FE0003DAF012E7FF430AF0023C0F87C32FFF7D3FC29E7012E7FF427AFC0F87C62FFF7E2
:20500000CBFC21E713437FF429AF7F2E3FF626AF90F87432032B3FF421AFF1B2D0F8A832C5
:2050200080F8761293F8BC23012A11D01A68002083F83810D2F8001821F4FE61C2F800186D
:20504000D2F8001841EA0611C2F8001883F8BC032046FFF7A1FC002E00F07C81022384F86B
:205060007432F1E6330A013B062B3FF6F7AE01A252F823F0F5510108DB510108C951010888
:205080005D4E01085D4E0108B35101086D510108012A7FF4E3AE90F87432022B00F2FF80D9
:2050A000002B3FF4DBAE0023014641F8083FFFF7BDFCC9E690F87432022B00F0D380032BF5
:2050C0007FF4CCAE4F063FF445AF56EA02037FF441AFF8F70FFF3DE790F87422022A00F064
:2050E000C180032A7FF4BAAE002E7FF4ADAE48063FF430AFD4F8A80201F00F014268914217
:205100003FF628AF13F0800F4FF01C0340F0268103FB01020025134602F5FE7283F8FD510D
:2051200000231170937090F8BC33012B3FF412AF0121036880F8BC1355781178012D0CBF0E
:2051400003F5106303F5306303EB4113196821F400111960D278023A012A03D81A6842F0B7
:2051600080521A60002380F8BC33F3E6037C002B7FF474AED0F88C320DF106001B6B984752
:2051800007234370BDF806306BB1B4F88622002A3FF4E0AE9A420146204628BF1A46ADF877
:2051A0000620FFF743FCB4F88632002B7FF44CAED0E6037C002B7FF451AED0F88C320DF142
:2051C00006005B6B9847DDE7F6B2052E3FF646AEDFE806F0302820184038037C002B40F0BD
:2051E0009F80D0F88C320DF106009B6A984702234370C7E7D0F888320DF10601007C1B6816
:205200009847BFE7D0F888320DF10601007C1B699847B7E7D0F888320DF10601007CDB68BF
:205220009847AFE7D0F888320DF10601007C9B689847A7E7D0F888320DF10601007C5B68C0
:2052400098479FE7D0F888320DF10601007C9B69984797E7D0F888320DF10601007C5B69BE
:2052600098478FE74D063FF4F9ADF8F743FE20468021F8F73FFEE7E5E08D01204A067FF42D
:20528000EDAD1B064FF000034FF002024CBF00F1140100F5A0710B60FFF7C8FBD4E5032BAC
:2052A0007FF4DCAD011DFFF7C1FBCDE59B69002B3FF4D4AD01F07F035A1C02EB820200EB48
:2052C0008202002B3FF428AED0F8A8121C2000FB031393F83E30002B3AD0012313601DE67F
:2052E00079B3416801293FF435AEC9B2FBF710FB95F8061220466160FBF712FB02287FF4B9
:2053000029AEABE500293FF425AE01210323416080F87432FBF704FB02287FF41BAE9DE517
:20532000D0F88C320DF10600DB6A98470223437028E7D0F8A8321C2000FB013393F8FE3111
:20534000C9E70223416080F87432FBF7E1FA01E61360E3E5012384F8743275E503FB010229
:20536000012513463C3283F83D50D9E603682DE9F04F13F0010785B000F0F080C44A13F404
:205380000025916821F400019160C46A9168B4FA84FE41EA04014FEA5E1E916000F0E38068
:2053A000BB49446BD1F88C20B4F5801F22F4401242EA0402C1F88C2000F0B681B4FA84F431
:2053C00013F480124FEA5414019240F0D280990600F1E480DE060CD5AD49D1F88C2022F048
:2053E0008072C1F88C20D1F88C20066B3243C1F88C20590408D5A649C66DD1F8902022F4AB
:2054000040323243C1F890201A0408D5A049066ED1F8902022F440223243C1F89020DE0334
:2054200008D59B49466ED1F8902022F440123243C1F89020590608D59549C66BD1F8902074
:2054400022F003023243C1F890201A0608D59049066CD1F8902022F00C023243C1F8902098
:20546000DE0508D58A49466CD1F8902022F030023243C1F89020990508D58549866CD1F848
:20548000902022F0C0023243C1F890205A0508D57F49C66CD1F8902022F440723243C1F805
:2054A00090201E0508D57A49066DD1F8902022F440623243C1F89020D90408D57449466DCD
:2054C000D1F8902022F440523243C1F890209A0408D56F49866DD1F8902022F44042324321
:2054E000C1F8902013F4001C0ED06949D0F87480D1F89020B8F1006F22F0006208BF0124E3
:2055000042EA0802C1F890205E0309D5DFF88081C26ED8F8901021F040710A43C8F89020B6
:20552000190209D5DFF86881826FD8F8901021F080510A43C8F890205A0100F18E80B3F1B4
:20554000007F00F09980BEF1000F40F09580012C00F0F180002005B0BDE8F08F13F400250D
:20556000BE467FF41DAF2C4613F4801201923FF42EAFDFF81CC1816BDCF88C20B1F5800FE5
:2055800022F4400242EA0102CCF88C2000F0D080002908BF012499067FF51CAFDFF8F0809A
:2055A0003C4AD8F840903C49944649F08059C8F84090D8F8408008F08058CDF80C80DDF83E
:2055C0000C80D2F8008048F48078C2F80080D1F8008005E00A68A2EB0802642A00F2A080B0
:2055E000DCF80020D205F5D5DFF8A480D8F8702012F4407C826A02F4407919D0E14517D068
:20560000D8F870C0D8F870A02CF4407C4AF4803AC8F870A0D8F870A02AF4803AC8F870A07E
:20562000C8F870C0D8F870C01CF0010F40F00581B9F5407F00F0EE80DFF854C0DCF8081006
:2056400021F4F811CCF808101149C2F30B02D1F870C042EA0C020A67BCE6DFF83480B3F1BF
:20566000007FC26FD8F8901021F0005142EA0102C8F890207FF467AF054A0749D2F8008097
:20568000964628F08068C2F80080D1F800800AE00038024000700040F83301200A68A2EB4C
:2056A0000802642A3CD8DEF800201601F6D46FB1C26A5AB98268DEF884704668120707F096
:2056C000706742EA86123A43CEF88420002D40F08380019A22B1826BB2F5800F00F0818066
:2056E0009A010AD5C36842681B06876843EA82135B4A43EA0773C2F88430594B1F681A4644
:2057000047F080671F600F6803E00B68DB1B642B06D813681B01F8D5012C7FF41BAF0AE004
:20572000032005B0BDE8F08F00244FF0010E1BE74FF0010E4BE64A4B4A491C681A4624F05A
:2057400080541C600C6803E00B681B1B642BE7D813689E00F8D4002D6BD1019BC3B1836B5F
:20576000B3B93F4A4369D2F8884005691B0604F4403443EA85132343C2F88830D2F88C30D8
:20578000046A23F4F853013C43EA0423C2F88C30BCF1000F10D0436FB3F1006F0CD1836908
:2057A0002F4C00691B04D4F8882043EA801302F070621343C4F88830294B18681A4640F0A0
:2057C00080501860086803E00B681B1A642BA7D813689B00F8D5BDE6426BB2F5801F7FF48C
:2057E00078AFDFF87CE0C268DEF884704668120607F0E04842EA861242EA0802CEF8842012
:20580000DEF88C70C26927F01F07013A3A43CEF88C2065E7DFF84880DFF84CC0D8F808106E
:2058200002EA0C0C21F4F81141EA0C01C8F808100AE7436B002B94D08FE7D1F800B041F2E6
:20584000883A06E0D1F800C0ACEB0B0CD4453FF667AFD8F870C01CF0020FF3D0E8E600BF98
:2058600000380240F8330120FFFCFF0F054A064B92680649C2F382220868134493F8203075
:20588000D8407047003802408CD80508F42B0120134908B58B6803F00C03042B1DD0082BB1
:2058A00019D14A684B68496802F03F0213F48003C1F388111ABF0B4800230B48A1FB00019F
:2058C00045F042F9064B5B68C3F3014301335B00B0FBF3F008BD044808BD024808BD00BF89
:2058E0000038024000127A000024F400F8B504468368B849E669E768B74DD0E904201A43CB
:20590000236802431868AB4201EA000142EA060242EA0102A1691A605868226A20F4405087
:2059200042EA010240EA07005860996821F4306142EA01029A605FD0A84A93421CD0A84AAB
:20594000934200F00881A74A934200F01281A64A934200F08B80A54A934200F0A380A44A2B
:20596000934200F05381A34A934200F0208100230120C4E91833F8BD9F4BA04AD3F89030EB
:2059800003F00C03134493F82C30B6F5004F17D0082BECD801A151F823F000BFD55A0108FA
:2059A000155A0108BB5A01086F5901088F5A01086F5901086F5901086F590108455A010873
:2059C000082B06D8DFE803F0BBA79E0592050505890001200023A3F110014FF6EF7291426B
:2059E000C5D823F00F02C3F3420321681343CB600023C4E91833F8BD7F4B804AD3F89030F2
:205A000003F00303013B022B40F29C80B6F5004F00F0818078497A4B89681B68C1F34231CA
:205A200060680A4492F82020D34003EB5003B3FBF0F39BB2A3F110020DE0302B97D1B6F553
:205A4000004F4AD06268530803F50043B3FBF2F39BB2A3F110024FF6EF718A4287D822689D
:205A60000020D3600023C4E91833F8BD624BD3F8903003F44073B3F5007F1BD066D833B3EB
:205A8000B3F5807F7FF473AFB6F5004F2ED0FFF7FFFE636800EB5300B0FBF3F39BB2A3F164
:205AA0001002D8E7544BD3F8903003F44063B3F5006F70D1B6F5004F24D06268514B03EBB7
:205AC0005203B3FBF2F39BB2A3F11002C3E7B6F5004F34D0FFF7CAFEDBE76268002053087E
:205AE00003F58033B3FBF2F39BB274E7FFF7D0FE6168034600204A0802EB4303B3FBF1F3B3
:205B00009BB268E7626800203F4B03EB5203B3FBF2F39BB25FE738490020394B89681D6871
:205B2000C1F3423166680A44730892F8202025FA02F203EB4203B3FBF6F39BB24BE7FFF78B
:205B400095FED5E7134493F828301EE7B3F5407F3FF475AF0BE7284BD3F8903003F03003E3
:205B6000202BA7D03FF669AF002BB0D0102B8BD0FDE6214BD3F8903003F0C003802B99D031
:205B800005D8002BA3D0402B3FF47EAFEFE6C02B3FF455AFEBE605D8D3B1B3F5806F3FF4CC
:205BA00073AFE4E6B3F5406F3FF449AFDFE6124BD3F8903003F44043B3F5004F3FF47AAFFD
:205BC0003BD8002B83D0B3F5804F3FF45DAFCEE60A4A1BE7F369FFEF001001400044004055
:205BE00000480040004C0040005000400014014000780040007C0040003802408CD805084D
:205C0000F42B01200024F4000048E8010D4BD3F8903003F44053B3F5005F3FF44BAF07D87B
:205C2000002B3FF454AFB3F5805F3FF42DAF9EE6B3F5405F3FF403AF99E6B3F5404F3FF4D4
:205C4000FEAE94E600380240002807DB00F01F0101234009024A8B4042F82030704700BF06
:205C600000E100E0034A0130116813685B1A8342FBD37047F833012001F01F01036A10B4A4
:205C800001248A408C4023EA04035DF8044B0362016A0A4302627047034690F83C00012823
:205CA00000F0C6800220F0B4012483F83D0083F83C40002A31D0042A73D0082A1A6800F0D4
:205CC0009580166AC86826F480560D684F688C68010316622D03D06989B2166A05F42045F1
:205CE00020F4407026F4204640EA0720354320F470400143D1611562D06920F44060D061C8
:205D0000D16941EA0421D16100220121104683F83D1083F83C20F0BC70471A68DFF814C1FD
:205D2000166A62450C6826F001064D68C86816629769166A1DD0B2F1804F1AD0ACF57C4C1C
:205D4000624516D00CF5806C624512D00CF5806C62450ED00CF5784C62450AD00CF5705CBB
:205D6000624506D0ACF5943C624502D047F0010502E027F003073D43000125F0F00526F0DB
:205D80000A0604F00A04C0B28F683443284390611462906920F00C009061916939439161D1
:205DA000B2E71A68C868166A0D6826F010064F688C68010316622D01906989B2166A05F079
:205DC000A00520F4407026F0A00640EA0720354320F47040014391611562906920F44060B7
:205DE0009061916941EA042191618DE7176AC86827F480770E684C688D680101176236026D
:205E0000D069C9B2176A06F4206620F0030027F4206720433E4320F0F0000143D161166246
:205E2000D06920F00C00D061D1692943D1616BE702207047000001400368012201F01F01F9
:205E4000186A02FA01F120EA010010B418620F4C1A6AA34241EA0201196212D00C4A93420F
:205E60000FD099680B4A0A40062A06D0B2F5803F03D01A6842F001021A6000205DF8044B6F
:205E800070475A6C42F400425A64EAE7000001400004014007000100F0B490F83D30002B2C
:205EA00066D0026802233B49B2F1804F80F83D30A2EB01011368B1FA81F14FEA51113BD075
:205EC000002939D1344D354CA24218BFAA4233D0334F05F50065D71BAA42B7FA87F74FEABC
:205EE00057174AD0002F48D12E4F2F4CA24218BFBA420CBF012700274AD02C4DA4F5963413
:205F0000A24218BFAA4220D004F58064A2423FD004F58064A2423BD0816923F08003C468A2
:205F20000B4341681360D46291620123536180F83D300020F0BC7047194F23F070038568B3
:205F4000D71B2B43B7FA87F77F09046923F4407385692343C668446823F080032B4313604E
:205F6000D662946209B9002FDFD043691363DCE703F0FF0280F83C2093E70D4C23F070034D
:205F80008568A24243EA0503DFD0002FDDD1ABE70027DAE700000140000400400008004028
:205FA00000040140004001400044014000480140000C004010B4016802240B4A034680F858
:205FC0003D4088680240062A06D0B2F5803F03D00A6842F001020A600122002083F83D20A7
:205FE0005DF8044B704700BF070001000B4B93F81621D20703D5012283F80722704793F8AD
:020000040801F1
:2060000007224AB9D3F8783133B1054B1A7810445A78114418705970704700BFE08D01204A
:20602000D852012040F0080210B50D4C84F8412294F9BC21022A06DD420704D583071CBFDE
:20604000012384F8C43105210648FAF761FF062184F842020348BDE81040FAF741BF00BF0F
:20606000F00301202D06012010B5FAF7E9FEA8B31B4C94F9BC31012B30DD59B3022B2DD070
:2060800094F8C4319BB971B180230521154884F84732FAF73DFF062184F848021148BDE8D6
:2060A0001040FAF71DBF0420BDE81040BAE7002914BF0020042094F8BF311A0748BF40F0F5
:2060C00002005B0701D411B108B940F00100BDE81040A7E7022BD3D10420ECE710BD00BFFC
:2060E000F003012033060120F8B5224C030A0546062104F2492784F84E0284F84D323846ED
:20610000FAF706FF94F8BF3184F84F02DB072AD4B4F8C021AA4226D1174D41F26F71D4F8AD
:20612000493205F50276C5F80832C3B2304685F80E324FF6FF738A4218BF012306211344D7
:20614000C3F3072285F80D3285F80C22FAF7E0FE072185F80E023046FAF7C2FE052104F52F
:206160001470FAF7BDFE07210448BDE8F840FAF7B7BE00BFF0030120E08D01203906012077
:2061800008B5FAF75DFE48B1A1F59C53083BB3F57A7F03D20846BDE80840A5E708BD2DE91D
:2061A000F0476A4E3368002B3AD0694D694C05F5DE77306827F086FD002833D1664B1988B6
:2061C0001D46092909D95F8864227A43B2FBF1F2452A40F39E811880588094F84932012B2A
:2061E00000F0C281022B00F0DD8133B905215B48FAF776FE012384F84932594B1D68594BEF
:206200001B78002B00F0D881574B1B68EB1A782B40F2D281D4F89001F7F7A6FCC4F84C52DE
:20622000BDE8F087306827F045FD94F80F328046052BBED8DFE803F00309151B3543AA28B8
:20624000B7D1012384F80F32B3E7552817BF424A0223938801331CBF9380002384F80F321A
:20626000A7E7032384F8100284F80F32A1E7132884F81102C4F82C0207DD374AD3880133EF
:20628000D380002384F80F3293E718B9052384F80F328EE70023C4F83032042384F80F3201
:2062A00087E7D4F83032E218013382F81202D4F82C22C4F8303293427FF47BAFE6E7D4F843
:2062C0002C322A4803F1020A4FFA8AF1FAF720FE804594F8109240F0148126201BF03CFCDA
:2062E000204B48B100221A701B4A538801335380002384F80F325CE71A784A4519D10022F7
:206300001A7009F1FF33102B00F2F680DFE813F030008D008D00DE008D00F400F400F400C9
:206320003000F400F400F400F400F400F400F4003000B9F1090F02D0B9F1110F01D1012AF6
:20634000DDD0054A538901335381DAE7D4520120F0030120E08D01200253012040060120D6
:20636000A82A01201053012014530120F08F0120BAF1060F59DDB9F1010F06D0B9F1090F36
:206380000CBF4FF002094FF0030994F8150294F8161294F8142241EA002194F912E294F92A
:2063A00014C2900709B294F8133285F8BC9185F8BDE185F8BFC1A5F8C01106D512F00C0F9C
:2063C00014BF0122002285F8C421B9F1030F12D1BAF1090F29DD94F918220020082AA8BF5B
:2063E000082222EAE27285F8F22143B201309A425ADC94F817320020D4F81CA09BB2024639
:206400005245904658DB7C4B85F8BE011B78232B0BD109EB8903794A03EB8303A2F802E0E9
:2064200091800CEB8303D08013800A227449754846F0FCFD10B1002384F83E32704B3A68E9
:206440001A607A685A603A891A8194F83E3233BB95F8C4316C4A002B117814BF02230123D6
:2064600084F8401284F83E3295F8BF3113F0010318BFB1FA81F3517818BF5B0984F8411215
:206480009188D8B29278A4F8421284F83F0284F8442213B109B1A4F8461284F848020EF08A
:2064A0004FF80EF04DF81FE704EB4308234493F81A32A8F87E3198E7013204EB480852B290
:2064C000B8F82080984508BF104699E7BAF1040FABDD94F8122294F8133243EA022359046C
:2064E0001AB204D5C3F30D03A5F8C2319DE7002AF8DBA5F8C03198E7444A93890133938121
:20650000F2E619F0010F01BF404A138901331381EEE63F4BD3F85822B3F85C12012A1AD10A
:2065200041F25632914203D14FF0FF32C3F85822D3F85822306802EB820202EB820201EBA9
:20654000420189B2A3F85C1203681B69984700232B806B8041E60132EAD1B1F5965F04BFBA
:206560000122C3F85822E3E7294D95F9BC61002E3FF443AE022E11D14FF48040FFF7B4FDCA
:2065800084F8496295F9BC31012B7FF736AE95F8BF31C3F3400385F8C4312EE6032384F835
:2065A0004932EFE71A4BB3F8C231002B3FF425AE032384F8493220E694F8342094F8353062
:2065C0009A4204D0FBF7F4FAC4F84C5228E6D4F84C32EB1AB3F57A7FBFF422AE0D4B1B6875
:2065E000ED1A952D7FF61CAE05210B48FAF778FCBDE8F047FBF7DCBA104901201449012059
:2066000014900120AC050120D852012002530120F00301201453012040060120104BD3F8F9
:20662000780110B5D8B10F4C217841B162780DF0E3F9A388834216BF01210021A080E28868
:206640005AB141F288339342B8BF13469A4204D0E380BDE8104039F055BE0029F9D110BD98
:20666000E08D0120D85201200023014410B410F8014B0822634013F0800F4FEA4304234679
:2066800016BF84F00703E3B2DBB2013AF3D18842EDD118465DF8044B704700BF30B54FF45E
:2066A000806085B021F0E4FD48B3164C002301214FF4E13294F8505290F904009D420191AF
:2066C00000924FF4806118BF08250F4A029521F02EFE206700384FF0FF0318BF012084F85F
:2066E0008C3084F89C3084F8AC3084F8BC3084F8CC3084F8DC3084F8EC3084F8FC3005B0E1
:2067000030BD00BFE08D0120C5110108364B1B6813F0006359D0354B2DE9F0471F78B8426F
:206720004ED3FF2853D1DFF8D8A09AF8CC31002B43D0DFF8D0800022C8E99522C8F85C22E2
:20674000A8F86022002F4BD008F18C031046144611461546164603EB0719B3F802E01033A9
:2067600033F804CC714413F810EC624413F90FCC764509B212B238BF7646654553F80CECFB
:20678000B8BF654653F808CC994574446044E4D188F8546288F8555291FBF7F192FBF7F282
:2067A000C8E99640124B0020A8F856121B78A8F86022092B8AF8CC010CD00E48BDE8F08747
:2067C0000D4A02EB0010BDE8F087184670470020BDE8F08798F85422084B0648DA80F2E71E
:2067E0003A463946DEE700BFD85101207007002010490120349001206C8E0120144901203D
:20680000F0030120E08D012070B40478A51E15F0FF061DD0451E02464FF6FF73354401E0C0
:2068200012F8014F1B1BAA429BB2F9D11C0A084410F8012CA24205BF10F8020CDBB20020B3
:20684000C01A08BFB0FA80F070BC08BF40097047FF244FF6FF73EAE72DE9F8434378434C44
:20686000190703F00F0594F8642200D072B10021AA4284F8681204D94FF000084046BDE89A
:20688000F883AA1AD1B20E29F6D803E084F8645284F86822224492F8AC110029ECD003F091
:2068A000F003802B40D0902B49D0A02BE4D1084665F05F05FAF7C6FC02462D48131D84F8B3
:2068C000695284F86832FBF705FB94F86882B8F1000FD1D0A8F1020313F0FF0641D0254A00
:2068E0004FF6FF71901912F8015B491B904289B2F9D15FFA81F90D0A4BB11E4FFE1817F821
:20690000011BD4F88C0227F003FABE42F7D14946D4F88C0227F0FCF9D4F88C02294627F050
:20692000F7F94046BDE8F883042365F07F050226984684F8683284F869523346CFE70846F1
:2069400065F06F05FAF77EFC0426062284F86B02334684F86952904684F86A1284F8682244
:20696000BDE7FF254FF00208A946C5E7E08D01204A90012048900120C21D2DE9F04F02F4BF
:20698000FC7285B0524C064600AFD4F89032ADEB020D04F5287A89460DEB0002E84653455C
:2069A000FA602FD094F8E0130DF1010C94F8E10301F00F0ED4F894520131C7F808C04EEAD3
:2069C000401E07F1080084F8E0138DF800E0ED1AA2EB0C0B1946AB4544DD2A4638F0F4F8E6
:2069E000D4F89022B96840462A44C4F890A2A1EB0801C4F89422C9B2C84700201437BD4617
:206A0000BDE8F08F94F8E05394F8E10305F00F01B4F99AC2013541EA4011BCF1000F84F82B
:206A2000E05341F01001D4F89452C9B2A5EB0A0BB8BF41F08001012888F8001022D1BBF18E
:206A4000FE0F38DD07F10800FF2594F8982208F103031FFA8BF1786088F8015088F80220CB
:206A6000BB6020E05A4638F0AFF8D4F89032404631465B44C4F89032C84701201437BD4666
:206A8000BDE8F08F07F1080094F89C2208F10203B4F89812786088F80120BB6038F0D8F8A8
:206AA0001FFA8BF1786838F0D3F87868D7E902C2D4E9A4358BE794F8981208F1030C07F1CC
:206AC000080088F801B088F80210C7F808C07EE7E08D012010B5062982B004464FF032038D
:206AE0000A460DF1010028BF062221468DF8003046F052FA024B68461B68984702B010BDBE
:206B0000189201205E2810B50ED05D2804D00B4BBDE810405B681847084C636898476368F2
:206B20003D20BDE810401847044C5D206368984763683E20BDE81040184700BF1892012026
:206B400070B5084E05460C465E2073689847284673689847E0B2FFF7D5FFC4F30720BDE8DE
:206B60007040CFE7189201200368002B2DE9F041B8BF5B423A4F04463A4DA7FB03013A4E6B
:206B8000890DB27905FB0135C5EB0515AD0087FB0537EB17C3EBA757002A55D101EB81015D
:206BA00001EB810107EB810109B2DFF8B8801320FFF7C6FF1B2008FB07552C4FE91787FBA4
:206BC0000535C1EBA511264D09B2FFF7B9FF23682320002BB4BF53214E21FFF7B1FF63687D
:206BE000B279002BB8BF5B42A5FB0301890D08FB0138C8EB08184FEA880885FB08354FEA23
:206C0000E873C3EBA5552ABB01EB810101EB810105EB810109B21220FFF792FF114B134912
:206C20001A2003FB058581FB0531ED17C5EBA11109B2FFF785FF63682220002BBDE8F04137
:206C4000B4BF572145217BE7C1EB011107EB810109B2AAE7C1EB011105EB810109B2DAE757
:206C60006BCA5F6B806967FF808F0120D34D621000234FF4167140F2D932018142814380D2
:206C80008380838130B4022515240580847130BC7047084B5A881B88801A9B1AC00090FB1A
:206CA000F3F00628A8BF062020EAE070C0F19600C0B27047BC8F0120094B03EB40021189E2
:206CC000084A127802EAD122520707D0D3F88420511CC3F88410134483F88800704700BFCE
:206CE0001892012050060120164B426810B51B7803F00303032B21D1134B1B88DBB11349ED
:206D00000A24134BB1F90410B3F9C63091FBF4F15B1A4FF4B4711B0103F5B9531433B3FB24
:206D2000F1F3C3F1080303F00F0360331370436800225A7010BD05231370F8E72D231370D4
:206D4000F5E700BF7C8F01207E8F0120A052012018920120436872221A70732243685A708D
:206D6000742243689A7000224368DA7070470F4B0A214268B3F9043093FBF1F31B014FF41A
:206D8000B47103F5B9531433B3FBF1F310B503F00F03074C1919E35813604B6853600B7A09
:206DA0001372002243685A7210BD00BFA0520120E4630608044B93F8CD3013F0FD0F14BF08
:206DC0009E209D20704700BF18920120094B93F8CD3013F0FD0F06D142F210735843064B92
:206DE00090FBF3F07047242358434FF47A7390FBF3F070471892012040D20600064B07EE0E
:206E0000900A93F8CD30B8EEE70A1BB9DFED037A20EE270A704700BF1892012048F951404A
:206E2000104B10B593F83421012A10D1D3F83821811A00290BDD0221B3F82E4183F8341179
:206E40000949B1FBF4F142B10A44C3F8382193F83401013818BF012010BD0844C3F83801FC
:206E6000F5E700BF1892012040420F00831E00F17A02EA2123F8021F9342FBD14E2243F67C
:206E80004913C280CE224385CD23028123228380A0F87220A0F87830704700BF30B400BB62
:206EA0001D48B0F83C3103F00103C3B990F84041ACB11A4A02F1F00502E00133A3420ED05A
:206EC00052F8041B4904F8D590F82C1200EB8101D1F8C41145F823100133A342F0D130BC28
:206EE00070470D48B0F83C31032B4FEA530408D90D6804F001030A4AA0F83C412A440A6024
:206F0000D3E70A6848F20504054BA0F83C41134430BC0B60704700BF189201205C9301209E
:206F2000A08601002DE9F04100283AD12D4A92F8400180B32C4A00242C4B92F804E092F931
:206F400005C003EB8000CEF1FF07AEF17F0692F9068003F1F002FFB2F6B203E0834202F12A
:206F6000040218D053F8041B8904F7D5E1B2A1EB0C0181EAE175A5EBE175012D0DDC71B154
:206F8000414514BF394631468342D17004F1010402F10402E6D1BDE8F0810821F4E7714621
:206FA000F2E7114B1A79F02A09D802F10F000D4A1871086844F21A1303440B60B7E7094AB6
:206FC0007F2593F9054092F842011D718442987901DA002C02DA4042C0B2987120445871FD
:206FE000E7E700BF18920120500601205C930120F0B5384E78B196F8B432002B46D0013B6D
:20700000354ADBB286F8B4321378DB0741D4334B0A681A440A6096F84041B4B3304B0025B0
:207020002D4F03EB840403F1F00003E09C4200F104002AD053F8041BC1F30322062AF5D191
:2070400097F800C0EA431CF0010F02F001020DD096F8B42296F843E102EB050CBCFBFEF20B
:207060000EFB12C2012ACCBF002201220135002ADCD0C1F383419C4200F1040006EB81016E
:20708000D1F8C42140F8042CD4D1F0BD96F84331B5E7D6EDB17A6420124BFDEEE77A124D70
:2070A000124C17EE902AA2F57A7200FB02F283FB0230D317C3EBA01303EB4303C3EB03134E
:2070C00085FB0302DB17C3EB6213053394FBF3F39EE700BF18920120F68E0120400D030065
:2070E0005C930120D34D62101F85EB5140420F00F0B4524C002864D194F8000300285CD0FB
:207100004F4BB3EE097AD3ED007AF4EEC77AF1EE10FA54DCBBEE097AF4EEC77AF1EE10FA03
:207120004CBF08270027B3EE097AD3ED017AF4EEC77AF1EE10FA6FDD47F0010794F84051DB
:20714000002D3AD03F4ADFF80CC102EB850502F1F00011E094F90363B142ACBF02210021EB
:2071600094F90463B34218DB41F004010F421CD1954200F1040020D052F8043BD903F7D5D2
:2071800003F00F0194F90263C3F30313B142E1DC94F904630121B342E6DA94F90563B342C9
:2071A000D8BF41F008010F42E2D0DCF80C30954200F1040040F8043CDED1F0BC704704276A
:2071C000B1E794F801338BB31D4B1F4ED3ED007A93ED017AF0EEE77A1C4DB0EEC77A0A6816
:2071E00094F80003C7FE877AFDEEE77A80F0010017EE903A84F80003193B03EB4303C3EBF9
:20720000031386FB0376DB17C3EBE6130533B5FBF3F31A440A6071E7BBEE097AF4EEC77A88
:20722000F1EE10FA48BF47F0020787E70A68084B94F8000313440B6060E700BF18920120C9
:20724000AC8F01205C930120353AFC4440420F00400D0300FCD80508F0B40D4F97F8406121
:20726000A6B107F5A272054607F50D77002302E00133B3420AD052F8044B35EA0400F7D150
:20728000086847F823000133B342F4D1F0BC704718920120294B30B460B9294A127DBAB91A
:2072A00093F82D322749203301EB83014FF4A06030BCD1E793F80603E0B10138204A83F887
:2072C00006030C68204820440860127D002AE7D01E4A12689106E3D51D4A93F806131278C7
:2072E00092071AD511BB93F82F321649203301EB8301DBE7124A93F80743157DA54205D8E3
:20730000042483F8070383F80643DAE70134012083F8074383F80603D3E70029C0D193F89D
:207320002E320849203301EB8301BFE793F82B320449203301EB8301B8E700BF1892012012
:20734000F05101205C930120801A0600F08E01207C8F01201D4A10B448B91D4C92F8080326
:207360000B6823440B6098B15DF8044B704792F8093303B3012B16D092F808030B68154C2D
:2073800080F00100234482F808030B600028EBD192F82B324FF440700F4920335DF8044B18
:2073A00001EB830158E792F808030C4C80F0010082F80803D4E708680124054B82F80843D6
:2073C00003445DF8044B0B60704700BF1892012040420F0048E801005C93012020A107007C
:2073E0003F4A10B4B0B992F80A336BB192F80B138A081341DB070AD501F00101032A06D8A7
:20740000DFE802F0534B433B92F811335BBB5DF8044B704792F80B33013303F00F0382F8DD
:207420000B3333B192F80A330C682E4820440860DBE72D4882F80A33437A002B46D12B484D
:20744000C07818B143F0040382F80A3328480078C00732D592F810030028E5D043F00803CC
:2074600082F80A33E0E792F81E33224901EB83014FF400305DF8044BEEE61E4B03F130025E
:20748000002914BF19461146F2E71B4B03F1180200290CBF19461146EAE7164B03F1080213
:2074A000002914BF19461146E2E7124B03F11802002914BF19461146DAE7D2F80C03002872
:2074C000C8D043F0010382F80A33C3E792F80933002BB4D00220034682F80A03AFE700BFC0
:2074E00018920120A0860100BC8F0120F88E0120F68E0120FCD805080CD9050870B4322198
:20750000022640F203154FF4FA7446F201420023C6708580C48001814281038070BC704780
:20752000F8B5224C94F82013621892F82423002A3AD000231E4D4A1C0133A5FB0261490876
:2075400001EBC101511A621892F824230AB1092BF1D1CBB284F8203302680C260025571C96
:20756000076001EB41071670026801EB8701561C066015700D2205680E4E6F1C3144076050
:207580002B7037F021FB94F820130120084B0A182144A3FB025381F82403C34003EBC30309
:2075A000D31A84F82033F8BD0B46D5E718920120398EE33848950120024B0146D3F8A80398
:2075C00026F0A6BB1892012008B5044BD3F8AC0326F078FBB0FA80F0400908BD1892012067
:2075E000044B93F831310BB11EF060B8024B1888704700BF18920120A48F0120084B07EEA3
:20760000900A93F8CD304BB9F8EEE77A9FED057A9FED050AA7EE870A44F04CBA704700BF81
:20762000189201206766E63F0000004210B5184CA379CBB194F82230C0B2DFED166A07EEF9
:20764000903A154BF8EEE77A03EB8000838986EEA77A07EE903AF8EEE77A67EE277AFDEEC3
:20766000E77A17EE900A10BD0C4B1B6813F000630CD0C0B2FFF74AF86423808910FB03F0E9
:2076800094F822305B0890FBF3F0ECE71846EAE7D4490120000048434C4E0020D85101206C
:2076A00008B5FFF7C3FF3C2390FBF3F008BD032811D8DFE800F00A0C0206084BD3F8B40305
:2076C0007047074B1B78DB0701D426F003B9034BD3F8B00370470020704700BF18920120A1
:2076E000F68E0120F0B52B4F0E462B4A83B03B682A4D82FB0312DC17B5F8DC33C4EBA2041A
:207700003F89A4B2A3420CD1D5F8E0332449F31AB5F8E4238B4298BFBA4214BF0123002341
:2077200034D0036834210022019003F1010CC0F800C019702146036803F1010CC0F800C085
:207740001A7037F085FA3946019837F081FA47F6FF71019837F07CFA47F6FF71019837F0EF
:2077600077FA47F6FF71019837F072FA47F6FF71019837F06DFA01980221F5F765FC0123BE
:20778000A5F8DC43A5F8E473C5F8E063184603B0F0BD00BFD88F01206766666618920120D0
:2077A00080841E0002680E2170B5561C7F250024066015700268551C05601470F5F744FCD4
:2077C000012070BD2DE9F0416A4F84B06A4D0446D7F800800E4640460CF061FB85F8E6033F
:2077E000B8F1000F0AD00DF1090202A940460CF086F9002840F08D8095F8E60300231946E5
:20780000ADF808308DF80A30431E0022FF208DF80C10DBB2ADF80E208DF80B00FD2B04D994
:207820000023184604B0BDE8F0819DF80830042B00F09480052B00F09780032B00F0968092
:20784000022B00F08A80012B00F092809DF809300DF10E023868013B9DF80A108DF80930AE
:207860000CF0B6F895F8E633032B74D0042B0CD1424A9DF80A000121002301E012F8011FBF
:2078800081426ED20133082BF8D1D5F8E8230DF10808029B3A4F9A4250D023680D210022D2
:2078A000581C2060204619702368591C21601A7023689DF80820591C21601A7023689DF8F2
:2078C0000920591C21601A7023689DF80C20591C21601A7023689DF80A20591C21601A7069
:2078E000BDF80E1037F0B4F923689DF80B202046591C216007211A70F5F7A6FB0123C5F81A
:20790000F06398E8030087E80300184604B0BDE8F08101A940460CF0E9F800283FF46CAF74
:2079200040460DF10A010CF0E7F800283FF464AF019995F8E60301F0010165E77A68D8F86E
:2079400004309A42A9D1D5F8F0330E4AF31A93427FF666AFA1E70C4A8BE703228DF80820C7
:2079600074E78DF80A3090E70122F7E70222F5E70422F3E7588F012018920120105E060826
:207980000096012080841E001C5E0608C74B1B682DE9F04F814613F0800083B000F0788136
:2079A000C34B187810F0020000F07281DFF820A39AF81430052B40F27281DAF80030BD4C74
:2079C000002B0093BC48B8BF5B42BC49A4FB0352920D00FB023302EB8202C3EB031302EBE7
:2079E00082029B0084FB0354DD17C5EBA45500FB053305EB820581FB0321ADB2DB17C3EBAC
:207A0000A111C5B10020AE4F0446A7FB053CC3B22E4601304FEADC0C9A00092E0CEB8C0362
:207A2000A5EB43031FFA8CF59BB203FA02F344EA0304EAD8250489B2C1B10020A04F044671
:207A4000A7FB013CC3B20E4601304FEADC0C9A00092E0CEB8C03A1EB43031FFA8CF19BB220
:207A600003FA02F344EA0304EAD82543DAF804B0904C8BEAEB739048904AA3EBEB73A4FB43
:207A80000361890D00FB013301EB8101C3EB031301EB81019B0084FB0364DE17C6EBA456FC
:207AA00000FB063306EB810682FB0312B6B2DB17C3EBA212CEB10021814F0846A7FB063E28
:207AC000CBB2344601314FEADE0E4FEA830C092C0EEB8E03A6EB43031FFA8EF69BB203FA13
:207AE0000CF340EA0300E9D8060492B2CAB10021734F0846A7FB023ECBB2144601314FEA7B
:207B0000DE0E4FEA830C092C0EEB8E03A2EB43031FFA8EF29BB203FA0CF340EA0300E9D84F
:207B20000643DAF80830664A002B18460193B8BF5842644C6449A2FB0030030AA4FB0343F8
:207B4000DB0901FB03F1C1EBD00189B2C1B1002496462746AEFB013CE3B20A4601344FEA81
:207B6000DC0C9800092A0CEB8C03A1EB43031FFA8CF19BB203FA00F347EA0307EAD8B9B2BF
:207B8000BAF81080B8F1000F1AD00024DFF830E12746AEFB083CE3B2424601344FEADC0C28
:207BA0009800092A0CEB8C03A8EB43031FFA8CF89BB203FA00F347EA0307EAD81FFA87F82C
:207BC000BAF812303E4AA2FB0307FF08632F28BF6327092B67D94FF0000C92466046AAFB96
:207BE000073E5FFA8CF33A460CF1010C4FEADE0E9C00092A0EEB8E03A7EB43031FFA8EF7EA
:207C00009BB203FA04F340EA0300E8D8C4B2009B019A002BCCBF39233823BBF1000F4FEA29
:207C2000226738DD27F07F07284A3B43934543F00207C8BF43F00607D9F8003016200022E5
:207C400003F1010CC9F800C018704846D9F8003003F1010CC9F800C01A7036F0F9FF2946F2
:207C6000484636F0DFFF3146484636F0DBFF4846414636F0EDFFD9F8003001201A18C9F831
:207C800000201C70D9F800301A18C9F800201F7003B0BDE8F08F27F07F071F43CCE70020EC
:207CA00003B0BDE8F08F0024B1E700BFD85101207C8F01206BCA5F6B806967FFD34D62101C
:207CC000CDCCCCCCC55A7C0AA0860100FFC99A3BF0510120AE4B1B682DE9F047064613F090
:207CE000800084B000F0A180AA4B187810F0020000F09B80DFF8B4E29EF81410052940F2A6
:207D00009980632900F29480002089B2A24F0446A7FB013CC3B20D4601304FEADC0C9A008F
:207D2000092D0CEB8C03A1EB43031FFA8CF19BB203FA02F344EA0304EAD8E4B2DEF8083045
:207D4000964AD91782FB0323C1EB633399B2002900F019810025DFF840C22846ACFB013824
:207D6000EBB20F4601354FEAD8089A00092F08EB8803A1EB43031FFA88F19BB203FA02F3CF
:207D800040EA0300EAD8C7B2BEF80E304FF4F365834942F20F7005FB03F5A1FB0535C5F3E7
:207DA0008F1585424AD8D5B10021DFF8ECE10846AEFB0538CBB2AC4601314FEAD8089A0063
:207DC000BCF1090F08EB8803A5EB43031FFA88F59BB203FA02F340EA0300E9D885B2714BD4
:207DE000D3E9FE2313433ED14FF0FF3833682946172000225D1C35601870304633685D1C48
:207E000035601A7036F024FF4146304636F00AFF3368304606215A1C32601C7033685A1CF1
:207E200032601F70F5F710F9012004B0BDE8F087992483E7002004B0BDE8F0870021DFF82C
:207E400058C10D46ACFB0032D20802EB8203A0EB430390B29BB28B400431102945EA0305C1
:207E6000F0D1ADB2BBE701A837F0C2F99DF80810002900F08A800020DFF81CE18046AEFB82
:207E80000139C3B28C4601304FEAD9099A00BCF1090F09EB8903A1EB43031FFA89F19BB284
:207EA00003FA02F348EA0308E9D84FEA08289DF80920E2B10021DFF8E0E00846AEFB023A2D
:207EC000CBB2944601314FEADA0A4FEA8309BCF1090F0AEB8A03A2EB43031FFA8AF29BB23B
:207EE00003FA09F340EA0300E8D848EA00089DF80A204FEA0828E2B10021DFF89CE00846E5
:207F0000AEFB023ACBB2944601314FEADA0A4FEA8309BCF1090F0AEB8A03A2EB43031FFADE
:207F20008AF29BB203FA09F340EA0300E8D848EA0008BDF80C304FEA08181B4A632BA2FB7E
:207F400003124FEA52127FF651AF0021DFF848E00846AEFB023ACBB2944601314FEADA0A01
:207F60004FEA8309BCF1090F0AEB8A03A2EB43031FFA8AF29BB203FA09F340EA0300E8D85A
:207F800048EA000832E70F46FEE688468FE700BFD85101207C8F0120CDCCCCCC89B5F81461
:207FA000D34D6210189201201F85EB51F0510120F8B53B4B054601687E27B3F90034002690
:207FC000384A481C03EBC3032860FF2082FB0342DC170F702B68C4EB62045A1C20342A6030
:207FE000A4B21E70FEF792FB2F4B00284DD01B78B0F90C1023BBA1F57A722C4B9A4246D833
:020000040801F1
:208000002B48B0FBF1F189B2284636F0FDFD294BDB7A7BB11DF04AFB0146284636F0F4FD84
:208020002146284636F0F0FD28460821F5F70CF80120F8BD204B2846198836F0E5FDEFE7A3
:208040001E4B1E78002ED6D000231D4800EB830201339289B3421144F8DB1A4B07EE901AE5
:208060009FED196A93F82230F8EE676A07EE103AB8EEC77AC6EE077A67EEA67AFCEEE77A42
:2080800017EE901AB1FBF6F1B5E71B7813B94EF69C21B9E7094B1E78002EF8D00146D3E721
:2080A00018920120676666660C1500201783930300879303808F0120A48F012070070020B3
:2080C0004C4E0020D449012000004843244A00234361D2F8DC1041F45C5130B541F02C010D
:2080E0000124C2F8DC104471D2F8D41004FA03F50133112B41EA0501F8D121F4F0314FF479
:2081000020634FF0A064C2F8D4105022C38040F6012314490381144BA0F856206FF07E427F
:208120000360142303718023037642F6140303824FF6FF73438303F58C03C36140F20123C3
:20814000C0E9161203840023084A80F8223080F8333080F84430A0F86830C0E9184230BDA1
:2081600018920120C4FF00FF98086400180B0C0008B5A0F101030228B3FA83F34FEA531301
:2081800001D0184608BD0F2019F05CFC28B9054B1B7803F00103184608BD0F20BDE8084061
:2081A00019F0DABCF68E012038B505468022002105F1800444F062FF00213822204644F05C
:2081C0005DFF00230B4951F8232044F8232001330E2BF8D11E22084905F1C00044F0DCFE36
:2081E0000B22064905F1E40044F0D6FE032385F8EF3038BDFCD8050834D9050854D9050835
:20820000034B01220349B3F90830406837F0A6BD50060120D45D060837B504462A4800EB42
:208220004303B3F8CE5005F00F0049B1022804F101011DD8002814BF9C239B2323700C46BE
:208240000AB3C5F30315FFF732FA204B3C21012DB0FBF3F3B3FBF1F201FB123315D0022D02
:2082600023D01B49204603B0BDE8304037F076BD032806D1174B1B7803F00103653BDBB204
:20828000DCE72023DAE71546DDE742F210716425B0FBF1F1B1FBF5F005FB10100E49009095
:2082A000204637F05BFD03B030BD0C490A25B0FBF1F1B1FBF5F005FB10100949009020462F
:2082C00037F04CFDEFE700BF1892012040420F002E5E0608F68E0120385E0608A086010033
:2082E000475E0608037801224068053B114693E71D4B1E499A68B1F8C83007EE902A9FEDC7
:208300001C7A4068F8EEE76A07EE903AF8EEE77A67EE877AF4EEE76AF1EE10FA02D8154938
:2083200037F01CBD934202DA134937F017BD9B1A124A07EE903AB8EEE77AD1EDEC7A3C21DD
:20834000F8EE677A67EE277A87EEA67AFDEEC77A17EE903AB3FBF2F3B3FBF1F201FB12336B
:20836000074937F0FBBC00BFD88F012018920120CDCCCC3D565E06085C5E060840420F0000
:208380002E5E0608064B07491A88074B40681B68534342F2107293FBF2F237F0DFBC00BF44
:2083A000A48F0120625E0608D88F0120054A064992F8053492F8042401334068013237F0CA
:2083C000CDBC00BF18920120675E06080B4B0A224FF4B4714068B3F9043093FBF2F31A01B7
:2083E00002F5B9521432B2FBF1F2C2F10802044902F00F02603237F0B1BC00BFA0520120A0
:208400006D5E0608034A072303499268406837F0A5BC00BFD88F0120745E060807B5144A55
:20842000406892F81414B2F81634012909D10093104992F818347B2237F090FC03B05DF8D0
:2084400004FB022906D17B220B4903B05DF804EB37F084BC0A220949534340F2FF32B3FBA7
:20846000F2F39BB27B22092B28BF0923EDE700BF189201207A5E06082F5F0608845E060816
:2084800013B54468FEF796FC0F4B02461B789B0712D50E4B93F823140D4B59B19889FEF790
:2084A00095FC0C49034600922046702237F056FC02B010BDD889F2E700902D237022064910
:2084C000204637F04BFCF3E77C8F012018920120F0510120E25E06088A5E06082DE9F0410A
:2084E000404F86B090F800C006463C78BCF1170F416890F803E00CBF4FF098084FF089080E
:2085000014F0040405D0BCF1170F374B0CBF5C681C6884EAE473354DBEF1010F01F1010019
:20852000A3EBE473B3FBF5F205FB123345D0BEF1020F46D181F800803C21BCF1170F01FB6B
:2085400003F3B3FBF5FE05FB1E3301FB03F3B3FBF5F105FB1135264BB5FBF3F528D1002C39
:20856000B4BF572345230593222302912149CDE903532723CDE900E3082337F0EFFB3378F6
:208580001D495A0903F01F0301EB8201012202FA03F33A78D1F8280402F00602042A0CBFDF
:2085A000034320EA0303C1F8283406B0BDE8F081002CB4BF53234E23D5E74FF47A75B3FB62
:2085C000F5F3002C81F8008002DA2D24881C4C700A4C0B49BEF1000F08BF214637F0BEFB8B
:2085E000CDE700BF7C8F0120F05101208096980040420F00A15E060818920120915E060866
:20860000995E06080D4B1B681B0137B514D50C4C4568D4F8303493F90100FEF7EFFF94F858
:20862000CD2003460749002A28460CBF0D220E2200927A2237F092FB03B030BDD851012026
:2086400018920120B75E0608034B0449D3F83424406837F083BB00BF18920120C05E0608AB
:20866000044B1B78DB0703D40349406837F076BB704700BFF68E0120C45E060807B5094AB9
:208680000949B2F906300193B2F904300093B2F90230B2F90020406837F060FB03B05DF8C7
:2086A00004FB00BF14490120CD5E060837B50A4C4568B4F90004FEF7A1FF94F8CD2003464E
:2086C0000649002A28460CBF0D220E2200927A2237F044FB03B030BD18920120E15E06083D
:2086E000084BD3F84424002A0ADD074B03EB82031A6E2AB1054B0649DB68406837F02EBB21
:20870000704700BF18920120FCD8050850060120EA5E06081FB5938802939378019353787C
:20872000009313780A46034937F018FB05B05DF804FB00BFF25E0608034B0449D3F848244D
:2087400040681432E6E700BF18920120055F0608034B0449D3F8482440680832DAE700BF2E
:2087600018920120095F0608034B0449D3F8482440680E32CEE700BF189201200D5F060845
:208780002DE9F0472DED028B82B0924607460C469DF8302099469DF83480002B52D0022BB5
:2087A00014BF0A25642507EE905AF8EEE77A27EE808A002A48D0B0EE480A43F07BF907EE1B
:2087C000900AF8EEE77AF0EEE77AFDEEE77A17EE906AB6FBF5F205FB12660CB13C70012490
:2087E000B5EEC08AF1EE10FA05D552EA060302D02D233B5501349AF800103819144B002922
:2088000014BF5146194637F0A9FA2518B9F1000F0AD04A460F49684637F0A0FA7819324695
:20882000694637F09BFA0544B8F1000F02D007F805800135002328467B5502B0BDEC028BF7
:20884000BDE8F0870125AEE7F0EE487ABBE700BF115F0608165F06081A4B1A6812F0200F27
:2088600002F0040313B5446825D0174A1278920721D5164BB3F90000FEF7C0FADFED147A06
:20888000144B204620EE270A134A93F8CD30B5EEC00AB0EEC00AF1EE10FA4CBF76217521F9
:2088A000002B0CBF99239F23019301230093FFF767FF02B010BD002BDBD12D2222704268BC
:2088C0005370F6E7F08E01207C8F0120E48F01200AD7233C1892012092AC06081FB5184B0B
:2088E0009FED187A1B88184A07EE903A9FED170A92F80923F8EEE77A4468F4EEC77A27EE08
:20890000800AF1EE10FAACBF01230223022A14D08DED030A02931CF0C9FEFEF7BAF9029BEC
:2089200001469DED030A01220620CDE90020084A2046FFF725FF04B010BD9721F3E700BF96
:20894000A48F012000007A44189201200AD7233C92AC0608114BB3F84C34B3F57A7F07B5CA
:20896000406806D201220E4903B05DF804EB37F0F5B907EE903A572200239FED0A0AF8EE50
:20898000E77ACDE90032012327EE800A064A1946FFF7F6FE03B05DF804FB00BF18920120A1
:2089A0001E5F06086F12833A92AC060873B5194E0546406896F86834052B07D01F231E226D
:2089C000154902B0BDE8704037F0C8B9134C1E221349237D00931F2337F0C0F996F8223159
:2089E000ABB16B6820220021DFED0E7A1A54638A441C686800EE103A01230B4A2044B8EE4B
:208A0000C00ACDE9003120EE270AFFF7B9FE02B070BD00BF18920120265F0608F05101205B
:208A20002D5F06080AD7233C92AC060807B5012347220649CDE90032054A91ED000A002198
:208A40004068FFF79DFE03B05DF804FB8896012092AC06080B4BDFED0C7A93ED000A9A235C
:208A6000B8EEC00A07B520EE270A0021074AB0EEC00ACDE9001302234068FFF781FE03B0F3
:208A80005DF804FBD88F01200AD7233C355F060813B504461CF00AFE0E4B00EE100A6468C5
:208AA00093F80933022B13D0FEF7F3F80146B8EEC00ADFED097A00230622204620EE270A09
:208AC000CDE900320223054AFFF75AFE02B010BD9721ECE7189201200AD7233C92AC06088B
:208AE00013B50378134A1A2BDFED137A134C0CBFB2F90220B2F900201A2B4FF0010300EE00
:208B0000102A0CBF152114210022B8EEC00ACDE9003220EE270A0A4A4068B5EEC00AB0EE25
:208B2000C00AF1EE10FA48BF2246FFF729FE02B010BD00BFA0520120CDCCCC3D395F06085D
:208B40003F5F0608194B37B51A68446812F0200F02F0040320D0164A127892071CD5154AFE
:208B6000C17892F8CD30D2F87404002B0CBF0F250C25FEF743F90123DFED0F7A20460093F5
:208B8000CB1A20EE270A0D4A18BF01237F210195FFF7F6FD03B030BD002BE0D17F222D21D5
:208BA00022704268517042689370F3E7F08E01207C8F0120189201200AD7233C92AC06080F
:208BC00013B5044608461146FEF718F9164B93F8CD30002B0BBF4FF4A5534FF47A737E22EF
:208BE0007D2207EE903A0CBF0F230C23F8EEE77AF4EEC07AF1EE10FA13DC80EE270AF2EE31
:208C0000047AB4EEE70AF1EE10FAACBF012302230192002220460092044AFFF7B1FD02B055
:208C200010BD1A460023F3E71892012092AC06080C4B10B41B78446803F00303032B06D19B
:208C4000094B204611225DF8044B1988B8E711232D22237043685A70002243689A705DF88C
:208C6000044B70477C8F01207E8F0120094B40681B7803F00303032B07D1074B7122D3F856
:208C800078146423B1FBF3F19AE72D237122034937F064B87C8F0120189201208C5E06084F
:208CA000224B1B885A0510B5446805D520462049BDE8104044F0C0BA180505D520461D49C5
:208CC000BDE8104044F0B8BA590605D520461A49BDE8104044F0B0BADA0705D520461749E3
:208CE000BDE8104044F0A8BA9B0705D520461449BDE8104044F0A0BA252018F02DFF28B1D5
:208D000020461049BDE8104044F096BA0E4B93F87C342BB120460D49BDE8104044F08CBA80
:208D200020460B49BDE8104044F086BAC4520120455F06084A5F06084F5F0608545F0608F3
:208D4000595F06085E5F060818920120635F0608685F0608074B93ED6E7AD3ED6B7AB4EE11
:208D6000E77AF1EE10FA03DD0349406844F064BA704700BF083100206D5F060810B50C46C3
:208D8000A0B9174A174892F87D1423680344236001B110BD92F82B324FF480601249203313
:208DA000BDE8104001EB8301FEF756BA11F046FF322808DD206801210A4B094A034482F8B1
:208DC0007D14236010BD064A142892F87D14C8BF064881F00101D8BF054882F87D14D4E719
:208DE0001892012040420F005C93012020A1070048E8010010B504461AF0C6FF04220346C1
:208E000002496068BDE8104036F0A8BFD45D06082B4BF0B51C6887B02A4E074620463178D4
:208E20000AF052FE7178054620460AF039FE002203460592B2788DF813206CB1039005A9DB
:208E400020460AF053FE327A039B2AB10DF1130120460AF051FE039B9DF81310ECB1E1B1F6
:208E6000194A1268914218DC184A02EB8102D2F880442620039318F06FFE0599039B70B938
:208E800011F0010F14BF502200228907786808D50F4936F063FF07B0F0BD0E4CE9E7442239
:208EA000F3E732B10C49CDE900422A4636F056FFF1E72A460949009436F050FFEBE700BF89
:208EC000588F0120D8520120FC8D012018920120705F0608CD650608785F0608845F0608D7
:208EE000F8B50446417882782C48237890F8E950302B2B4B05F1FF354FEA85052B4448D1B2
:208F000093F8E85093F8E96000EB85054FF47A7700EB86004FF0030CD5EDAE7A40F2CF75F2
:208F2000FDEEE77A17EE903AD0EDAE7AAB42FDEEE77AA8BF2B4617EE900AB3F57A7FB8BF69
:208F40004FF47A73A842A3F57A73A8BF2846C3EB0313B842B3FBF7F3C3F10E03B8BF38468D
:208F6000DBB2A0F57A70B3FBFCFCC0EBC00062440CEB4C0ED2B2A3EB0E03B0FBF7F70833E6
:208F800039442046DBB2C9B2F4F7E2FD00232373F8BD93F8EA5093F8EB60B5E718920120AC
:208FA000FCD805082DE9F04790F80290044690F80180002609F10207FFB2002508EB060A14
:208FC000032E1BD108F10301022DC9B20ED10B233A462046F4F7BCFD0135052DF0D10136D6
:208FE000072EEAD100232373BDE8F08709EB050216232046D2B2F4F7ABFDEDE7022DEBD13C
:2090000017233A465FFA8AF12046F4F7A1FDE3E770B504466FF00205A278132361782046A5
:2090200052FA85F2EEB207390135D2B2C9B2F4F78FFDA27861781323324420460731D2B220
:20904000C9B2F4F785FD042DE6D161780323A27820460639C9B2F4F77BFD61780223A2788C
:2090600006312046C9B2F4F773FD0023237370BD2D492DE9F84391F8D830054691F8D92072
:2090800091F8E71003EB830302EB8202274800294FEA43034FEA4202B0F9004014BF4FF0DC
:2090A000FF310121C2F100084C43444503DB9442A8BF1446A046B0F902205C424A43A24256
:2090C00003DB9A42A8BF1A4614461BB11922544394FBF3F4293C4FEA88066FF003074FF0CD
:2090E0000909002E3346B8BF06F13F03C4EBA313512B0FD8284693FBF9F101EBC1029B1AF5
:20910000AA780A446978803B3944D2B2DBB2C9B2F4F71EFD0137A6EB0806052FE1D1002354
:209120002B73BDE8F88300BF18920120A052012010B5044611F0BEFD6422074902FB00F343
:2091400060680122C3F38F23632BBDE8104028BF632336F003BE00BF2F5F06082DE9F84339
:209160000546002415F044F91C4E07464FF08808DFF86C9033786968A342214403DC00231D
:209180000B70BDE8F88337B3D6ED427A09EB8403FDEEE77A17EE900AD3ED007AFDEEE77ADF
:2091A00017EE902AD6ED437AFDEEE77A121AD20017EE903A1B1A204692FBF3F3C3F188030A
:2091C0000B70FEF733FAB0F57A7F02DA6B6853221A550134CEE781F80080FAE77007002066
:2091E00060300020374B13B5C17804469A680229354B9B8941D0032945D0012905D19A1A1B
:209200009A42A8BF1A4622EAE272D3B19A1A0B209A42A8BF1A46B3FBF0F322EAE27207EE5F
:20922000902AB8EEE77A07EE903AF8EEE77AC7EE276AFAFE667AFCEEE77ACDED017A9DF834
:20924000043062688A21117001229342ACBF8B208D206168885401320C2AF6D162688F21DA
:2092600011735A1E092A03D8626813448E225A70636800225A7302B010BD9A1A9A42A8BF19
:209280001A4622EAE272ABB107EE902AB8EEE70ADFED0E7A20EE270A07EE903AF8EEE77AD3
:2092A00080EE270A42F006FC64280346A8BF642323EAE37307220649606802B0BDE81040CE
:2092C00036F04CBDD88F0120BC8F01200000C8428D5F060810B50446132018F03DFC48B3E9
:2092E0000CF06EFA30B9606810221349BDE8104036F034BD0CF090FA034660682BB110221A
:209300000E49BDE8104036F029BD0D4B93F8A524022A4FF0100208D1D3F8C034002B04DB2A
:209320000849BDE8104036F019BD0749BDE8104036F014BD10BD00BF945F0608985F06081D
:20934000189201209C5F060801A10608244B1A6812F0200213B5044624D0224B1A7812F06D
:2093600001021FD0204B1A7812F002021AD01F4BD88963282AD9FDF729FD1D4BB2EE040A85
:2093800007EE100AD3ED007A1A48F8EEE77A67EE807AB8EEC70A87EE800A43F0DDFF42F0D5
:2093A00089FB0246144B42F20E716068541E93F8CD30002B0CBF7E237D238C4208D8009395
:2093C00007230E4936F0CAFC02B010BD0022E9E707220B4902B0BDE8104036F0BFBC00BF2B
:2093E000F08E0120F68E01207C8F0120F0510120D88F0120E096012018920120A15F0608A3
:20940000AA5F0608F8B52D4F0A240546B7F9002092FBF4F484EAE473A3EBE4739BB25A2BD2
:2094200005D90A32CCBFB4236FF0B3031C1B244E96F8102332B9234B1B78DB0729D417F05F
:2094400093F930BB96F8D434B32B02D817F08CF9F8B9B7F902100A2391FBF3F304B9C3B178
:20946000002B84EAE4706A68B8BF5B42A0EBE4709BB2B3EB400F13DAB0EB430F10DA09290A
:2094800008DD002CCCBF6E23622313706B6800225A70F8BD002CCCBF6A2366231370F5E7F7
:2094A000834205DD0929CCBF602368231370EDE7002CCCBF6C2364231370E7E7A0520120B2
:2094C00018920120F68E012030B585B0054601A835F08EFE044618B92870204605B030BDA2
:2094E000044A012301A92846B2F9002036F04CFCF3E700BF245301204068E5E773B50D4D82
:2095000004461646009102460023022128682AF07DF9094B224614210093002328682AF015
:2095200075F9002322461621286800962AF06EF902B070BDD0520120B5AE06082DE9F04378
:20954000B44C8BB094F8D634DBB1B34F4FF0010CB249DFF818E3B24EB24A94F8D734D4F834
:20956000DC80FD18172B31D984F8D73494F8D63494F8D824002A40F0AC82012084F8D83458
:2095800021E094F8D854002DDFD0A74A29461068027A9542A8BF1146954201D2013101234D
:2095A000521A02EBD272C2F3470213B984F8D624CBE7531C022184F8D6349C4B0093002367
:2095C0002AF024F900200BB0BDE8F08315F8010B01330CFA00F9DBB219EA080FC2D094F850
:2095E000D65484F8D7341728B7D8DFE810F0180036004F0079008F00B200D300F3004101C6
:20960000500161015D007201BA01CD01E301F80103029F0013023602410254022A0202AEFB
:209620003046FFF751FF18B98149304636F096FB7D48002300962A46022100682AF0E6F835
:2096400094F8D634784A01331268DBB2127A84F8D6349A428CD90020B5E7B4F8CE200023AB
:2096600002A812F00F02194618BF0122FEF7D4FDB4F8CE3003F00F026E4B284603EB8203C6
:2096800002AAD3F8F810FFF739FFD9E7B4F8D0200123002102A812F00F0218BF1A46FEF793
:2096A000BBFDB4F8D030E5E7D4F8C403FDF7A6FB94F8CD30DFED607A0021002B5F4A20EE20
:2096C000270A02A80CBF0F230C23019301230093FFF756F802AA5A492846FFF70FFFAFE79D
:2096E00013681B067FF539AFB4F9B803FDF76EFB0246FDF75FFB5349034602A836F02EFB39
:2097000002AA51492846FFF7F9FE99E7136818067FF523AFB4F9C81302A80022FFF750FAB5
:2097200002AA4A492846FFF7E9FE89E713681B067FF513AFD4F87814642302A80022B1FB06
:20974000F3F1FFF73DFA02AA41492846FFF7D6FE76E7B4F9BA334FF0060CDFED377A0021A4
:2097600000EE103A0123354A02A8B8EEC00ACDE9003C20EE270A0223FFF702F894F83101F0
:20978000344B02AA3449002808BF19462846FFF7B5FE55E7B4F8BC330627DFED277A00212A
:2097A00000EE103A0123254A02A8B8EEC00ACDE9003720EE270A0223FEF7E2FF94F83101DF
:2097C000264B02AA2649002808BF19462846FFF795FE35E7FDF704FF07EE900A01230626C6
:2097E000B8EEE70ADFED147A144A002102A820EE270ACDE900360223FEF7C2FF94F831018B
:20980000184B02AA1849002808BF19462846FFF775FE15E71892012004DA0508C408002015
:20982000BC8F0120D8510120D0520120F45F060804600608FCD805080AD7233C92AC0608EF
:209840000B600608186006081D6006082760060834600608C15F0608B45F0608DA5F0608B1
:20986000CD5F0608DE5F0608E65F0608F08E012002A994F8C003F3F73FFB974902A843F096
:20988000BFFC02AA95492846FFF738FED8E6B37A002B3FF462AEB4F9BE239A23904902A8C2
:2098A00036F05CFA02AA8F492846FFF727FEC7E6B37A002B3FF451AE8B4A0723884902A86E
:2098C000926836F04BFA02AA88492846FFF716FEB6E694F8A534002B3FF43FAE032B3FF481
:2098E0003CAE0BF06DFF94F8A534012B21D0022B30D188B3F8F730FD4FF4FA62066841F2D0
:20990000A873B6FBF2F67A4AD0584FF47A22B0FBF2F0301A642277495043B0FBF6F202A8DB
:2099200092B236F01BFA02AA73492846FFF7E6FD86E688B1F1F728FD074637F041FABE8852
:209940007A88B21A466802FB066636F047FF800AB60ADFE700B1FFDE684902A836F0FEF9A0
:20996000E1E794F8A534022B7FF4F7ADD4F8C0040028FFF6F2AD02A9F3F7BEFA02AA604988
:209980002846FFF7BBFD5BE6DEF8003098077FF5E4AD0123472294EDF30A002102A8CDE934
:2099A0000032584AFEF7ECFE02AA57492846FFF7A5FD45E6B4F9D003FDF720FE94F8CD305C
:2099C00002464749002B02A80CBF0D230E2336F0C5F902AA4D492846FFF790FD30E602A9D6
:2099E000D4F8D403F3F788FA02AA49492846FFF785FD25E6B4F8D82302A8464936F0AEF97C
:209A0000354902A843F0FCFB02AA43492846FFF775FD15E6CB68002B7FF79FAD0A69002A2E
:209A200009DD3E4902A836F099F902AA3C492846FFF764FD04E63B4A28463949FFF75EFDB1
:209A4000FEE5B4F9DA2302A8374936F087F902AA36492846FFF752FDF2E502A9D4F8340445
:209A6000F3F74AFA02AA32492846FFF747FDE7E53C21D4F8383402A8B3FBF1F3B3FBF1F2BB
:209A800001FB12332B4936F069F902AA2A492846FFF734FDD4E594F8CD30D4F83C2473B93B
:209AA00040F249617E2302A8B2FBF1F20C4936F055F902AA21492846FFF720FDC0E54FF4A7
:209AC0007A717D2302A8B2FBF1F2054936F046F9EFE7012077E500BF925F0608446006084B
:209AE000186006084D600608D88F0120596006088C7501208F5F0608686006086260060812
:209B00007160060892AC06087C600608886006089560060862AA0608A1600608AA600608F6
:209B2000AF600608B8600608EE5E0608C1600608CE600608DC600608E5600608F76006081B
:209B4000714B2DE9F0431F6883B0002F54D0FF238DF803308DF80230002875D16B4B93F8B3
:209B6000D924002A4BD093F84051002D44D0002193F8DE34664C8B42664862690B4614BF6C
:209B80004FF00F0E8E4602F0010C94F8108000F1F0020F4611E0984553D3BCF1000F50D171
:209BA00074461E26013316809770DBB2D470013104328D4220DD052B1ED850F8044B2404EC
:209BC000F5D5002BE7D174467826EBE7012203EB82027169D2F8C4210192CA077AD593F852
:209BE000DE34002B14BF0F23002301A94FF400408DF80730FDF730FB03B0BDE8F083444E9B
:209C0000B3F8DA2441F228618A42DFD941F24F618A4261D941F276618A425FD941F29D6133
:209C20008A425DD941F2C5618A4268D941F2EB618A4266D941F212718A4294BF0B220D2201
:209C4000C5E700242646ADE7314E0DF102020C4638460DF1030109F052FF06F11001384611
:209C600009F04AFF06F11401384609F03FFF9DF803909DF8028038464946424609F0BCFE5A
:209C80007369317C03F00105204B05EB410593F8D924A3F8DA0405EB091505EB0825ADB216
:209CA00022B9B3F8DC24AA421CD00F2293F8DE04013A1949A3F8DC54D2B2256880F00100BE
:209CC00083F8D924294483F8DE042160002A7FF44AAF94E7FF2388E7022278E7032276E71A
:209CE000042274E793F8DE0425680B4980F00100A3F8DC24294483F8DE04216080E70622AF
:209D000065E70A2263E700BF588F012018920120500601205C930120400D030001297FD996
:209D2000F0B5037815465D4A83B0C3F3411403F00F06032C147000F0858013F0100306D027
:209D4000012C6FD0052913D8002003B0F0BD544C94F8B025002AF7D094F8B125013202F085
:209D60000F02B24255D0184684F8B03503B0F0BD437847184A4C811D84F8AC354388A4F888
:209D8000A8358388C02B74D8464A4FF0000C01201344C4F8A025A4F8AAC5C4F8A43584F8B4
:209DA000B0059A1A7F1A84F8B16597425CDB3E4F002A52D1B4F9A835FA2B02D10DB10523BD
:209DC0002B703A4E3946D4F8A0754FF0000C384D06F5A073C4F8A47536482A46314F6B6014
:209DE00001AB8069C5F808C0C4F8A0752E6084F8B0C5CDF804C01EF073FF013048D0019B0B
:209E00000BB1002098472B680120C5E9006303B0F0BD4718D4F8A435411CD4F8A025C0E7C9
:209E20000020704702298FD043781D4C8278FF2BA4F8A82515D1042986D94718B0F8033064
:209E4000411D9FE7194B0024194A01201A49136003F8014BC2E9013177E7384634F0B4FE66
:209E6000A8E74718C11C8DE73A460F4834F0ACFE6AE70F4A4FF6F6750C4B0321B4F8A805D0
:209E800013601081012003F8011B558153605CE72B680222591C29601A70B0E7C191012071
:209EA00018920120F8960120B89701208090012070900120500601200000F6FF0B4B9B7A8F
:209EC00013B10B4B9B8B53B90A4B0B4AB3F9043082FB0312D817C0EBA20000B27047074A24
:209EE000906890FBF3F000B2704700BFBC8F0120808F0120A052012067666666D88F012004
:209F0000F8B50546174CEEB2D4F8B405C5F30727314623F0FDFE94F8B8353946D4F8B405D9
:209F20005E4084F8B86523F0F3FE94F8B835C5F30746D4F8B4052D0E5F40314684F8B875E9
:209F400023F0E6FE94F8B8352946D4F8B4055E4084F8B86523F0DCFE94F8B805454084F82F
:209F6000B855F8BD1892012070B504460B4DE6B2D5F8B405240A314623F0CAFE95F8B83575
:209F80002146D5F8B4055E4085F8B86523F0C0FE95F8B805444085F8B84570BD189201208B
:209FA00038B50B4C002305462421D4F8B40584F8B83523F0ADFED4F8B405542123F0A8FE4B
:209FC0002946D4F8B405BDE8384023F0A1BE00BF189201202DE9F043DFF868930E461546AA
:209FE00099F8B9452DED028B83B0002C00F02682013C89F8B9459FEDC88AC84FDFF84883E1
:020000040801F1
:20A000003378002B60D099F8B945002C5CD135B123F060FC2B68C01A002880F2D98399F809
:20A02000BA25002A40F07C8399F8BB05062840F2C981BB4B93F8211093F820408C4200F082
:20A04000ED8153F81C4F013099F8BCC54A1C34F81140C0B2D2B2644489F8BB055A71A4B2B6
:20A06000B4F5E06F00F0C48100F2A880B4F5806F00F0C58263D9B4F5A06F00F099823BD9B7
:20A08000B4F5A16F25D8601EC0B2FCF73FFBC8B1B0F90C301021A34A684603EB83038DF8CA
:20A0A000001092F8221003EB8303D9F800204908ADF801409B0093FBF1F3CDF8033090475C
:20A0C00000233370002D9BD103B0BDEC028BBDE8F083B4F5C06FF5D1934B9B89002B00F065
:20A0E0002C831BF0FBFA1022CDF803000024062368468DF8002048E2B4F5826F00F01782CA
:20A10000B4F5846F40F08880884B1B789A07D9D58749102020220423098800248DF8000013
:20A12000CDF803108DF802306846D9F800308DF8012098473470002D7FF462AFC4E7B4F5B3
:20A14000067FBFD8B4F5007F76D3A4F50073182BB8D801A252F823F0A7A4010895A40108FD
:20A1600095A4010895A4010895A4010895A4010895A4010895A4010895A40108C5A00108A3
:20A18000C5A00108C5A00108C5A00108C5A00108C5A00108C5A0010881A401086BA40108E5
:20A1A0006BA401086BA401086BA401086BA401086BA401086BA401086BA40108B4F5116FCE
:20A1C00000F0AB8100F28D80B4F5026F00F09B8151D9B4F5036F00F05B82B4F5046F7FF49D
:20A1E00071AF544B102240210024B3F9043068468DF80020082203EB83038DF801108DF8FD
